:100000000C94E4060C9428070C9428070C942807F9
:100010000C9428070C9428070C9428070C942807A4
:100020000C9428070C9424170C9428070C94280788
:100030000C941A350C9428070C9428070C94280764
:100040000C9428070C9428070C9488150C94280706
:100050000C94580C0C9428070C94220C0C94280730
:100060000C94821C0C9428070C94BE300C94280726
:100070000C9483770C9428070C947F72AD1CB21CEF
:10008000B71CC01CD71CEE1CFE1C0E1D2B1D171F01
:10009000EE1CD91DEA1D191E371E541EAE1E091F67
:1000A000E72079213622B6221F23CF23DA253726EF
:1000B000A426EE2639278627D727312890282A29F3
:1000C000C529BF2AE6300D315031C031D83119323F
:1000D000CC328C338C338C338C338C338C338C33E9
:1000E0008C338C338C338C33433345334A33623314
:1000F00064330A0D426174743A002025642043651C
:100100006C6C732000204C6F77207761726E696E83
:1001100067206C6576656C3A2025642E2564000A9C
:100120000D466F756E6420424C2D4374726C3A20FC
:10013000002564000A0D0A0D2121204D4953534921
:100140004E4720424C2D4354524C3A2025642021E6
:1001500021000A0D3D3D3D3D3D3D3D3D3D3D3D3D8B
:100160003D3D3D3D3D3D3D3D3D3D3D3D3D3D3D3DBF
:100170003D3D3D3D3D3D3D000A0D43616C69627270
:100180006174696E67207072657373757265207330
:10019000656E736F722E2E004F4B0A0D000A0D46CE
:1001A0006C696768742D74696D65202575206D69AB
:1001B0006E2020546F74616C3A2575206D696E0055
:1001C0000A0D436F6E74726F6C3A2000486561646B
:1001D000696E67486F6C64004E6F726D616C2028A9
:1001E0004143432D4D6F646529000A0D3D3D3D3D62
:1001F0003D3D3D3D3D3D3D3D3D3D3D3D3D3D3D3D2F
:100200003D3D3D3D3D3D3D3D3D3D3D3D3D3D3D0A51
:100210000D00416E676C654E69636B2020202020C5
:100220002020416E676C65526F6C6C20202020206E
:1002300020204163634E69636B2020202020202012
:100240002020416363526F6C6C20202020202020EE
:1002500020205961774779726F20202020202020AC
:1002600020204865696768742056616C7565202098
:1002700020204163635A202020202020202020209D
:1002800020204761732020202020202020202020B3
:100290002020436F6D706173732056616C7565200B
:1002A0002020566F6C74616765205B302E31565D7F
:1002B00020205265636569766572204C6576656CB1
:1002C00020204779726F20436F6D70617373202017
:1002D00020204D6F746F722031202020202020209C
:1002E00020204D6F746F722032202020202020208B
:1002F00020204D6F746F722033202020202020207A
:1003000020204D6F746F7220342020202020202068
:1003100020203136202020202020202020202020B6
:1003200020203137202020202020202020202020A5
:100330002020313820202020202020202020202094
:100340002020313920202020202020202020202083
:100350002020536572766F2020202020202020202E
:100360002020486F7665726761732020202020204E
:10037000202043757272656E74205B302E31415DB2
:1003800020204361706163697479205B6D41685D11
:100390002020323420202020202020202020202037
:1003A0002020323520202020202020202020202026
:1003B0002020323620202020202020202020202015
:1003C0002020323720202020202020202020202004
:1003D00020204932432D4572726F72202020202048
:1003E0002020424C204C696D697420202020202060
:1003F00020204750535F4E69636B2020202020202F
:1004000020204750535F526F6C6C2020202020200A
:10041000202021212120494E434F4D504154494233
:100420004C4520212121002E000A0D20444143206B
:100430006F7220493243204552524F522120436867
:1004400065636B204932432C2033567265662C203D
:1004500044414320616E6420424C2D4374726C0011
:100460005B25695D005B25695D002B204D696B7222
:100470006F4B6F70746572202B0048573A56256495
:100480002E25642053573A25642E256425632D417B
:1004900072746875722D50310053657474696E679B
:1004A0003A25642025730048617264776172652083
:1004B0004572726F7220313A2564202121004D6906
:1004C0007373696E6720424C2D4374726C3A2564D5
:1004D0002121004D69786572204572726F7221008A
:1004E000493243204552524F52212121004865692B
:1004F0006768743A202025356900536574706F6908
:100500006E743A2535690050726573737572653A79
:10051000253569004F66667365743A202025356974
:100520000048656967687420636F6E74726F6C0051
:1005300044495341424C454400486569676874200A
:10054000636F6E74726F6C0044495341424C454472
:10055000006163742E2062656172696E67004E6986
:10056000636B3A20202020202025356900526F6CD3
:100570006C3A20202020202025356900436F6D70C3
:100580006173733A202020253569004B313A2534B8
:100590006920204B323A25346920004B333A253408
:1005A0006920204B343A25346920004B353A2534F4
:1005B0006920204B363A25346920004B373A2534E0
:1005C0006920204B383A25346920004E693A253499
:1005D000692020526F3A253469200047733A253448
:1005E00069202047693A253469200050313A253482
:1005F00069202050323A253469200050333A25349E
:1006000069202050343A25346920004779726F20E0
:100610002D2053656E736F72004E69636B253469CC
:1006200020282533692E25692900526F6C6C2534EA
:100630006920282533692E256929004769657225B7
:100640003469202825336929004E69636B202534DD
:100650006920282533692E25782900526F6C6C207B
:1006600025346920282533692E257829005961779A
:100670002020253469202825336929004E69636BC1
:100680002025346920282533692928253369290044
:10069000526F6C6C20253469202825336929282560
:1006A00033692900596177202025346920282533B2
:1006B0006929282533692900414343202D205365AA
:1006C0006E736F72004E69636B2025346920282594
:1006D00033692900526F6C6C20253469202825333A
:1006E0006929005A202020202534692028253369D3
:1006F0002900566F6C746167653A202020253369A4
:100700002E253169560043757272656E743A202049
:10071000202533692E2531694100506F7765723A83
:1007200020202020202534695700446973636861C4
:100730007267653A202535696D41680052656365C9
:10074000697665720052432D525353493A20202056
:10075000202534690052432D5175616C6974793AD2
:10076000202534690052432D4368616E6E656C73B9
:100770003A25346900436F6D706173730048656199
:1007800064696E673A20202535690056616C75658D
:100790003A202020202535690053746172743A2074
:1007A00020202025356900506F7469313A202025BA
:1007B000336900506F7469323A2020253369005044
:1007C0006F7469333A202025336900506F7469349F
:1007D0003A202025336900506F7469353A2020256E
:1007E000336900506F7469363A2020253369005010
:1007F0006F7469373A202025336900506F74693867
:100800003A202025336900536572766F202000530B
:100810006574706F696E74202025336900506F73A2
:100820006974696F6E3A202533690052616E67659D
:100830003A2533692D2533690045787465726E4316
:100840006F6E74726F6C2020004E693A25346920F7
:1008500020526F3A253469200047733A25346920C5
:100860002047693A253469200048693A25346920CF
:100870002043663A2534692000424C2D4374726C43
:10088000204572726F727320002533642025336413
:10089000202533642025336420002533642025334C
:1008A000642025336420253364200025336420250B
:1008B000336420253364202533642000424C2054C7
:1008C000656D7065726174757265002533692025E8
:1008D00033692025336920253369200025336920B9
:1008E00025336920253369202533692000253369A4
:1008F0002025336920253369202533692000424CA7
:100900002D4374726C20666F756E64200020256321
:1009100020202025632020202563202020256320FF
:10092000002025632020202563202020256320200F
:1009300020256320002025632020202D2020202D2D
:100940002020202D2000313000313100313200468E
:100950006C696768742D54696D65202000546F744C
:10096000616C3A2535756D696E004163743A2020DB
:100970002535756D696E0028726573657429000AE6
:100980000D47656E65726174696E672064656661A6
:10099000756C7420506172616D6574657220536569
:1009A00074202564000A0D5573696E6720506172CA
:1009B000616D6574657220536574202564000A0DAD
:1009C00047656E65726174696E67206465666175FE
:1009D0006C74204D69786572205461626C65000A00
:1009E0000D4D697865722D436F6E6669673A2027F1
:1009F00025732720282575204D6F746F7273290089
:100A00000A0D3D3D3D3D3D3D3D3D3D3D3D3D3D3D79
:100A10003D3D3D3D3D3D3D3D3D3D3D3D3D3D3D3D06
:100A2000000A0D414343206E6F742063616C69625C
:100A30007261746564210D0A000A0D506C65617362
:100A40006520636F6E6E656374205370656B74729E
:100A5000756D20726563656976657220666F7220B8
:100A600062696E64696E67204E4F572E2E2E006F9E
:100A70006B2E0A0D0054696D656F75742E0A0D009A
:100A800000008F001E01AD013B02CA025803E603BD
:100A9000740402058F051B06A7063307BE07480826
:100AA000D2085B09E3096B0AF20A780BFD0B810C93
:100AB000040D860D070E870E060F840F00107B10A5
:100AC000F5106E11E5115B12CF124213B31323140C
:100AD0009214FE146A15D3153B16A1160517671755
:100AE000C81727188318DE1837198E19E319361A14
:100AF000871AD61A231B6E1BB61BFD1B411C831CB9
:100B0000C31C001D3C1D751DAB1DE01D121E421EA9
:100B10006F1E9A1EC31EE91E0D1F2E1F4D1F691F3B
:100B2000841F9B1FB01FC31FD31FE11FEC1FF51FA6
:100B3000FB1FFF1F002003010000D76B0002010113
:100B4000CA6C010302025E6D02000303BB6D253215
:100B5000692E2531695600253364256320253033FD
:100B6000646D00537461747573004552524F523A6C
:100B70002025326400253469202532693A25303237
:100B800069002534696D25630025336920253369A3
:100B900020253369202533690025336920253369F1
:100BA00020253369202533690054656D70657261B5
:100BB0007475726573202020200025634320202057
:100BC0002020002532692E253169562020253369E1
:100BD0002E253169410025346957202536696D413C
:100BE00068002532756D2F73205361743A25642097
:100BF0000020203344004E6F467800444750530095
:100C0000486F6D653A2533646D2025336425630094
:100C10004E6F204E6176694374726C21000A0D7725
:100C200077772E4D696B726F4B6F707465722E649F
:100C3000652028632920486953797374656D732092
:100C4000476D6248000A0D74686520757365206FF2
:100C500066207468697320736F66747761726520AB
:100C60006973206F6E6C79207065726D697474653C
:100C700064200A0D6F6E206F726967696E616C2067
:100C80004D696B726F4B6F707465722D4861726441
:100C900077617265004143542044534C004A6574A7
:100CA0006920736174656C6C6974005370656B7452
:100CB00072756D20736174656C6C697420284C6F5B
:100CC00077207265736F6C7574696F6E290053704D
:100CD000656B7472756D20736174656C6C697420DA
:100CE000283230343829005370656B7472756D206A
:100CF000736174656C6C6974004D756C74697369AB
:100D0000676E616C2050504D000A0D526563656935
:100D10007665723A2000756E6B6E6F776E2E205579
:100D200073696E672050504D2E2E2E006E6F74200A
:100D3000737570706F727465642062792068617277
:100D4000647761726521000A0D3D3D3D3D3D3D3DAD
:100D50003D3D3D3D3D3D3D3D3D3D3D3D3D3D3D3DC3
:100D60003D3D3D3D3D3D3D3D3D3D3D3D000A0D464A
:100D70006C69676874436F6E74726F6C0A0D4861BA
:100D80007264776172653A25642E25640A0D536F8B
:100D90006674776172653A5625642E256425632052
:100DA000000A0D3D3D3D3D3D3D3D3D3D3D3D3D3D13
:100DB0003D3D3D3D3D3D3D3D3D3D3D3D3D3D3D3D63
:100DC0003D3D3D3D3D3D000011241FBECFEFD0E134
:100DD000DEBFCDBF11E0A0E0B1E0E4E0F3EF02C080
:100DE00005900D92A43FB107D9F718E0A4EFB1E048
:100DF00001C01D92A23AB107E1F76AEAE2E0F0E031
:100E000081E2809357007491AE014F5F5F4F20EFF6
:100E100037EFDA019FE0F9012F5F3F4F84918D9307
:100E2000915097FFF8CF773911F40000FECFFA0107
:100E30009EE0819168276095915097FFFACF88894D
:100E4000681721F0773911F40000FECF0C94E90700
:100E50000C94000080910A06E82FFF27EE0FFF1F79
:100E6000EF5CF84F808191818D5E9F4F14F010925E
:100E70000301808191818A5B9F4FCCF480910301B3
:100E80008823A9F481E080930301809161048F5F3E
:100E900080936104853038F088EE93E090932402CB
:100EA0008093230204C066E970E00E948438809138
:100EB000610499279093DB058093DA0508951F93C9
:100EC000CF93DF93182F882389F082EF90E09F93D0
:100ED0008F938CE692E19F938F93E0912D04F09194
:100EE0002E0409950F900F900F900F9080912D0672
:100EF000823308F044C084EF91E00E949316EC0125
:100F0000112329F0CE010E949C168823D9F3C2E058
:100F1000D0E026E530E080911F01909120018217FA
:100F2000930730F02196255D3F4FC730D10598F3E8
:100F300080912D069927C89F9001C99F300DD89F99
:100F4000300D1124209300011123D9F068EC70E0DA
:100F50008C2F0E948438DF93CF938AEF90E09F9389
:100F60008F938CE692E19F938F93E0912D04F09103
:100F70002E0409958DB79EB706968DBF02C080934B
:100F80000001112311F1809100016AE00E94AD7807
:100F9000892F99279F938F93809100010E94AD78AC
:100FA00099279F938F9385E091E09F938F938CE691
:100FB00092E19F938F93E0912D04F0912E04099577
:100FC0002DB73EB7285F3F4F2DBFDF91CF911F91C7
:100FD0000895CFEFD0E1DEBFCDBF8824992414B8A7
:100FE00015B807EE13E00253104017FFFCCF189B13
:100FF00006C0199B02C08DE007C08BE005C0199B9D
:1010000002C084E101C08AE08093020181E887B9CF
:101010003E9A8FEF88B98BE184B981E085B98EE380
:101020008AB987E48BB9469A84B7877F84BF809159
:1010300060008861809360001092600084EC99E009
:10104000909324028093230210921C0310921B039E
:10105000109236071092350710921E0310921D034E
:101060001092200310921F0320910201243128F0D6
:1010700084EC94E0A0E0B0E004C08BE095E0A0E058
:10108000B0E08093970190939801A0939901B09359
:101090009A012A3011F0243110F0289801C0289AC2
:1010A0000E940D170E94CD160E9474120E94FE34F9
:1010B0000E943A1B0E9475300E94E2630E94AA6E51
:1010C0000E94B676809102018C3010F4299A01C0FA
:1010D000299878940E94942F809171028260809365
:1010E0007102109273020E94EC4384EF91E00E941F
:1010F00093168C018091710280FD05C0C8010E9489
:101100009C168823B9F38FE191E09F938F93BCE6FF
:10111000AB2EB2E1BB2EBF92AF92E0912D04F091C5
:101120002E04099580EA9FE00E9493168C01C0E08E
:10113000D0E00F900F900F900F90A3EDEA2EA6E055
:10114000FA2EF7E8CF2EF6E0DF2E0E94EC438091D6
:10115000710280FD05C0C8010E949C168823B9F366
:10116000F60180811816ACF40BC00E94EC4380910C
:10117000710280FD05C0C8010E949C168823B9F346
:10118000C8010E949C16882321F4F70180818823DE
:1011900064F7F701808187FF18C02196DF93CF9312
:1011A000219781E391E09F938F93BF92AF92E0915B
:1011B0002D04F0912E0409958091F4018F5F8093A6
:1011C000F4018DB79EB706968DBF2196E4E0F0E05E
:1011D000CE0EDF1E88E090E0E80EF91ECC30D1057F
:1011E00008F4B3CFC0E0D0E000ED16E0E7E8EE2E63
:1011F000E6E0FE2EF801838187FD1CC0F7018081A7
:101200001816C4F42196DF93CF93219784E391E0DD
:101210009F938F938CE692E19F938F93E0912D049F
:10122000F0912E04099582E0809321028DB79EB73C
:1012300006968DBFF801838180788383219684E0B0
:1012400090E0E80EF91E085F1F4FCC30D10590F2F8
:1012500082E591E09F938F93CCE6D2E1DF93CF9329
:10126000E0912D04F0912E0409959091080680914B
:10127000F4010F900F900F900F90981728F4809121
:10128000470480618093470488E791E09F938F93A0
:10129000DF93CF93E0912D04F0912E04099588EE11
:1012A00093E00E9493168C010E94401B0F900F90B8
:1012B0000F900F90C8010E949C168823D9F388E9EB
:1012C00091E09F938F93DF93CF93E0912D04F09162
:1012D0002E04099580E00E944639809102010F900A
:1012E0000F900F900F908A3011F0843110F02898F1
:1012F00001C0289A80ED97E0909324028093230206
:1013000085E5809363048EE090E00E94632E992728
:10131000182F00278FE090E00E94632E080F111D08
:101320001093FA010093F9018AE090E00E94632E85
:101330009927182F00278BE090E00E94632E080F5A
:10134000111D1093F8010093F7010F5F1F4F39F043
:101350008091F9019091FA018F5F9F4F41F41092B3
:10136000FA011092F9011092F8011092F7018091A0
:10137000F7019091F8019F938F938091F9019091DB
:10138000FA019F938F938DE991E09F938F93DF9361
:10139000CF93E0912D04F0912E0409958DB79EB75F
:1013A00008968DBF80EC91E09F938F93DF93CF934E
:1013B000E0912D04F0912E040995809116060F906E
:1013C0000F900F900F90E0912D04F0912E0482FF6A
:1013D00007C08CEC91E09F938F93DF93CF9308C06D
:1013E00088ED91E09F938F938CE692E19F938F938A
:1013F00009950F900F900F900F900E945E2088E843
:1014000093E1909394018093930181E0809362042F
:101410000E945F07809130060E941C768AEE91E060
:101420009F938F93DF93CF93E0912D04F0912E043F
:10143000099580ED97E00E9493168C018AEF90E069
:101440000E949316EC0183E08093B2050F900F90F9
:101450000F900F90CE010E949C16882339F084E6ED
:1014600090E00E949316EC010E947277809127020F
:10147000882309F4DFC180911101882309F4DAC1BE
:101480001092270280916104882319F00E942A0794
:1014900002C00E9480460E94EC43209102012A3043
:1014A00011F0243110F0289801C0289A809121036E
:1014B00090914704882339F08091210381508093D3
:1014C0002103977F0AC080916F00806280936F0034
:1014D00010923207109231079860909347048091E0
:1014E00093019091940101979093940180939301BB
:1014F0008091930190919401892B29F0809172023F
:10150000882309F43EC08091930190919401892B26
:1015100001F50E949B3085E090E0909394018093C8
:1015200093018091EC059091ED0501969093ED0566
:101530008093EC058091ED0280688093ED028091AC
:1015400047048160809347048091B3058260809353
:10155000B30580910801909109018F5F9F4F19F5A4
:10156000809118038823F9F080E197E29093240298
:101570008093230280E890E0909309018093080112
:1015800012C02A3011F0243110F0289801C0289A96
:101590008091230290912402892B29F48091ED02FD
:1015A0008F778093ED0280912702882309F042C152
:1015B0000E94B8120E94960EC8010E949C168823B1
:1015C00009F434C10C5E1F4F809172029091470460
:1015D000882339F09260909347048091B30582602C
:1015E0000CC09D7F9093470480919301909194014A
:1015F000079728F08091B3058D7F8093B305809184
:10160000930190919401079728F0809147048E7F71
:101610008093470480910501882321F081508093B5
:10162000050125C080936D041092F9021092F80212
:101630001092F7021092F6021092F5021092F40244
:1016400080910801909109018F5F9F4F81F48091F3
:101650002103882361F488E99AE39093240280931C
:10166000230280E09CE0909309018093080180911F
:10167000EA01893C70F081508093EA018091ED028B
:101680008F7B8093ED02809147048B7F809347048A
:1016900035C080910F08882309F18091ED028064A4
:1016A0008093ED0280914704846080934704809189
:1016B0000801909109018F5F9F4F81F48091180379
:1016C000882361F088E99AE39093240280932302AF
:1016D00080E098EA90930901809308011092FF033B
:1016E0001092FE031092FD031092FC038FEF9FEF08
:1016F00090933D0880933C081092EA01809100018C
:10170000282F332780911F01909120018217930782
:10171000CCF48091ED0280628093ED02809108010B
:10172000909109018F5F9F4FC1F480E797E19093FB
:1017300024028093230280E093E090930901809338
:1017400008010BC08091230290912402892B29F477
:101750008091ED028F7D8093ED020E94E06784E02E
:101760008093220280911803882329F45AEA852E57
:1017700055E0952E12C08091FB018F5F8093FB0195
:10178000813359F41092FB018091F5019091F6019B
:1017900001969093F6018093F5010894811C911CA9
:1017A000F2E78F16FBE09F0609F040C088249924D9
:1017B0002091F9013091FA012F5F3F4F3093FA01E8
:1017C0002093F9018091F7019091F801019690938F
:1017D000F8018093F701832F9927682F8EE090E01E
:1017E0000E94692E8091F9019091FA019070682F02
:1017F0008FE090E00E94692E8091F7019091F801AE
:10180000892F9927682F8AE090E00E94692E8091A5
:10181000F7019091F8019070682F8BE090E00E94A2
:10182000692E84E190E00E9493168C010E9430683A
:101830000E94C16E80912202882309F00BCE0E9483
:10184000036408CE1F920F920FB60F9211248F934C
:101850009F93EF93FF93809107018823E1F4809198
:10186000150290911602019690931602809315022C
:10187000FC01EE5EFA4FE081ED3019F0803A9105FF
:1018800039F4109216021092150281E0809307013C
:10189000E093C60004C01092160210921502FF9148
:1018A000EF919F918F910F900FBE0F901F90189501
:1018B0001F920F920FB60F9211242F933F934F93C5
:1018C0005F936F937F938F939F93AF93BF93CF93C8
:1018D000EF93FF9390E08091C60080930D025091AA
:1018E0001B02503A10F090931C0280910D028D3033
:1018F00009F065C080911C02823009F060C09093AD
:101900001C02852F992780599B4FFC0132974081FB
:101910002091170230911802241B3109DC01119724
:101920008C91281B3109C9019F70909318028093F4
:10193000170246E0969587954A95E1F7982F935CB4
:10194000909319022F733070235C20931A028081C8
:10195000981729F48C91281711F491E006C090E0B3
:1019600080910A028F5F80930A02C0910C02CC23FF
:1019700009F074C0992309F471C081E080930C02CE
:10198000580F509309025150E52FFF27E059FB4FA4
:101990008DE0808380917204823509F05FC00E94DF
:1019A0005E2088E190E02CE00FB6F894A895809333
:1019B00060000FBE20936000C09321024FC02091B1
:1019C0001C02822F992781309105F9F08230910510
:1019D0001CF4892B21F040C0029711F13DC0809189
:1019E0000D02833239F480910C02882319F481E0CE
:1019F00080931C0280910D028093700481E080939B
:101A00001B0280910D02992722C02F5F20931C0298
:101A1000E52FFF27E059FB4F80910D02808309C01D
:101A2000E52FFF27E059FB4F80910D028083503A4C
:101A300020F45F5F50931B0202C010921C022091A1
:101A40000D028091170290911802820F911D9093C0
:101A500018028093170202C010921C02FF91EF91AE
:101A6000CF91BF91AF919F918F917F916F915F9136
:101A70004F913F912F910F900FBE0F901F9018958F
:101A8000AC01A0E0B0E09D01A817B90748F4E2E17D
:101A9000F5E08191280F311D1196A417B507C8F301
:101AA0003F70FD01EE5EFA4FC90156E096958795AD
:101AB0005A95E1F7835C80831196FD01EE5EFA4F43
:101AC0002F733070822F835C8083AD5EBA4F8DE0C0
:101AD0008C9310920701809112058093C60008959F
:101AE000A0E0B0E0E6E7FDE00C9426792C859D852A
:101AF0000E85BB2483E2809312059F5990931305B2
:101B00002093140533E0E32EF12C002309F49EC04A
:101B1000CF84D888BE016D5E7F4FA989BA890150F4
:101B2000109709F493C01097B9F0F601EB0DF11D71
:101B3000B3949081119791F4002349F1FB016E5FFA
:101B40007F4FDB01C080D1806E5F7F4F0D90BC91D5
:101B5000A02DBB24015002C090E019C01097B9F02D
:101B6000F601EB0DF11DB3944081119791F4002320
:101B700041F1FB016E5F7F4FDB01C080D1806E5F62
:101B80007F4F0D90BC91A02DBB24015002C040E0BE
:101B900018C01097B1F0F601EB0DF11DB394108150
:101BA000119781F4002371F0FB013296DB01CD9097
:101BB000DC90BF016E5F7F4FA081B181BB240150DB
:101BC00001C010E0F701EE5EFA4F892F86958695E9
:101BD000835C80830894E11CF11CF701EE5EFA4FF0
:101BE000892F99278370907024E0880F991F2A9578
:101BF000E1F755279A0194E0369527959A95E1F7F4
:101C0000822B835C80830894E11CF11CF701EE5E5B
:101C1000FA4F4F705070440F551F440F551F812FBE
:101C2000992726E0969587952A95E1F7842B835C82
:101C300080830894E11CF11CF701EE5EFA4F1F73DC
:101C4000135C10830894E11CF11C6ACFC7010E9449
:101C5000400DE9E00C944279A3E07A2F409109020B
:101C60004650442309F458C0E72FFF27E059FB4FA3
:101C700080818D537F5FE72FFF27E059FB4F208145
:101C80002D537F5FE72FFF27E059FB4F30813D53F6
:101C90007F5FE72FFF27E059FB4F60816D537F5F28
:101CA0009927880F991F880F991F522F52955F709F
:101CB000582B822F99278F709070F4E0880F991F0E
:101CC000FA95E1F7232F26952695282B832F992720
:101CD00083709070E6E0880F991FEA95E1F7682B12
:101CE00041504F3FC9F0EA2FFF27E059FB4F508387
:101CF000AF5F41504F3F81F0EA2FFF27E059FB4F84
:101D00002083AF5F41504F3F39F0EA2FFF27E05962
:101D1000FB4F6083AF5FA5CF83E794E09093080209
:101D200080930702A350A09306020895A2E0B0E0BA
:101D3000ECE9FEE00C942C7980910C02882309F4E4
:101D4000C7C30E942C0E80917104823609F081C2B3
:101D50008091720499278137910509F4C0C08237B8
:101D60009105C4F48D36910509F482C08E36910533
:101D700044F48B34910531F18636910509F454C150
:101D800068C28E36910509F45BC08037910509F46D
:101D90009FC05FC28537910509F4E2C1863791057E
:101DA00044F48337910509F4DCC08437910539F197
:101DB00050C28737910509F410C28937910509F49B
:101DC0006AC147C2E0910702F091080280819181C7
:101DD0009093340380933303209131033091320385
:101DE000821B930B845E9D4F68E671E00E94CD7864
:101DF000845B90409093300380932F032AC280919C
:101E00000902A0910702B0910802853140F080E1FB
:101E1000EBE4F4E00D9001928A95E1F70DC08D910D
:101E20009D910D90BC91A02D80934B0490934C04F8
:101E3000A0934D04B0934E0480EF809304024BC0F6
:101E4000809107018823E1F38DE490E09F938F93C5
:101E50008AE796E09F938F9381E08F938F938EE430
:101E60008F930E94700D8DB79EB707968DBFF1C1FD
:101E7000A0910702B09108021C91113081F48DE409
:101E8000EAE7F6E00D9001928A95E1F70E94202F93
:101E90001983809147048F7E8093470401C0198283
:101EA000809107018823E1F381E090E09F938F9375
:101EB000CE0101969F938F9381E08F938F938DE452
:101EC0008F930E94700DADB7BEB71796ADBFC1C15D
:101ED00081E080930F028FEF80930501BAC1E091FA
:101EE0000702F091080280818F3F39F40E94852F0C
:101EF000E0910702F09108028083E0910702F091DF
:101F000008028081882311F481E003C0863010F03C
:101F100085E08083E0910702F091080280810E94B1
:101F2000782EE0910702F0910802808189838091E8
:101F300007018823E1F380E790E09F938F9389E086
:101F400096E09F938F9381E090E09F938F93CE01D3
:101F500001969F938F9382E08F9381E08F9381E529
:101F600071C12091070230910802D9018C918150F2
:101F7000853008F040C0F90181818435E1F52F5F9B
:101F80003F4F80E7E9E0F6E0D9010D9001928A9594
:101F9000E1F7F90182910E94BC2E809148069927B1
:101FA000AA27BB27BC01CD0124EC39E040E050E07A
:101FB0000E948E78DC01CB018093B7019093B80129
:101FC000A093B901B093BA01809149069927AA2735
:101FD000BB27BC01CD010E948E78DC01CB01809330
:101FE000B3019093B401A093B501B093B6010E94E0
:101FF000852F898301C01982809107018823E1F32D
:1020000081E090E09F938F93CE0101969F938F93F1
:1020100081E08F938F9383E58F930E94700D8DB72E
:102020009EB707968DBF26C0E0910702F091080287
:10203000E0818E2F8150853018F48E2F0E94782EEB
:102040000E94852F8983809107018823E1F381E035
:1020500090E09F938F93CE0101969F938F9381E0A1
:102060008F938F9386E48F930E94700DADB7BEB7A8
:102070001796ADBF80911803882329F46EE670E0AF
:1020800089810E94843880E00E945F078091300639
:102090000E941C76DEC0E0910702F0910802808168
:1020A000992787FD909590934C0780934B078181EA
:1020B000992787FD909590934E0780934D078281D5
:1020C000992787FD90959093500780934F078381C0
:1020D000992787FD909590935207809351078481AB
:1020E000992787FD90959093540780935307858196
:1020F000992787FD90959093560780935507868181
:10210000992787FD9095909358078093570787816B
:10211000992787FD909590935A078093590780855A
:10212000992787FD909590935C0780935B07818545
:10213000992787FD909590935E0780935D07828530
:10214000992787FD90959093600780935F0783851B
:10215000992787FD9095909362078093610779C0D6
:10216000E0910702F091080280810E9457348A832F
:10217000882319F481E0898301C0198280910701C5
:102180008823E1F388E090E09F938F9388EC96E0BA
:102190009F938F9321E030E03F932F93809107022C
:1021A000909108029F938F933F932F93CE010296B5
:1021B0009F938F933F932F93CE01820F931F9F93F3
:1021C0008F9384E08F9381E08F9385E58F930E94B6
:1021D000700DEDB7FEB773963BC080910602893053
:1021E000C0F120910702309108022F5F3F4F88E035
:1021F000A8ECB6E0F90101900D928A95E1F7D901BA
:102200008E910E94AD338A83882319F481E08983FB
:1022100001C01982809107018823E1F321E030E0B9
:102220003F932F93CE0102969F938F933F932F93CB
:10223000CE01820F931F9F938F9382E08F9381E053
:102240008F9387E58F930E94700DEDB7FEB73B9695
:10225000EDBF8091720499278436910509F4CDC0B1
:1022600085369105ACF48136910509F481C082363A
:1022700091052CF48B34910509F45DC021C182369F
:10228000910509F482C08336910509F491C018C103
:102290008C36910509F4FFC08D3691054CF48736D4
:1022A000910509F40AC18836910509F4C4C008C132
:1022B0008437910529F08637910509F4FAC000C1E9
:1022C00080910902A0910702B0910802803140F08C
:1022D00080E1EBE4F4E00D9001928A95E1F70DC006
:1022E0008D919D910D90BC91A02D80934B04909366
:1022F0004C04A0934D04B0934E04809107018823B1
:10230000E1F31F92809104018F9384E58F930E94E3
:10231000700D8AEF809304028FEF8093050180EAAD
:102320009FE00E9493169093FD018093FC010F9013
:102330000F900F90C5C0E0910702F09108028081D4
:102340009181909334038093330320913103309132
:102350003203821B930B845E9D4F68E671E00E94FE
:10236000CD78845B90409093300380932F03A8C076
:10237000E0910702F091080280818093060180328B
:1023800098F08FE1809306010FC0A0910702B091F1
:1023900008028BE0E3E6F4E00D9001928A95E1F704
:1023A00080916C048093F4058FEF8093050188C0C1
:1023B0008091000290910102892B89F4E09107023B
:1023C000F0910802E081EE2351F08AE0E89FC0011D
:1023D00011240E94931690933E0480933D04E09153
:1023E0000702F091080290818AE0989FC0011124B1
:1023F000909301028093000215C08FEF8093050136
:10240000E0910702F091080290818AE0989FC00154
:1024100011249093030280930202892B19F081E02A
:102420008093110280EA9FE00E9493169093FD0131
:102430008093FC0145C08FEF80930501E091070276
:10244000F0910802908197FD08C082E080930E020F
:102450001092FF011092FE011AC0909580916A02BD
:10246000892B80936A0291818AE0989FC001112490
:102470009093FF018093FE0184E080930E0280EA36
:102480009FE00E9493169093FD018093FC0181E0F0
:102490008093120215C08FEF80930501E09107022F
:1024A000F0910802808180936B0281E08093130297
:1024B00007C081E08093100203C081E08093140282
:1024C00010920C021092080210920702109206025B
:1024D000E3E0CE5F0C944879982F8091C00085FF8F
:1024E000FCCF9093C60008950F931F9388E18093CB
:1024F000C1008091C00082608093C0008091C100C3
:1025000080688093C1008091C10080648093C10085
:1025100000E010E00093C5008AE290E08093C400E0
:1025200080910202909103020E94931690934004BE
:1025300080933F048CED90E00E94931690936F047B
:1025400080936E041092410480E58093420486E0FB
:10255000809345048BE080934304109244041093CD
:10256000080200930702109206021F910F9108952E
:10257000A0E1B0E0EEEBF2E10C9429798091070143
:10258000882309F4C1C28091FC019091FD010E9451
:102590009C16882361F01092FF011092FE011092A8
:1025A0000302109202021092010210920002809126
:1025B000FE019091FF01892B41F0809110059091CF
:1025C00011050E949C16882329F480911202882309
:1025D00009F460C080910701882309F45BC08091F1
:1025E0000E0202E211E08430A8F00E94722080E521
:1025F00090E09F938F931F930F9381E08F938F931E
:1026000088E48F930E94700D2DB73EB7295F3F4F2E
:102610002DBF34C010926C0282E194E09F938F939F
:1026200087E690E29F938F93E0912D04F0912E0422
:10263000099584E190E09F938F931F930F9381E01E
:1026400090E09F938F938EE092E09F938F9382E030
:102650008F9381E08F9388E48F930E94700D809117
:102660000E02982F8F5F80930E022DB73EB7215F29
:102670003F4F2DBF943010F010920E028091FE015A
:102680009091FF010E94931690931105809310057D
:102690001092120280911302882351F18091070158
:1026A000882331F10E94722080E590E09F938F9300
:1026B00082E291E09F938F9321E030E03F932F934C
:1026C00081E291E09F938F933F932F938BE692E06B
:1026D0009F938F9383E08F9381E08F938CE48F930C
:1026E0000E94700D109213028DB79EB70F968DBF8A
:1026F000809110028823D1F0809107018823B1F0E6
:102700008AE090E09F938F9381E494E09F938F936E
:1027100081E08F938F9386E58F930E94700D1092C6
:1027200010022DB73EB7295F3F4F2DBF8091140295
:102730008823D9F0809107018823B9F08BE090E0DD
:102740009F938F9383E694E09F938F9381E08F9381
:10275000809104018F9387E48F930E94700D1092F3
:1027600014028DB79EB707968DBF80916E0490912D
:102770006F040E949C16882309F461C080910701B0
:10278000882309F45CC0809125069927880F991F3A
:10279000880F991F7C010027F7FC0095102F80916E
:1027A000750390917603A0917703B0917803BC01F3
:1027B000CD01A80197010E94027930935C04209317
:1027C0005B0480916D0390916E03A0916F03B091B3
:1027D0007003BC01CD01A80197010E9402793093DA
:1027E0005E0420935D048091020380935F048091D6
:1027F00001038093600488E090E09F938F938BE5C2
:1028000094E09F938F9381E08F9383E08F938BE687
:102810008F930E94700D809161042DB73EB7295FA0
:102820003F4F2DBF853018F086E08093610483E62A
:1028300090E00E94931690936F0480936E048091B1
:10284000020290910302892B41F080913F04909104
:1028500040040E949C16882321F480911102882351
:1028600039F180910701882319F10E947A3782E4B7
:1028700090E09F938F9382EB95E09F938F9381E0FD
:102880008F938F9384E48F930E94700D10921102A6
:102890008DB79EB707968DBF80910202909103027B
:1028A000009731F00E9493169093400480933F0468
:1028B0008091000290910102892B09F4B8C08091A7
:1028C0003D0490913E040E949C16882309F4AFC0F9
:1028D00080910701882309F4AAC0809125069927D1
:1028E000880F991F880F991F7C010027F7FC00951E
:1028F000102F8091750390917603A0917703B0918A
:102900007803BC01CD01A80197010E9402793093A0
:10291000300420932F0480916D0390916E03A09159
:102920006F03B0917003BC01CD01A80197010E9413
:10293000027930933204209331042091F7073091CB
:10294000F8074091F9075091FA07DA01C90163E0ED
:10295000880F991FAA1FBB1F6A95D1F7820F931F7B
:10296000A41FB51F820F931FA41FB51F20919701AD
:10297000309198014091990150919A01BC01CD018B
:102980000E940279309334042093330480913D03F4
:1029900090913E03A0913F03B091400339E0B5957B
:1029A000A795979587953A95D1F7809335048091AF
:1029B000390390913A03A0913B03B0913C0329E085
:1029C000B595A795979587952A95D1F78093360465
:1029D0008091450390914603A0914703B09148032D
:1029E00009E0B595A795979587950A95D1F78093B6
:1029F00037048EE090E09F938F938FE294E09F9353
:102A00008F9381E08F938F9383E48F930E94700D57
:102A100080910002909101020E94931690933E04CF
:102A200080933D042DB73EB7295F3F4F2DBF809166
:102A300006018F3F71F1992714E0880F991F1A95AD
:102A4000E1F78E5E9D4F40E150E0BC01CE01019662
:102A50000E94BC7780E190E09F938F93CE01019616
:102A60009F938F9381E090E09F938F9386E091E016
:102A70009F938F9382E08F9381E08F9381E48F9374
:102A80000E94700D8FEF809306018DB79EB70B9655
:102A90008DBF8091F4058823D1F0809107018823B0
:102AA000B1F081E090E09F938F9384EF95E09F9346
:102AB0008F9381E08F938F9382E48F930E94700DA8
:102AC0001092F4052DB73EB7295F3F4F2DBF80917F
:102AD0000F028823C9F0809107018823A9F084E3BD
:102AE00090E09F938F9381E397E09F938F9381E092
:102AF0008F938F9380E58F930E94700D10920F0239
:102B00008DB79EB707968DBFE6E0C05F0C94457900
:102B10001F920F920FB60F9211242F933F935F9342
:102B20006F937F938F939F93AF93BF93EF93FF9395
:102B300020E080912202882329F080912202815096
:102B40008093220280911004882319F08150809391
:102B5000100480912E02815080932E028F3F09F045
:102B60005BC089E080932E02809128029091290217
:102B70000196909329028093280280910C018F5F27
:102B8000817080930C01882319F481E080932702DF
:102B9000349903C081E080932F02809123029091A9
:102BA0002402892B21F180912302909124020B971A
:102BB00050F080912302909124020A97909324026E
:102BC0008093230204C01092240210922302809169
:102BD000230290912402209108013091090182235F
:102BE0009323892B11F021E008C020E006C08FEF6D
:102BF0009FEF9093090180930801809102012223A5
:102C000031F08A3011F45A9A07C0479A05C08A30C9
:102C100011F45A9801C0479880912F02882309F433
:102C200072C02091EA01222309F06DC0809116063E
:102C300083FF69C086B19927FC01E071F07084FFC1
:102C400014C080912502909126020196909326024D
:102C5000809325028091250290912602895E9340FF
:102C600008F451C020932F024EC08091250290910C
:102C70002602892B09F443C08091250290912602F7
:102C80008A569140E0F5809125029091260269E2F2
:102C900070E00E94B9788091250290912602860FFB
:102CA000971F909326028093250280912502909190
:102CB00026020B9750F080912502909126020A97E8
:102CC000909334038093330304C0F0933403E09370
:102CD0003303809133039091340320913103309179
:102CE0003203821B930B845E9D4F68E671E00E9465
:102CF000CD78845B90409093300380932F031092A3
:102D0000260210922502FF91EF91BF91AF919F9102
:102D10008F917F916F915F913F912F910F900FBE97
:102D20000F901F9018952091280230912902280FAA
:102D3000391FC90101960895209128023091290276
:102D4000821B930B892F9927869580749070089524
:102D5000CF93DF930E949316EC01CE010E949C1644
:102D60008823D9F3DF91CF910895CF93DF930E9409
:102D70009316EC0109C080911101882329F09093EA
:102D800011018FEC80937A00CE010E949C16982F3F
:102D9000882389F3DF91CF9108954FB78091FB028B
:102DA000282F33272F773070C901880F991F880F7C
:102DB000991F820F931F90932D0280932C02F894F9
:102DC0005F983E9A469A8091B0008F708093B000D1
:102DD0008091B00083608093B0008091B1008B73CC
:102DE0008093B1008091B1008B608093B10010920C
:102DF000B2008FEF8093B3008091B0008068809321
:102E0000B000809170008A7F809370008091700084
:102E10008260809370004FBF08958AE090E00E9426
:102E20009316909337028093360282E085BD83EA41
:102E300084BD17BC84EB88BD86E086BD80916E00A2
:102E4000816080936E0008951F920F920FB60F92CB
:102E500011242F933F934F935F936F937F938F939F
:102E60009F93AF93BF93CF93DF93EF93FF938091A3
:102E70000201843108F017C18091FB0287FD13C164
:102E800080913002882309F0AEC38091B00086FFA4
:102E9000ECC08091B0008F7B8093B00089EA93E012
:102EA000909332028093310280910D0190910E0136
:102EB0009C01220F331F280F391F8091A3019927EE
:102EC000880F991F880F991F280F391F37FF02C0DD
:102ED0002D5F3F4FC901959587959595879590935F
:102EE0000E0180930D019093200280931F02809128
:102EF0006B066091370620917503309176034091FF
:102F000077035091780380FF2CC077278827992773
:102F1000EA01D90157FF04C0A158BF4FCF4FDF4F7F
:102F2000E7E0D595C795B795A795EA95D1F79D01A7
:102F3000AE010E948E789B01AC0197FF04C0215C1A
:102F40003F4F4F4F5F4F66E0559547953795279513
:102F50006A95D1F780911F0290912002820F931FF2
:102F60002BC0772788279927EA01D90157FF04C08A
:102F7000A158BF4FCF4FDF4F27E0D595C795B795E5
:102F8000A7952A95D1F79D01AE010E948E789B01ED
:102F9000AC0197FF04C0215C3F4F4F4F5F4FF6E0FD
:102FA0005595479537952795FA95D1F780911F024A
:102FB00090912002821B930B9093200280931F021A
:102FC00080913806282F3327220F331F220F331FFB
:102FD00080911F0290912002821793077CF08091CC
:102FE0003906282F3327220F331F220F331F8091DA
:102FF0001F02909120022817390724F430932002F1
:1030000020931F02209131023091320280911F02E1
:1030100090912002280F391F205032403093320205
:103020002093310280911F029091200297FD039618
:1030300095958795959587959093200280931F028B
:1030400045E02D3D340718F08CED95E005C027577D
:10305000314030F487E791E090933202809331025F
:10306000809131029091320287C28091B0008064D9
:103070008093B00080913E06282F33278DED96E097
:10308000289FA001299F500D389F500D1124CA017F
:103090002091330230913402821B930B90933202C1
:1030A000809331029DC280913002882309F09BC237
:1030B0008091B00086FF65C28091B0008F7B8093C5
:1030C000B000E0913502EE23F1F480913E06282F06
:1030D00033278DED96E0289FA001299F500D389F42
:1030E000500D1124CA012091330230913402821B09
:1030F000930B90933202809331021092340210921B
:103100003302469A6DC249EA53E05093320240932B
:1031100031028E2F99278330910509F4A4C18430A0
:1031200091053CF48130910561F0029709F4D2C019
:10313000ECC18430910509F4DBC1059709F4DBC1CA
:10314000E4C180910D0190910E019C01220F331F6B
:10315000280F391F8091A3019927880F991F880F85
:10316000991F280F391F37FF02C02D5F3F4FC9013C
:10317000959587959595879590930E0180930D0170
:103180009093200280931F0280916B066091370616
:103190002091750330917603409177035091780325
:1031A00080FF2CC0772788279927EA01D90157FF8C
:1031B00004C0A158BF4FCF4FDF4F27E0D595C7952B
:1031C000B795A7952A95D1F79D01AE010E948E78FB
:1031D0009B01AC0197FF04C0215C3F4F4F4F5F4FF5
:1031E000F6E05595479537952795FA95D1F7809153
:1031F0001F0290912002820F931F27C077278827F4
:10320000992757FF04C021583F4F4F4F5F4FE7E0CA
:103210005595479537952795EA95D1F70E948E7871
:103220009B01AC0197FF04C0215C3F4F4F4F5F4FA4
:1032300066E055954795379527956A95D1F7809122
:103240001F0290912002821B930B90932002809387
:103250001F0280913806282F3327220F331F220F99
:10326000331F80911F0290912002821793077CF0F8
:1032700080913906282F3327220F331F220F331F47
:1032800080911F02909120022817390724F430936F
:10329000200220931F0280913102909132022091EE
:1032A0001F0230912002820F931F80509240909312
:1032B00032028093310280911F029091200297FD8B
:1032C0000396959587959595879590932002809381
:1032D0001F022EC180910F01909110019C01220FBD
:1032E000331F280F391F8091A2019927880F991F3A
:1032F000880F991F280F391F37FF02C02D5F3F4FDE
:10330000C901959587959595879590931001809320
:103310000F0190931E0280931D0280916B066091B5
:103320003B06A0916D03B0916E03C0916F03D091E5
:10333000700381FF2AC07727882799279D01AE0156
:10334000D7FF04C021583F4F4F4F5F4FE7E05595DF
:10335000479537952795EA95D1F70E948E789B017E
:10336000AC0197FF04C0215C3F4F4F4F5F4FC6E059
:103370005595479537952795CA95D1F780911D02A8
:1033800090911E02820F931F29C0772788279927C3
:103390009D01AE01D7FF04C021583F4F4F4F5F4FF3
:1033A000B7E05595479537952795BA95D1F70E947F
:1033B0008E789B01AC0197FF04C0215C3F4F4F4FBB
:1033C0005F4FA6E05595479537952795AA95D1F774
:1033D00080911D0290911E02821B930B90931E02FE
:1033E00080931D0280913C06282F3327220F331F24
:1033F000220F331F80911D0290911E0282179307A6
:103400007CF080913D06282F3327220F331F220F97
:10341000331F80911D0290911E022817390724F452
:1034200030931E0220931D0280913102909132024E
:1034300020911D0230911E02820F931F80509240F6
:10344000909332028093310280911D0290911E026E
:1034500097FD0396959587959595879590931E0270
:1034600080931D0265C080911006E82FFF27EE0FA4
:10347000FF1FEF5CF84F80819181805E9F4FACF120
:103480008081918181971CF08CED95E04DC08091F9
:103490002C0290912D02C29778F020912A0230914F
:1034A0002B0280912C0290912D022817390749F4A4
:1034B00010922B0210922A02509332024093310252
:1034C00037C080912A0290912B02019690932B0293
:1034D00080932A0220912A0230912B0280910A01C6
:1034E00090910B012817390719F587E791E01CC067
:1034F00080919F0702C08091CD079927880F991F5F
:10350000880F991F87559E4F0FC0FF27EE0FFF1F93
:10351000EF5CF84F20813181220F331F80913102FF
:1035200090913202820F931F909332028093310266
:10353000809131029091320245E08D3D940718F060
:103540008CED95E005C08757914030F487E791E016
:1035500090933202809331022091310230913202F5
:103560002C5B304030933202209331028091330241
:1035700090913402820F931F909334028093330210
:103580002FC08091B00080648093B0008CEB90E0FD
:1035900090933202809331028091330290913402F1
:1035A00084549F4F90933402809333028091210280
:1035B000882321F080912103853B20F48091210212
:1035C000823011F4469801C0469A809135028F5F8F
:1035D0008093350290913E06981710F410923502B0
:1035E00081E080933002209131023091320281E0FB
:1035F0002F37380730F08FEF8093B3002F5F3040C4
:103600000FC02F3F3105C9F0C0F0A9014F5F5040F6
:103610004F37510550F480E88093B3002058304074
:10362000309332022093310212C08FEF8093B300A7
:1036300050933202409331020AC08091310280934C
:10364000B300109232021092310210923002FF91B8
:10365000EF91DF91CF91BF91AF919F918F917F912A
:103660006F915F914F913F912F910F900FBE0F90EF
:103670001F90189510927C008FEC80937A0008952B
:10368000CF93DF9310923C0283E090E00E94632E80
:10369000C82FDD27C531D10508F02A97C7BD84E6BC
:1036A00090E00E94B516809115019091160180520C
:1036B000934010F4C0E0D0E0CA3FD105F8F4C7BD94
:1036C00082E390E00E94B51687E294E09F938F9387
:1036D0008CE692E19F938F93E0912D04F0912E045C
:1036E000099580911501909116010F900F900F9000
:1036F0000F908052934010F02196DECFC0930506C4
:103700006C2F83E090E00E94692E8091160680FF66
:103710000AC0809105068A508B3E28F080914604AD
:10372000806480934604C7BD8CE291E00E94B51688
:10373000DF91CF910895EF92FF921F93CF9310E006
:1037400080ED97E00E9493167C01CCE8133019F4C9
:10375000CB3008F0C9E010E080914C0290914D020E
:103760008C5F934024F48091140181500AC08091B1
:103770004C0290914D028750944034F08091140196
:103780008F5F8093140101C011E080914A029091F3
:103790004B028C5F934024F48091130181500AC046
:1037A00080914A0290914B028750944034F080916E
:1037B00013018F5F8093130101C01F5F8091480246
:1037C000909149028C5F934024F4809112018150C2
:1037D0000AC0809148029091490287509440C4F0F9
:1037E000809112018F5F8093120113C089E294E0EF
:1037F0009F938F938CE692E19F938F93E0912D049A
:10380000F0912E0409950F900F900F900F905FC0CC
:103810001F5F82E180937602809171028E7F809398
:10382000710285EA8093BC00809114018A3040F4D3
:10383000809146048160809346048AE0809314015D
:1038400080911401863F40F080914604816080930E
:10385000460485EF80931401809113018A3040F46F
:10386000809146048260809346048AE0809313012D
:1038700080911301863F40F08091460482608093DE
:10388000460485EF80931301809112018A3040F441
:10389000809146048460809346048AE080931201FC
:1038A00080911201863F40F08091460484608093AD
:1038B000460485EF8093120180917602882339F0C7
:1038C000C7010E949C16882309F090CFF5CF109273
:1038D00011018FEC80937A00809111018823E1F32C
:1038E000CA3020F48AE090E00E94B516C15009F079
:1038F0002DCF86E490E00E94B516CF911F91FF90E6
:10390000EF9008951F920F920FB60F921124AF926D
:10391000BF92CF92DF92EF92FF920F931F932F935C
:103920003F934F935F936F937F938F939F93AF9347
:10393000BF93EF93FF9380915502282F332744279D
:1039400055278F5F80935502F9012231310508F028
:103950008CC3E25CFF4F0C94547980917800909175
:10396000790046C080917800909179002CC18091B7
:10397000780090917900909358028093570257C134
:1039800080917E0390917F0320917800309179009F
:10399000821B930B9093F6058093F5058091F505B6
:1039A0009091F60590936202809361025EC18091CE
:1039B0007800909179002091800330918103821BDF
:1039C000930B9093040680930306809103069091D5
:1039D0000406909364028093630249C380915B0262
:1039E00090915C022091780030917900820F931FB2
:1039F00090935C0280935B0281E03AC3809159020C
:103A000090915A022091780030917900820F931F93
:103A100090935A028093590284E02AC380911F0137
:103A2000909120019C01220F331F280F391F809194
:103A300078009091790063E070E00E94B978260FD9
:103A4000371F36952795369527953093200120937B
:103A50001F0185E00DC3809178009091790040911D
:103A60007A0350917B03841B950B909343028093C0
:103A700042028091420290914302029704F122E0B7
:103A80004E3E520784F4209156022B5F209356023B
:103A900025508091EE029091EF02845F914018F4DE
:103AA000215F2093560280915602853684F14F5F44
:103AB0005F4F50937B0340937A03845626C08091D6
:103AC0004202909143028F5F9F4F0CF532E04732E4
:103AD0005307ECF0209156022550209356022B5F9D
:103AE0008091EE029091EF02845F914018F42F5084
:103AF00020935602809156028C394CF4415050402C
:103B000050937B0340937A038C598093560281E053
:103B10008093410280917800909179009093FC0508
:103B20008093FB0580914202909143029C014427BF
:103B300037FD4095542F8091350390913603A09125
:103B40003703B0913803820F931FA41FB51F8093D2
:103B5000350390933603A0933703B0933803209135
:103B6000350330913603409137035091380357FFA6
:103B700004C021503C4F4F4F5F4F0AE05595479589
:103B8000379527950A95D1F78091350390913603A3
:103B9000A0913703B0913803821B930BA40BB50B94
:103BA0008093350390933603A0933703B093380383
:103BB0002EC18091590290915A0220917800309143
:103BC0007900820F931F90935A02809359021092AA
:103BD000540250C2809102018A3071F480917800C1
:103BE000909179002091570230915802820F931FD3
:103BF00001969695879517C04091570250915802AB
:103C0000843158F02091780030917900240F351FCD
:103C10008FEF97E0821B930B06C080917800909104
:103C20007900840F951F909349028093480286E0A3
:103C30001FC280917E0390917F0320917800309184
:103C40007900821B930B9093F6058093F505809184
:103C5000F5059091F6052091610230916202820F84
:103C6000931F909347028093460287E001C28091A0
:103C70007800909179002091800330918103821B1C
:103C8000930B909304068093030680910306909112
:103C900004062091630230916402820F931F909377
:103CA000450280934402E3C120915B0230915C02A3
:103CB0008091780090917900280F391F30935C0231
:103CC00020935B02809102018A3019F4220F331F86
:103CD00004C0220F331F220F331F30935C02209346
:103CE0005B0220915B0230915C02C90137FD0796AF
:103CF000A3E095958795AA95E1F790934D0280935F
:103D00004C0280915D0290915E02820F931F97FD9D
:103D100001969595879590935E0280935D02209120
:103D20008A0330918B03821B930B90931E01809327
:103D30001D01209152023091530280911D019091FA
:103D40001E01280F391F37FF02C02F5F3F4F3595E7
:103D5000279530935302209352024ECE2091590260
:103D600030915A028091780090917900280F391F84
:103D700030935A0220935902809102018A3019F43B
:103D8000220F331F04C0220F331F220F331F309323
:103D90005A02209359022091590230915A02C901C6
:103DA00037FD079663E0959587956A95E1F79093BF
:103DB0004B0280934A0280915F0290916002820FD1
:103DC000931F97FD01969595879590936002809338
:103DD0005F022091880330918903821B930B90939B
:103DE0001C0180931B01209150023091510280915F
:103DF0001B0190911C01280F391F37FF02C02F5F54
:103E00003F4F35952795309351022093500283E020
:103E10002FC11092550281E08093110180913802E8
:103E200090913902019690933902809338028091E3
:103E300078009091790090931601809315018091FC
:103E4000150190911601AA27BB27A0906502B0909A
:103E50006602C0906702D0906802A80EB91ECA1E02
:103E6000DB1EA0926502B0926602C0926702D092F9
:103E70006802809169028F5F80936902823108F441
:103E8000F6C08091170190911801A0911901B0918D
:103E90001A017C018D0123E0EE0CFF1C001F111F95
:103EA0002A95D1F7E81AF90A0A0B1B0BEA0CFB1C3E
:103EB0000C1D1D1D80913C02992787FD9095A92F0F
:103EC000B92FBC01CD0126EC34E240E050E00E9465
:103ED0008E78DC01CB01E81AF90A0A0B1B0BD8011A
:103EE000C7010496A11DB11DB7FF05C0D801C701C8
:103EF0000B96A11DB11D13E0B595A79597958795D4
:103F00001A95D1F78093170190931801A093190186
:103F1000B0931A018091FD059091FE057C01002768
:103F2000F7FC0095102F8091170190911801A09136
:103F30001901B0911A01E81AF90A0A0B1B0BE09259
:103F40001303F092140300931503109316032091AA
:103F50003D0230913E0240913F025091400257FF96
:103F600004C0215F3F4F4F4F5F4FF4E05595479599
:103F700037952795FA95D1F780913D0290913E02B1
:103F8000A0913F02B0914002821B930BA40BB50B92
:103F900080933D0290933E02A0933F02B093400273
:103FA00080913D0290913E02A0913F02B09140026B
:103FB0008E0D9F1DA01FB11F80933D0290933E0266
:103FC000A0933F02B093400280913A0290913B024D
:103FD000AC01E5E0440F551FEA95E1F7481B590B8A
:103FE00080913D0290913E02A0913F02B09140022B
:103FF000B7FF03C00F96A11DB11D74E0B595A7953D
:10400000979587957A95D1F72091130330911403F2
:10401000281B390B63E0220F331F6A95E1F7240F49
:10402000351F37FF02C0215E3F4F45E0359527958C
:104030004A95E1F730933B0220933A02D601C5013D
:10404000D7FE03C00196A11DB11DB595A795979503
:1040500087958093650290936602A0936702B09360
:10406000680289E08093690202C01092550282E0E2
:10407000809354028091540280937C008091550279
:10408000882319F08FEC80937A00FF91EF91BF9114
:10409000AF919F918F917F916F915F914F913F91E0
:1040A0002F911F910F91FF90EF90DF90CF90BF90D5
:1040B000AF900F900FBE0F901F90189590E2E2E224
:1040C000F1E08FE49193815087FFFCCF08959091A8
:1040D0006C02E2E2F1E0E90FF11D80839F5F9093B3
:1040E0006C020895EF92FF920F931F93CF93DF938B
:1040F00020916A0220FF0AC080916B02882311F090
:10410000815002C08091210180936B0221FF0CC07D
:1041100090916B0280912101981719F410926B0213
:1041200003C09F5F90936B02822F992780FF04C08A
:1041300081FF02C010926B020E945E2080916B0290
:10414000282F3327C7E6EC2EC0E2FC2EC0912D04A9
:10415000D0912E048A3098F481E180936C023F93D1
:104160002F9380E694E09F938F93FF92EF92FE014E
:1041700009952DB73EB72A5F3F4F2DBF11C080E193
:1041800080936C023F932F9385E694E09F938F93E7
:10419000FF92EF92FE0109958DB79EB706968DBFEF
:1041A00020916B02822F9927AA27BB27FC014297F7
:1041B00010F00C941F2BE05BFF4FB7E6EB2EB0E244
:1041C000FB2EC0912D04D0912E040C9454791092A2
:1041D0006C028AE694E09F938F9307E610E2FF92C9
:1041E000EF92FE01099584E180936C020F900F908D
:1041F0000F900F9087E690E09F938F9380E590E07B
:104200009F938F931F921F92809102016AE00E94F8
:10421000AD78892F99279F938F93809102010E94F7
:10422000AD7899279F938F938AE794E09F938F931C
:10423000FF92EF92E0912D04F0912E04099588E20F
:1042400080936C022DB73EB7225F3F4F2DBF8BE7A7
:1042500096E09F938F930E94852F99279F938F932A
:1042600089E994E09F938F93FF92EF92E0912D0460
:10427000F0912E0409958DB79EB708968DBF909149
:104280004604992351F08CE380936C02892F99277F
:104290009F938F9387EA94E085C690917202992349
:1042A00071F08CE380936C02892F99279F938F93F1
:1042B0008EEB94E09F938F931F930F9391C0809107
:1042C000470484FF07C08CE380936C0283ED94E085
:1042D0000C94B12A8091930190919401069710F06B
:1042E0000C94282B8CE380936C0280EE94E00C9469
:1042F000B12A80911606A7E6EA2EA0E2FA2EC09116
:104300002D04D0912E0480FF74C010926C02809115
:10431000130390911403A0911503B0911603BC01EF
:10432000CD0125E030E040E050E00E9402793F936B
:104330002F938DEE94E09F938F93FF92EF92FE0167
:10434000099584E180936C022DB73EB72A5F3F4FF9
:104350002DBF80910F0390911003A0911103B09194
:104360001203BC01CD0125E030E040E050E00E94A6
:1043700002793F932F938AEF94E09F938F93FF925C
:10438000EF92E0912D04F0912E04099588E280933C
:104390006C028DB79EB706968DBF809115019091E6
:1043A00016019F938F9387E095E09F938F93FF92E1
:1043B000EF92E0912D04F0912E0409958CE3809307
:1043C0006C022DB73EB72A5F3F4F2DBF87B59927A7
:1043D0009F938F9384E195E09F938F93FF92EF9249
:1043E000E0912D04F0912E0409958DB79EB70696A5
:1043F0002FC710926C0281E295E09F938F93FF92FA
:10440000EF92FE01099584E180936C020F900F906A
:104410000F900F9080E395E09F938F93FF92EF9220
:10442000E0912D04F0912E04099588E280936C02AE
:104430000F900F900F900F9089E395E09F938F93CB
:10444000FF92EF92E0912D04F0912E0409958CE3F8
:1044500080936C020F900F900F900F9088E495E07E
:104460009F938F93FF92EF920C94B52A10926C0257
:1044700081E595E09F938F9307E610E2FF92EF921C
:10448000FE01099584E180936C020F900F900F90CC
:104490000F908091750390917603A0917703B0916E
:1044A0007803B7FF04C081509C4FAF4FBF4FFAE075
:1044B000B595A79597958795FA95D1F7BF93AF9343
:1044C0009F938F938EE595E09F938F931F930F9308
:1044D000E0912D04F0912E04099588E280936C02FE
:1044E0002DB73EB7285F3F4F2DBF80916D03909150
:1044F0006E03A0916F03B0917003B7FF04C08150A9
:104500009C4FAF4FBF4FEAE0B595A795979587951C
:10451000EA95D1F7BF93AF939F938F938DE695E084
:104520009F938F931F930F93E0912D04F0912E048E
:1045300009958CE380936C028DB79EB708968DBF6A
:1045400080913303909134039F938F938CE795E090
:104550009F938F931F930F93E0912D04F0912E045E
:1045600009952DB73EB72A5F3F4F0DC710926C02D9
:1045700080913507909136079F938F9380913307F1
:10458000909134079F938F938BE895E09F938F933F
:10459000FF92EF92FE01099584E180936C028DB742
:1045A0009EB708968DBF8091390790913A079F93E7
:1045B0008F9380913707909138079F938F938BE962
:1045C00095E09F938F93FF92EF92E0912D04F091ED
:1045D0002E04099588E280936C022DB73EB7285FC0
:1045E0003F4F2DBF80913D0790913E079F938F9342
:1045F00080913B0790913C079F938F938BEA95E0C6
:104600009F938F93FF92EF92E0912D04F0912E04EF
:1046100009958CE380936C028DB79EB708968DBF89
:1046200080914107909142079F938F9380913F071C
:10463000909140079F938F938BEB95E0A2C01092CF
:104640006C0280910B06E82FFF27EE0FFF1FEF5C37
:10465000F84F808191819F938F9380910A06E82F74
:10466000FF27EE0FFF1FEF5CF84F808191819F9332
:104670008F938BEC95E09F938F93FF92EF92FE01C7
:10468000099584E180936C028DB79EB708968DBF23
:1046900080910D06E82FFF27EE0FFF1FEF5CF84F0C
:1046A000808191819F938F9380910C06E82FFF2743
:1046B000EE0FFF1FEF5CF84F8081918188589F4F6C
:1046C0009F938F938BED95E09F938F93FF92EF9243
:1046D000E0912D04F0912E04099588E280936C02FC
:1046E0002DB73EB7285F3F4F2DBF80910F06E82FB3
:1046F000FF27EE0FFF1FEF5CF84F808191818259F9
:104700009F4F9F938F9380910E06E82FFF27EE0F08
:10471000FF1FEF5CF84F8081918182599F4F9F93DB
:104720008F938BEE95E09F938F93FF92EF92E091A2
:104730002D04F0912E0409958CE380936C028DB7C3
:104740009EB708968DBF80911106E82FFF27EE0FC8
:10475000FF1FEF5CF84F8081918182599F4F9F939B
:104760008F9380911006E82FFF27EE0FFF1FEF5C5D
:10477000F84F8081918182599F4F9F938F938BEF48
:1047800095E09F938F93FF92EF92E0912D04F0912B
:104790002E0409952DB73EB7285F3F4FF4C5109200
:1047A0006C028BE096E09F938F9307E610E2FF92F6
:1047B000EF92FE010995809102010F900F900F90EA
:1047C0000F908A3009F0A1C084E180936C0280913F
:1047D0008A0390918B039C0197FF02C0295F3F4F92
:1047E000287F821B930B9F938F9380918A039091D4
:1047F0008B0397FD079673E0959587957A95E1F77A
:104800009F938F9320918A0330918B0337FF02C0CF
:10481000295F3F4F63E0359527956A95E1F78091D1
:104820004C0290914D02821B930B9F938F9389E1D1
:1048300096E09F938F931F930F93E0912D04F09137
:104840002E04099588E280936C028DB79EB70A9674
:104850008DBF80918803909189039C0197FF02C0CE
:10486000295F3F4F287F821B930B9F938F938091EB
:1048700088039091890397FD079653E09595879556
:104880005A95E1F79F938F93209188033091890384
:1048900037FF02C0295F3F4F43E0359527954A9582
:1048A000E1F780914A0290914B02821B930B9F93F8
:1048B0008F938AE296E09F938F931F930F93E091DB
:1048C0002D04F0912E0409958CE380936C022DB792
:1048D0003EB7265F3F4F2DBF80918603909187039F
:1048E0009F938F9380918603909187032091480234
:1048F00030914902821B930B9F938F938BE396E039
:104900009F938F931F930F93A3C38B3019F0843120
:1049100008F4ADC084E180936C0280918A03909189
:104920008B039C0197FF02C0215F3F4F207F821BBA
:10493000930B97FD0196959587959F938F93809103
:104940008A0390918B0397FD0F9624E095958795A8
:104950002A95E1F79F938F9320918A0330918B03DF
:1049600037FF02C0295F3F4F83E0359527958A9531
:10497000E1F780914C0290914D02821B930B9F9323
:104980008F9389E496E09F938F931F930F93E09109
:104990002D04F0912E04099588E280936C022DB7C6
:1049A0003EB7265F3F4F2DBF8091880390918903CA
:1049B0009C0197FF02C0215F3F4F207F821B930B1A
:1049C00097FD0196959587959F938F938091880386
:1049D0009091890397FD0F96B4E095958795BA95C8
:1049E000E1F79F938F93209188033091890337FFDC
:1049F00002C0295F3F4FA3E035952795AA95E1F7BF
:104A000080914A0290914B02821B930B9F938F934C
:104A10008BE596E09F938F931F930F93E0912D0466
:104A2000F0912E0409958CE380936C028DB79EB7AC
:104A30000A968DBF809186039091870397FD01961A
:104A4000959587959F938F93809186039091870387
:104A50002091480230914902821B930B9F938F93C0
:104A60008DE696E09F938F931F930F938ECE8D309C
:104A700009F0EEC584E180936C02809114019927BE
:104A80009F938F9380918A0390918B0397FD0F964C
:104A9000E4E095958795EA95E1F79F938F932091B0
:104AA0008A0330918B0337FF02C0295F3F4F73E0C9
:104AB000359527957A95E1F780914C0290914D02BA
:104AC000821B930B9F938F938CE796E09F938F931A
:104AD0001F930F93E0912D04F0912E04099588E225
:104AE00080936C028DB79EB70A968DBF809113019B
:104AF00099279F938F93809188039091890397FDC5
:104B00000F9664E0959587956A95E1F79F938F934B
:104B1000209188033091890337FF02C0295F3F4FFE
:104B200053E0359527955A95E1F780914A02909187
:104B30004B02821B930B9F938F9380E996E09F9388
:104B40008F931F930F93E0912D04F0912E040995FC
:104B50008CE380936C022DB73EB7265F3F4F2DBF8D
:104B60008091120199279F938F9380918603909152
:104B7000870397FD0196959587959F938F938091D5
:104B80008603909187032091480230914902821B4D
:104B9000930B9F938F9384EA96E09F938F931F9339
:104BA0000F93E0912D04F0912E0409958DB79EB7D7
:104BB0000A964EC310926C0288EB96E09F938F93F7
:104BC000FF92EF92FE01099584E180936C020F90B1
:104BD0000F900F900F9080918003909181039F938D
:104BE0008F9380914402909145029F938F9385EC1F
:104BF00096E09F938F93FF92EF92E0912D04F091B6
:104C00002E04099588E280936C022DB73EB7285F89
:104C10003F4F2DBF80917E0390917F039F938F9391
:104C200080914602909147029F938F9384ED96E086
:104C30009F938F93FF92EF92E0912D04F0912E04B9
:104C400009958CE380936C028DB79EB708968DBF53
:104C500080917A0390917B039F938F93809142027E
:104C6000909143029F938F9383EE96E08ACD1092AA
:104C70006C0280911F01909120016AE070E00E9417
:104C8000CD789F938F9380911F01909120016AE0CE
:104C900070E00E94CD787F936F9382EF96E09F93B0
:104CA0008F93FF92EF92FE01099584E180936C024D
:104CB0008DB79EB708968DBF80916E0890916F0852
:104CC0006AE070E00E94B9789F938F9380916E089C
:104CD00090916F086AE070E00E94B9787F936F93BB
:104CE00086E097E09F938F93FF92EF92E0912D04DF
:104CF000F0912E04099588E280936C022DB73EB79F
:104D0000285F3F4F2DBF80917008909171089F934D
:104D10008F938AE197E09F938F93FF92EF92E091B8
:104D20002D04F0912E0409958CE380936C028DB7CD
:104D30009EB706968DBF80917208909173089F93DD
:104D40008F938AE297E02EC110926C028CE397E079
:104D50009F938F93FF92EF92FE01099584E18093D8
:104D60006C020F900F900F900F90809131079091EF
:104D700032079F938F9385E497E09F938F93FF92E1
:104D8000EF92E0912D04F0912E04099588E2809332
:104D90006C028DB79EB706968DBF8091210399272F
:104DA0009F938F9385E597E09F938F93FF92EF9268
:104DB000E0912D04F0912E0409958CE380936C0210
:104DC0002DB73EB72A5F3F4F2DBF809130079927FF
:104DD00001979F938F9385E697E0FECA10926C022D
:104DE00085E797E09F938F93FF92EF92FE010995DD
:104DF00084E180936C020F900F900F900F90809140
:104E00002F03909130039F938F938DE797E09F93AB
:104E10008F93FF92EF92E0912D04F0912E0409956B
:104E200088E280936C022DB73EB72A5F3F4F2DBFBB
:104E300080913303909134039F938F938BE897E095
:104E40009F938F93FF92EF92E0912D04F0912E04A7
:104E500009958CE380936C028DB79EB706968DBF43
:104E600080913103909132039F938F9389E997E06A
:104E700099C010926C028091220399279F938F937F
:104E800087EA97E09F938F93FF92EF92FE01099537
:104E900084E180936C028DB79EB706968DBF80919A
:104EA000230399279F938F9383EB97E09F938F938F
:104EB000FF92EF92E0912D04F0912E04099588E283
:104EC00080936C022DB73EB72A5F3F4F2DBF809174
:104ED000240399279F938F938FEB97E09F938F9352
:104EE000FF92EF92E0912D04F0912E0409958CE34E
:104EF00080936C028DB79EB706968DBF8091250377
:104F000099279F938F938BEC97E04CC010926C0283
:104F10008091260399279F938F9387ED97E09F9326
:104F20008F93FF92EF92FE01099584E180936C02CA
:104F30008DB79EB706968DBF8091270399279F93C3
:104F40008F9383EE97E09F938F93FF92EF92E09180
:104F50002D04F0912E04099588E280936C022DB700
:104F60003EB72A5F3F4F2DBF8091280399279F931B
:104F70008F938FEE97E09F938F93FF92EF92E09144
:104F80002D04F0912E0409958CE380936C028DB76B
:104F90009EB706968DBF8091290399279F938F9383
:104FA0008BEF97E09F938F93FF92EF92D5CA109269
:104FB0006C0287E098E09F938F93FF92EF92FE013F
:104FC000099584E180936C020F900F900F900F90E1
:104FD0008091A30199279F938F938FE098E09F93EF
:104FE0008F93FF92EF92E0912D04F0912E0409959A
:104FF00088E280936C028DB79EB706968DBF809134
:105000001F02909120029F938F938DE198E09F93D0
:105010008F93FF92EF92E0912D04F0912E04099569
:105020008CE380936C022DB73EB72A5F3F4F2DBFB4
:105030008091390699279F938F93809138069927FD
:105040009F938F938BE298E09F938F93FF92EF92C1
:10505000E0912D04F0912E0409958DB79EB7089626
:10506000F7C010926C0289E398E09F938F93FF92B0
:10507000EF92FE01099584E180936C020F900F90EE
:105080000F900F9080916704992787FD90959F93CB
:105090008F9380916604992787FD90959F938F93B6
:1050A00089E498E09F938F93FF92EF92E0912D0413
:1050B000F0912E04099588E280936C022DB73EB7DB
:1050C000285F3F4F2DBF80916804992787FD9095F9
:1050D0009F938F938091690499279F938F9389E57C
:1050E00098E09F938F93FF92EF92E0912D04F091BF
:1050F0002E0409958CE380936C028DB79EB70896B9
:105100008DBF80916D0499279F938F9380916A043E
:10511000992787FD90959F938F9389E698E031CBEF
:1051200010926C0289E798E09F938F93FF92EF9221
:10513000FE01099584E180936C020F900F900F900F
:105140000F908091EB0699278F7790709F938F93A4
:105150008091E30699278F7790709F938F9380912A
:10516000DB0699278F7790709F938F938091D3065A
:1051700099278F7790709F938F9389E898E09F93FA
:105180008F93FF92EF92E0912D04F0912E040995F8
:1051900088E280936C028DB79EB70C968DBF80918C
:1051A0000B0799278F7790709F938F9380910307B8
:1051B00099278F7790709F938F938091FB06992703
:1051C0008F7790709F938F938091F30699278F77B5
:1051D00090709F938F938AE998E09F938F93FF92AB
:1051E000EF92E0912D04F0912E0409958CE38093C9
:1051F0006C022DB73EB7245F3F4F2DBF80912B0728
:1052000099278F7790709F938F9380912307992789
:105210008F7790709F938F9380911B0799278F773B
:1052200090709F938F938091130799278F77907039
:105230009F938F938BEA98E09F938F93FF92EF92C7
:10524000E0912D04F0912E0409958DB79EB70C9630
:105250008DBFFEC110926C028CEB98E09F938F93F0
:10526000FF92EF92FE01099584E180936C020F900A
:105270000F900F900F908091EF06992787FD9095E2
:105280009F938F938091E706992787FD90959F9331
:105290008F938091DF06992787FD90959F938F9339
:1052A0008091D706992787FD90959F938F938BECDC
:1052B00098E09F938F93FF92EF92E0912D04F091ED
:1052C0002E04099588E280936C022DB73EB7245FC7
:1052D0003F4F2DBF80910F07992787FD90959F9392
:1052E0008F9380910707992787FD90959F938F93C0
:1052F0008091FF06992787FD90959F938F938091CA
:10530000F706992787FD90959F938F938CED98E0F2
:105310009F938F93FF92EF92E0912D04F0912E04D2
:1053200009958CE380936C028DB79EB70C968DBF68
:1053300080912F07992787FD90959F938F93809158
:105340002707992787FD90959F938F9380911F073B
:10535000992787FD90959F938F93809117079927A1
:1053600087FD90959F938F938DEE98E09F938F93F9
:10537000FF92EF92E0912D04F0912E0409952DB744
:105380003EB7245F3F4F2DBF63C110926C028EEF7A
:1053900098E09F938F9307E610E2FF92EF92FE0151
:1053A000099584E180936C020F900F900F900F90FD
:1053B0008091EB06881F8827881F97E0899FC0018E
:1053C00011248D969F938F938091E306881F8827E1
:1053D000881F96E0899FC00111248D969F938F931B
:1053E0008091DB06881F8827881F95E0899FC00170
:1053F00011248D969F938F938091D306881F8827C1
:10540000881F9927880F991F880F991F8D969F9342
:105410008F938DE099E09F938F93FF92EF92E091AD
:105420002D04F0912E04099588E280936C028DB7CB
:105430009EB70C968DBF80910B07881F8827881F09
:105440009BE0899FC00111248D969F938F9380913B
:105450000307881F8827881F9AE0899FC0011124AD
:105460008D969F938F938091FB06881F8827881FB6
:1054700099E0899FC00111248D969F938F9380910D
:10548000F306881F8827881F992723E0880F991F14
:105490002A95E1F78D969F938F9381E299E09F93F0
:1054A0008F93FF92EF92E0912D04F0912E040995D5
:1054B0008CE380936C022DB73EB7245F3F4F2DBF26
:1054C00080911307881F8827881F9CE0899FC0014F
:1054D00011248D969F938F9385E399E09F938F93EB
:1054E000FF92EF92E0912D04F0912E0409958091A6
:1054F0001B072DB73EB72A5F3F4F2DBF87FF12C056
:1055000080E480936C0286E499E09F938F93FF92EE
:10551000EF92E0912D04F0912E0409950F900F90D9
:105520000F900F908091230787FF12C084E480932F
:105530006C0289E499E09F938F931F930F93E091FE
:105540002D04F0912E0409950F900F900F900F905D
:1055500080912B0787FF7CC088E480936C028CE4E9
:1055600099E09F938F931F930F93E0912D04F091F7
:105570002E0409950F900F900F900F9069C0109214
:105580006C028FE499E09F938F93FF92EF92FE015C
:10559000099584E180936C020F900F900F900F900B
:1055A0008091F7019091F8019F938F938DE599E099
:1055B0009F938F93FF92EF92E0912D04F0912E0430
:1055C000099588E280936C028DB79EB706968DBFD1
:1055D0008091F9019091FA019F938F938AE699E067
:1055E0009F938F93FF92EF92E0912D04F0912E0400
:1055F000099589E480936C022DB73EB72A5F3F4F2F
:105600002DBF87E799E09F938F93FF92EF92E091F0
:105610002D04F0912E04099580916A020F900F904D
:105620000F900F9083FF14C01092FA011092F901AD
:1056300060E070E08EE090E00E94732E09C08091DF
:105640002101281719F421502093210110926B0297
:1056500010926A02E6E0CDB7DEB70C9445794AEACB
:1056600020E030E02617370740F4FC018191480F15
:105670002F5F3F4F26173707C8F3842F99270895C8
:10568000AC019AEA20E030E02617370750F4DA013F
:10569000A20FB31F0E945A79802D980F2F5F3F4FA2
:1056A000F3CF892F9927089581E080930C0682E03B
:1056B00080930B0683E080930A0684E080930D06B6
:1056C00085E080930E0686E080930F0687E0809346
:1056D000100688E08093110689E0809312068AE024
:1056E000809313068BE0809314068CE0809315065C
:1056F00008951F93CF93DF9384E5809309068091EB
:105700000201843150F08AE08093290610924B0602
:105710008BE1809325068EE40AC083E080932906FE
:1057200080E280934B068EE18093250685E5809389
:105730004806809349068AE68093160683E08093A4
:105740006C06AEE1A09317068FEF80931906EFE089
:10575000E0931A06A093180610921C06F8E0F09346
:105760001D0680E480931E0610921F0684E180933C
:105770001B068EE080932006B0E1B09321061CE06A
:1057800010932206F093230686EE8093240680E889
:105790008093260650E55093270686E980932806D5
:1057A00050932A0680932B0676E070932C0681E2B4
:1057B00080932D068DE280932E069AE590932F0616
:1057C00080E28093310610923206109233061092D6
:1057D00034061092350610924D0610924E06109225
:1057E0004F061092500634E63093360648E2409356
:1057F000370661E060936B061092380627EF20931E
:10580000390670933E068DE780933F0680934006ED
:105810008093410630933A0640933B0610923C0633
:1058200020933D0682E38093420690934306809343
:10583000440610926A06909345065093460660937C
:105840004706B0934A0630934C068FE58093510685
:1058500083EF809353068AEA809355068093560619
:10586000E0935206E09354068EEF809357063093F0
:1058700058069093590690935A0690935B068BE4D2
:1058800080935C0680935D0680935E0610925F06AF
:1058900070936006F093610690936206A09363068E
:1058A000309364063093650682E0809366066093C9
:1058B00030061092680610926906ADE6B6E0E2E79F
:1058C000F1E0ED01019009921A95E1F760E770E0CF
:1058D000CD01845690400E942F2B80937906DF9152
:1058E000CF911F910895CF93DF9384E580930906AC
:1058F00080910201843150F08AE080932906109251
:105900004B068BE1809325068EE40AC083E08093EA
:10591000290680E280934B068EE18093250685E57B
:1059200080934806809349068AE68093160683E0B2
:1059300080936C067EE1709317068FEF80931906B3
:105940009FE090931A067093180610921C0668E068
:1059500060931D0680E480931E0610921F069093AC
:105960001B068AE08093200680E18093210656E0A2
:10597000509322066093230686EE8093240680E8E7
:10598000809326062AE52093270688E78093280639
:1059900020932A0680932B0650932C0681E2809355
:1059A0002D068DE280932E0620932F06E0E2E093F1
:1059B000310610923206109233061092340610927D
:1059C000350610924D0610924E0610924F06109218
:1059D000500644E64093360638E230933706F1E04D
:1059E000F0936B061092380697EF90933906509318
:1059F0003E068DE780933F068093400680934106E4
:105A000040933A0630933B0610923C0690933D0635
:105A100082E38093420620934306809344061092CB
:105A20006A062093450680E5809346068CE38093C2
:105A30004706E0934A069BE490934C068FE58093DB
:105A4000510683EF809353068AEA8093550680932C
:105A5000560684E180935206809354068EEF80931D
:105A60005706409358062093590620935A062093D0
:105A70005B0690935C0690935D0690935E06109291
:105A80005F065093600660936106209362067093F0
:105A90006306409364064093650682E08093660641
:105AA000F09330061092680610926906ADE6B6E0F3
:105AB0008CE0E9E7F1E0ED01019009928A95E1F7C8
:105AC00060E770E0CD01845690400E942F2B8093B8
:105AD0007906DF91CF910895CF93DF9384E580938A
:105AE000090680910201843150F08AE080932906F2
:105AF00010924B068BE1809325068EE40AC083E06A
:105B00008093290680E280934B068EE180932506E0
:105B100085E580934806809349068AE680931606B9
:105B200083E080936C066EE1609317068FEF80939D
:105B300019069FE090931A066093180610921C06AF
:105B400078E070931D0680E480931E0610921F0675
:105B500090931B067093200690E19093210656E0E7
:105B6000509322067093230686EE8093240680E8E5
:105B70008093260634E63093270688E7809328062C
:105B800030932A0680932B0650932C0681E2809353
:105B90002D068DE280932E062AE520932F06909302
:105BA000310610923206109233061092340610928B
:105BB000350610924D0610924E0610924F06109226
:105BC00050063093360648E240933706E1E0E09312
:105BD0006B061092380697EF9093390650933E0665
:105BE0008DE780933F068093400680934106309373
:105BF0003A0640933B0610923C0690933D0682E3A2
:105C000080934206209343068093440610926A06CE
:105C10002093450680E58093460696E490934706D8
:105C200080E280934A0690934C068FE5809351065C
:105C300083EF809353068AEA809355068093560635
:105C400060935206609354068EEF8093570630930C
:105C500058062093590620935A0620935B068BE43E
:105C600080935C0680935D0680935E0610925F06CB
:105C700050936006709361062093620660936306FA
:105C8000309364063093650682E080936606E09365
:105C900030061092680610926906ADE6B6E08CE018
:105CA000E1E8F1E0ED01019009928A95E1F760E702
:105CB00070E0CD01845690400E942F2B809379068E
:105CC000DF91CF910895DC010E945A79802D9927A8
:105CD0000895DC01062E0E946C790895DC010E9473
:105CE0006779CF010895DC010B010E94787908954E
:105CF000FF920F931F93CF93DF93982F815085309E
:105D000008F093E081E7F82E9F9D80011124E801BF
:105D10002D9760E770E0CE010E94402B982FD801AC
:105D2000AD59BF4F0E945A79802D891731F4DE0199
:105D30000E945A79802D843519F080E090E00AC0E5
:105D4000E9E0F6E0DE011F2C0E9462790E942168E2
:105D500081E090E0E5E0CDB7DEB70C94467986307F
:105D600010F085E003C0882309F481E0A2E0B0E0F0
:105D7000082E0E946C7908951F93CF93DF93182FFC
:105D8000C9E0D6E080910906843591F5163010F00F
:105D900015E002C0112361F160E770E089E096E050
:105DA0000E942F2B8093790681E7189FD001112440
:105DB0001D97FE01182E0E947D79EAE0F6E0A0E52D
:105DC000B0E02CE030E0122E0E947D79B9018AE02B
:105DD00096E00E942F2BACE5B0E0082E0E946C7973
:105DE000812F0E94AF2E0E94216881E090E002C0C6
:105DF00080E090E0DF91CF911F9108956DE470E015
:105E000088EE93E00E94402BA5E3B4E00E945A790B
:105E1000902D981739F4A8EEB3E00E945A79802D9E
:105E2000813019F080E090E00895EAE7F6E0A8EE0E
:105E3000B3E08EE4182E0E94627981E090E008952C
:105E4000CF93DF93CAE7D6E080917A06813089F458
:105E50006DE470E0CE010E942F2B8093C706A8EE60
:105E6000B3E08EE4FE01182E0E947D7981E090E07F
:105E700002C080E090E0DF91CF910895CF93DF934F
:105E800081E080937A06EAE7F6E08FE015861686D1
:105E90001786108A8150349687FFF8CF80E480936C
:105EA0008706809388061092890680938A068093DD
:105EB0008B0690EC90938C0610928D0680938E0644
:105EC00080938F061092900690939106909392067D
:105ED000809393061092940680939506909396066D
:105EE000ABE7B6E087E0EBE8F1E0ED010190099265
:105EF0008A95E1F76DE470E0CD0101970E942F2BA8
:105F00008093C706DF91CF910895A2E0B0E00E9490
:105F10005A79802D863030F083E0A2E0B0E0082E80
:105F20000E946C7999270895DF92EF92FF920F9368
:105F30001F93CF93FF24DF2CEF2C81E090E00E9491
:105F4000632E843539F031E0E32E64E581E090E0A2
:105F50000E94692E6CE070E080E590E00E94402B8A
:105F6000C82FACE5B0E00E945A79802D8C1711F44F
:105F700021E0D22EC1E001E010E0EE2029F48C2FC8
:105F80000E94782E8823B1F591E0F92E1F930F938C
:105F90008FE799E09F938F938CE692E19F938F9385
:105FA000E0912D04F0912E0409958DB79EB70696C9
:105FB0008DBF0230110549F0033011054CF401305A
:105FC000110531F40E94792B05C00E94732C02C088
:105FD0000E946C2DDD2049F0EAE0F6E0A0E5B0E09B
:105FE0008CE0182E0E94627902C00E94542B8C2FE4
:105FF0000E94BC2ECF5F0F5F1F4FC63008F4BDCF8D
:10600000FF2019F083E00E94AF2E0E94852FC82F39
:106010000E94782E8C2F99279F938F9385EA99E081
:106020009F938F930CE612E11F930F93E0912D0441
:10603000F0912E0409958DB79EB706968DBFEE2080
:1060400021F40E94FE2E882399F48EEB99E09F9311
:106050008F931F930F93E0912D04F0912E040995D7
:106060000E943E2F0E94202F0F900F900F900F90B4
:106070001092080690E0E7E8F6E0CFE080813496E1
:1060800018160CF49F5FC150C7FFF8CF9093080615
:10609000892F99279F938F938BE796E09F938F93F8
:1060A0008FED99E09F938F931F930F93E0912D04B1
:1060B000F0912E0409958DB79EB708968DBF80E0AC
:1060C0009AE09F938F931F930F93E0912D04F0918B
:1060D0002E0409950F900F900F900F90CF911F9164
:1060E0000F91FF90EF90DF9008959FB7F894399843
:1060F000389A88B1836088B98091B9008C7F809389
:10610000B9008AE28093B80010927602109274026D
:1061100010927302E0EDF6E08BE0108211821282A1
:10612000138214821582168217828150389687FF57
:10613000F4CF9FBF08951092760284E98093BC004B
:10614000109274021092730280E88093BC00109247
:10615000BD001092BA001092BB001092B9001092CC
:10616000B8000E9475301092BB0085E88093BC0097
:106170008091710282608093710208951F920F9244
:106180000FB60F9211242F933F934F935F938F93EA
:106190009F93EF93FF9380917602282F3327442714
:1061A00055278F5F80937602F9012731310508F07A
:1061B000B3C2EE59FF4F0C945479809174028C3025
:1061C00090F4809174028F5F8093740280917402C6
:1061D000E82FFF27EE0FFF1FEE0FFF1FE658F94FC6
:1061E0008585181654F7809174028C3070F01092E7
:1061F000700210926F021092740285E08093760212
:1062000080917302880F8D5A04C080917402880FA8
:106210008E5A8093BB0085E874C280917402E82F87
:10622000FF2783E0EE0FFF1F8A95E1F7E053F94F58
:1062300081818093BB0085E88093BC0080917402CB
:10624000E82FFF27EE0FFF1FEE0FFF1FEE0FFF1FC0
:10625000E053F94F808180FF91C080917402E82F54
:10626000FF27EE0FFF1FEE0FFF1FEE0FFF1FE05384
:10627000F94F8281882329F080910806873008F43D
:106280005FC280916F0290917002892B09F058C211
:1062900080916D0290916E02892B09F051C26EC0FF
:1062A0008091740221E030E002C0220F331F8A95F2
:1062B000E2F780916D0290916E0228233923232BFF
:1062C00079F080917402E82FFF27EE0FFF1FEE0F89
:1062D000FF1FEE0FFF1FE053F94F80E184830DC0D5
:1062E00080917402E82FFF27EE0FFF1FEE0FFF1FB4
:1062F000EE0FFF1FE053F94F148280917402E82FD4
:10630000FF2753E0EE0FFF1F5A95E1F7E053F94FD7
:106310008481282F332743E0220F331F4A95E1F76A
:1063200080917402E82FFF2793E0EE0FFF1F9A95EC
:10633000E1F7E053F94F82818770822B8093BB0095
:1063400085E88093BC002091740281E090E002C057
:10635000880F991F2A95E2F720916F023091700201
:1063600082239323892B51F088EC96E090937A0254
:106370008093790288E080937B02E2C184E080C14F
:10638000E0917902F0917A0281918093BB0085E8D7
:106390008093BC00F0937A02E093790280917B02B3
:1063A000815080937B02882309F4CAC183E068C1CD
:1063B0008091B900803351F580917702882329F4C8
:1063C000809174028F5F8093770280917402E82F2E
:1063D000FF2783E0EE0FFF1F8A95E1F7E053F94FA7
:1063E000838199278F7790708F3791057CF4809106
:1063F0007402E82FFF27EE0FFF1FEE0FFF1FEE0FB7
:10640000FF1FE053F94F83818F5F838310927602E1
:1064100084E98093BC008AE090E09093940180939B
:106420009301809174028F5F8093740210927602C0
:1064300062C18091B9008034A9F180917302E82F84
:10644000FF27EE0FFF1FEE0FFF1FEE0FFF1FE053A2
:10645000F94F83818F778383809173028F5F80935D
:106460007302809173028C30A0F01092730210922C
:106470006E0210926D02809178028F5F8093780295
:106480008C3038F010927802809171028D7F809369
:106490007102809171028160809371021092760284
:1064A00084E971C080917302E82FFF27EE0FFF1F70
:1064B000EE0FFF1FEE0FFF1FE053F94F838180683F
:1064C000838380917302E82FFF27EE0FFF1FEE0FEB
:1064D000FF1FEE0FFF1FE053F94F808180FF2FC099
:1064E00080917302E82FFF2753E0EE0FFF1F5A95AC
:1064F000E1F7E053F94F84819927009751F04097D5
:10650000D9F588EC96E090937A028093790288E03E
:1065100031C080917302992743E0880F991F4A95F3
:10652000E1F78B52994F90937A0280937902909180
:106530007302809178029817E1F483E01BC0809188
:106540007302992733E0880F991F3A95E1F78B5230
:10655000994F90937A02809379028091710281FD24
:1065600006C09091730280917802981711F482E02E
:1065700001C081E080937B0280917B02813011F425
:1065800085E801C085EC8093BC0080917702809300
:10659000720210927702D4C0E0917902F0917A02EF
:1065A0008091BB0080838091790290917A0201965C
:1065B00090937A028093790280917B02815080933C
:1065C0007B02823010F085EC58C0813011F485E8F0
:1065D00054C08091710281FF2DC08091ED0280FD39
:1065E0001DC080917302E82FFF2723E0EE0FFF1FED
:1065F0002A95E1F7E053F94F86818A3F79F480913B
:106600007302E82FFF2793E0EE0FFF1F9A95E1F743
:10661000E053F94F8081816080830CC080917302C8
:10662000E82FFF2783E0EE0FFF1F8A95E1F7E05385
:10663000F94F1082809173028F5F80937302809173
:1066400073028C30A0F01092730210926E021092BE
:106650006D02809178028F5F809378028C3038F0E1
:1066600010927802809171028D7F80937102109256
:10667000760284E98093BC0049C08093BC0086E028
:10668000809376025DC088E9C4CD80917502880F41
:10669000805FBFCD8091750299278130910561F0AF
:1066A000823091051CF4892B21F04AC0029739F001
:1066B00047C080911401ADCD80911301AACD809186
:1066C0001201A7CD80E8A5CD1092760284E98093CF
:1066D000BC008AE090E090939401809393018091B4
:1066E0007502823088F4809175028F5F8093750205
:1066F00082E180937602809171028E7F8093710295
:1067000085EA8093BC001CC01092750280917102D2
:1067100081608093710214C01092760284E98093A4
:10672000BC00809171028160809371028AE090E0E8
:1067300090939401809393011092740210927302CB
:10674000FF91EF919F918F915F914F913F912F9189
:106750000F900FBE0F901F9018951F93CF93DF934C
:10676000182F80911803882321F480910402882334
:1067700019F081E090E097C01D3008F092C011231D
:10678000B1F0E12FFF2723E0EE0FFF1F2A95E1F77D
:10679000E053F94F35978081359688230CF081C0FE
:1067A0003897808180FD03C083E090E07CC08091B9
:1067B000C806823019F084E090E075C067E070E0B0
:1067C00088EC96E00E942F2B9091CF06891719F044
:1067D00085E090E068C080ED97E00E949316EC01A0
:1067E0008091710280FD05C0CE010E949C16882315
:1067F000B9F3112319F48FEF90E00BC0212F332749
:106800002150304081E090E002C0880F991F2A9506
:10681000E2F79093700280936F02A1E0B0E0E0EDA8
:10682000F6E040E050E06BE0CD01042E02C0880F9E
:10683000991F0A94E2F720916F023091700282232F
:106840009323892B11F01182128261504F5F5F4FA9
:10685000389667FFE9CF1092740210927602809109
:1068600071028E7F8093710285EA8093BC008091D3
:10687000710280FD05C0CE010E949C168823B9F3E9
:1068800080916F0290917002892B29F0CE010E94B5
:106890009C16882311F380916F02909170020097EB
:1068A00011F082E090E0DF91CF911F9108950F9356
:1068B0001F93CF93DF93982F80911803882321F49F
:1068C00080910402882319F081E090E092C09D300D
:1068D000A0F4992319F486E090E08BC0C92FDD273E
:1068E000FE0133E0EE0FFF1F3A95E1F7E053F94F59
:1068F00035978081359687FD03C082E090E079C0AE
:106900003897808180FD03C083E090E072C080ED05
:1069100097E00E9493168C018091710280FD05C062
:10692000C8010E949C168823B9F3219721E030E02A
:10693000C90102C0880F991FCA95E2F790936E02B1
:1069400080936D02D901E0EDF6E040E050E06BE0AD
:10695000CD01042E02C0880F991F0A94E2F72091FE
:106960006D0230916E0282239323892B11F01182E4
:10697000128261504F5F5F4F389667FFE9CF1092E8
:1069800073021092C8061092CF0610927602809180
:1069900071028E7F8093710285EA8093BC008091A2
:1069A000710280FD05C0C8010E949C168823B9F3BE
:1069B00080916D0290916E02892B29F0C8010E948E
:1069C0009C16882311F38091C806823019F084E068
:1069D00090E00FC067E070E088EC96E00E942F2BFB
:1069E0009091CF06891719F085E090E002C080E011
:1069F00090E0DF91CF911F910F91089589E1A5E675
:106A0000B7E0E1E3F7E011821082329611961C9212
:106A10001E921296815087FFF6CF10928703109234
:106A20008603109289031092880310928B031092B0
:106A30008A0308951F920F920FB60F9211240F939D
:106A40001F932F933F934F935F936F937F938F93F6
:106A50009F93AF93BF93CF93DF93EF93FF93809177
:106A60006C0682FDCFC040918600509187008091D6
:106A70007D0290917E02481B590B80918600909177
:106A8000870090937E0280937D02CA018D549440CA
:106A9000A0917F02B0918002835F9A4178F4809147
:106AA0007F0280933007149714F01092950181E0D3
:106AB00090E09093800280937F0207C2AD30B105D1
:106AC0000CF003C2CA018B5F9040845B914008F0D8
:106AD00074C0425D5140FD01EA0FFB1FEF5CF84FAF
:106AE00080819181FA01E81BF90BCF01F7FF03C008
:106AF000909581959F4F06975CF480912103883C87
:106B000020F480912103865F01C088EC80932103EB
:106B1000FD01EA0FFB1FEF5CF84F808191819C0122
:106B2000220F331F280F391F240F351F37FF02C0D4
:106B30002D5F3F4FE901D595C795D595C795CA01FA
:106B400001968C179D0714F4219706C041505040C0
:106B5000C417D5070CF4219680912103833CE0F003
:106B60008D010A0F1B1FF801EF5CF84F80819181A6
:106B70009E01281B390BC90163E070E00E94CD78AB
:106B8000CB01880F991F860F971F0B59184FD801FB
:106B900011969C938E9307C0AA0FBB1FAB59B84F99
:106BA00011961C921E92E0917F02F0918002EE0FEE
:106BB000FF1FEF5CF84FD183C08320917F0230919B
:106BC00080022F5F3F4F3093800220937F0280919D
:106BD0000201843108F079C12530310511F45D9A44
:106BE00001C05D9880917F0290918002863091056E
:106BF00011F45C9A01C05C98079711F45B9A65C127
:106C00005B9863C14091860050918700809181021A
:106C100090918202481B590B8091860090918700C9
:106C20009093820280938102CA018D5494406091B6
:106C3000EB02835F9A4108F07AC060937C028091F6
:106C40007C02843008F453C09091300780917C021C
:106C5000981709F04CC05091EC025B3008F43FC02B
:106C6000109295011092EB0240E05F31C0F0E42FEA
:106C7000FF27EE0FFF1F9F0129543D4FDF01AF5C3F
:106C8000B84F8D919C91D9018D939C93DF01AB59A5
:106C9000B84F8D919C91EF52FD4F91838083E42FEB
:106CA000FF27EE0FFF1F9F012F5C384FDF01AD570D
:106CB000BD4F8D919C91D90111969C938E93DF01CC
:106CC000A356BD4F8D919C91EB59F84F91838083D2
:106CD000842F8F5F482F8D3040F28093EB0280919C
:106CE000EC028F3FB9F08F5F8093EC0213C080916C
:106CF000EC02853620F08AE08093EC0202C010920C
:106D0000EC02809102018A3011F0843110F0289A4F
:106D100001C0289881E08093EB02809118038823BA
:106D200009F0D3C080917C0280933007CEC06D30D3
:106D300008F0A3C0CA018B5F9040845B914008F0CB
:106D40007EC0425D5140E62FFF27EE0FFF1FED573B
:106D5000FD4F80819181FA01E81BF90BCF01059667
:106D60000B97B0F48091EC028A3120F080912103DE
:106D7000865F05C08B3028F0809121038E5F809361
:106D8000210380912103893C18F088EC8093210332
:106D9000E62FFF27EE0FFF1FED57FD4F80819181FA
:106DA0009C01220F331F280F391F240F351F37FF77
:106DB00002C02D5F3F4FE901D595C795D595C79581
:106DC000CA0101968C179D0714F4219706C0415003
:106DD0005040C417D5070CF42196809121038E3BB7
:106DE000D8F0E62FFF27EE0FFF1FDF01AD57BD4F95
:106DF0008D919C919E01281B390BC90163E070E0C5
:106E00000E94CD78CB01880F991F860F971FE356FC
:106E1000FD4F9183808308C0E62FFF27EE0FFF1FF1
:106E2000E356FD4F118210828091EB02E82FFF277D
:106E3000EE0FFF1FED57FD4FD183C08309C0809136
:106E400002018A3011F0843110F0289A01C028988C
:106E500080910201843188F48091EB02853011F435
:106E60005D9A05C05D98863011F45C9A05C05C9807
:106E7000873011F45B9A01C05B988091EB028431FA
:106E800020F48F5F8093EB0220C08431F1F4809175
:106E900002018A3011F0843110F0289A01C028983C
:106EA0008EE18093EB022CE0C5E6D7E0A7EBB2E0E1
:106EB000E1E3F7E08D919D91918380833296198271
:106EC00018822296215027FFF5CFFF91EF91DF9195
:106ED000CF91BF91AF919F918F917F916F915F9172
:106EE0004F913F912F911F910F910F900FBE0F90D7
:106EF0001F901895EF92FF920F931F938091250694
:106F00009927880F991F880F991F7C010027F7FC8C
:106F10000095102F8091750390917603A0917703CF
:106F2000B0917803BC01CD01A80197010E940279BC
:106F30003093B5052093B40580916D0390916E0355
:106F4000A0916F03B0917003BC01CD01A80197011E
:106F50000E9402793093B7052093B6058091EB0724
:106F60009091EC0797FD0396959587959595879554
:106F70009093B9058093B8058091FB079091FC0729
:106F800097FD039695958795959587959093BB0565
:106F90008093BA05809186039091870320914802DF
:106FA00030914902821B930B9093BD058093BC05E1
:106FB0008091130390911403A0911503B0911603CF
:106FC000BC01CD0125E030E040E050E00E940279B4
:106FD0003093BF052093BE058091420290914302F9
:106FE0009093C1058093C005809133039091340341
:106FF0009093C5058093C40580911F019091200155
:107000009093C7058093C60580912103992790939B
:10701000C9058093C8058091F7079091F807A09162
:10702000F907B091FA0720919701309198014091AA
:10703000990150919A01BC01CD010E9402793093CF
:10704000CB052093CA058091D10699279093CD0551
:107050008093CC058091D90699279093CF05809392
:10706000CE058091E10699279093D1058093D005B4
:107070008091E90699279093D3058093D20580915A
:107080001F02909120029093DD058093DC05809192
:107090006E0890916F089093E1058093E0058091D0
:1070A0007208909173089093E3058093E2058091B4
:1070B000740899279093EF058093EE058091FE0365
:1070C0009091FF039093F1058093F0058091FC036C
:1070D0009091FD039093F3058093F205809146040F
:1070E000882321F480914704882321F08091B305FF
:1070F000816003C08091B3058E7F8093B3051F919B
:107100000F91FF90EF9008951F93CF93DF93182F67
:10711000EB01809118038823A1F411501F3F89F0DF
:10712000D0932402C09323028091230290912402E1
:10713000892BD1F7CE018C0F9D1F0E94A8161150EC
:1071400078F7DF91CF911F910895CF93DF938091CE
:1071500002018D3011F40E949B1B10927A008091E5
:107160004C0290914D029093B2078093B1078091A9
:107170004A0290914B029093A3078093A2078091BB
:107180004802909149029093F1078093F007209173
:10719000440230914502C901880F991F880F991F39
:1071A000820F931F820F931F9093EC078093EB073E
:1071B0002091460230914702C901880F991F880F1C
:1071C000991F820F931F820F931F9093FC07809348
:1071D000FB078FEC80937A00A2E2B3E0CEE0D6E02A
:1071E00097E08991E82FFF27EE0FFF1FEF5CF84F24
:1071F0000190F081E02DE259FF4F1E161F061CF092
:10720000E0E0F0E005C0EF3FF10514F0EFEFF0E053
:107210008C91282F3327E217F30714F4815004C010
:107220002E173F0714F48F5F8C939150119697FFA0
:10723000D8CF809148069927AA27BB27BC01CD014A
:1072400024EC39E040E050E00E948E78DC01CB0174
:107250008093B7019093B801A093B901B093BA019C
:10726000809149069927AA27BB27BC01CD010E941E
:107270008E78DC01CB018093B3019093B401A0938D
:10728000B501B093B601DF91CF910895A0E0B0E0D1
:10729000ECE4F9E30C942379882EC0E0D0E07E0181
:1072A0006E0110924604469AD0938103C0938003E6
:1072B000D0937F03C0937E03D0937B03C0937A0364
:1072C000D0938B03C0938A03D0938903C093880320
:1072D000D0938703C09386031092A00110929F0160
:1072E00010923C020E94A53884E690E00E94B516F8
:1072F0000E94A5388091160680FF10C0809115016C
:1073000090911601875B934038F48091150190911C
:1073100016018E5E924010F40E94401B0FE18AE03D
:1073200090E00E94B5168091480290914902C80FE2
:10733000D91F80914C0290914D02E80EF91E809168
:107340004A0290914B02C80ED91E015007FFE7CFA9
:107350009701205F3F4F36952795369527953093B7
:107360008B0320938A03C601409696958795969540
:10737000879590938903809388036096F5E0D6956E
:10738000C795FA95E1F7D0938703C093860390934E
:1073900085038093840330938303209382038820A2
:1073A00009F441C08091EB079091EC0797FF03C06F
:1073B000909581959F4F6CE070E00E94CD789B0185
:1073C00070938103609380038091FB079091FC0789
:1073D00097FF03C0909581959F4F6CE070E00E94ED
:1073E000CD7870937F0360937E038091FB0590912D
:1073F000FC0590937B0380937A03B90184E090E0CD
:107400000E94732E60917E0370917F0386E090E06E
:107410000E94732E60917A0370917B0388E090E064
:107420000E94732E65C084E090E00E946E2E9093BF
:1074300081038093800386E090E00E946E2E9093FB
:107440007F0380937E0388E090E00E946E2E9C0173
:1074500090937B0380937A038091800390918103C2
:107460008150984050F480917E0390917F03815029
:10747000984018F421503440D8F181E29AE09F936B
:107480008F938CE692E19F938F93E0912D04F0917E
:107490002E0409958091EB079091EC0797FF03C0AC
:1074A000909581959F4F6CE070E00E94CD7870932D
:1074B0008103609380038091FB079091FC0797FF05
:1074C00003C0909581959F4F6CE070E00E94CD784D
:1074D00070937F0360937E038091FB059091FC0580
:1074E00090937B0380937A030F900F900F900F90EF
:1074F0001092B2071092B1071092A3071092A20740
:107500001092F1071092F00784E690E00E94B51601
:1075100080914402909145029C01220F331F220F5B
:10752000331F280F391F280F391F3093EC07209382
:10753000EB0780914602909147028C01000F111FCA
:10754000000F111F080F191F080F191F1093FC07B8
:107550000093FB0780912506C82EDD24EE24FF242E
:10756000442737FD4095542FC701B6010E948E78FD
:107570004B015C01609375037093760380937703EE
:10758000909378039801442737FD4095542FC70105
:10759000B6010E948E78DC01CB0180936D0390933D
:1075A0006E03A0936F03B093700380925103909287
:1075B0005203A0925303B0925403809349039093D3
:1075C0004A03A0934B03B0934C03109245031092CF
:1075D000460310924703109248038091170190913F
:1075E0001801A0911901B0911A019093FE058093A2
:1075F000FD0510923B0210923A0210923503109250
:107600003603109237031092380380913303909120
:10761000340390933203809331030E94B86382E372
:1076200090E090932402809323028091480699274A
:10763000AA27BB27BC01CD0124EC39E040E050E093
:107640000E948E78DC01CB018856954CAF4FBF4F1E
:107650008093B7019093B801A093B901B093BA0198
:10766000809149069927AA27BB27BC01CD010E941A
:107670008E78DC01CB018856954CAF4FBF4F80937D
:10768000B3019093B401A093B501B093B6011092E9
:107690009C0110929B018091330390913403AA279F
:1076A00097FDA095BA2F20919701309198014091B4
:1076B000990150919A01BC01CD010E948E78DC01A4
:1076C000CB018093F7079093F807A093F907B09345
:1076D000FA0710922C0310922B0381E08093010192
:1076E0000E9421688091ED0284608093ED028FEF0B
:1076F0008093690810926A0880E280936B08C2E266
:10770000D3E0AEE0B6E007E08D91E82FFF27EE0F63
:10771000FF1FEF5CF84F808191818259899301505E
:1077200007FFF2CF84E68093210380912102882312
:1077300011F0469A579A80918A0390918B03805654
:107740009940815C9B4228F080914604816080933F
:107750004604809188039091890380569940815C0A
:107760009B4228F080914604826080934604809179
:107770008603909187038C5291408957954028F059
:1077800080914604846080934604809180039091A8
:1077900081038C529140835C914028F08091460493
:1077A00088608093460480917E0390917F038C5281
:1077B0009140835C914028F08091460480618093E1
:1077C000460480917A0390917B03805092408355C8
:1077D000914028F080914604806280934604ECE05A
:1077E000CDB7DEB70C943F79A3E1B0E0EAEFFBE35D
:1077F0000C941D7980918603909187032091480213
:1078000030914902821B930B9093F1078093F0070C
:10781000809152029091530297FD07969C0153E08C
:10782000359527955A95E1F73093B2072093B10724
:10783000809150029091510297FD079643E09595F3
:1078400087954A95E1F79093A3078093A207309319
:10785000BD072093BC079093B5078093B407809130
:10786000EB079091EC07AC01440F551F480F591FCF
:107870002091440230914502C901880F991F880F59
:10788000991F820F931F820F931F480F591F57FF95
:1078900002C04D5F5F4F559547955595479550935D
:1078A000EC074093EB078091FB079091FC07AC013C
:1078B000440F551F480F591F20914602309147022F
:1078C000C901880F991F880F991F820F931F820F7C
:1078D000931F480F591F57FF02C04D5F5F4F5595CB
:1078E0004795559547955093FC074093FB0720918A
:1078F000440230914502C901880F991F880F991FD2
:10790000820F931F820F931F9C01442737FD4095E0
:10791000542F8091650390916603A0916703B09105
:107920006803820F931FA41FB51F80936503909374
:107930006603A0936703B0936803209146023091D9
:107940004702C901880F991F880F991F820F931F43
:10795000820F931F9C01442737FD4095542F80913F
:10796000610390916203A0916303B0916403820F5D
:10797000931FA41FB51F8093610390936203A0938C
:107980006303B09364038091C6079091C707209169
:10799000440230914502820F931F9093C707809352
:1079A000C6078091F3079091F40720914602309129
:1079B0004702820F931F9093F4078093F3078091FF
:1079C0007C0390917D03019690937D0380937C03CB
:1079D0008091FB059091FC0520917A0330917B0307
:1079E000821B930B9C01442737FD4095542F8091B7
:1079F0005D0390915E03A0915F03B0916003820FDD
:107A0000931FA41FB51F80935D0390935E03A09303
:107A10005F03B09360038FEC80937A0010921101A2
:107A200020914D0330914E0340914F0350915003EC
:107A300029873A874B875C8729543B464140504011
:107A40002CF028E43BE641E050E00DC089859A85A2
:107A5000AB85BC85885B9449AE4FBF4F4CF428EB97
:107A600034E94EEF5FEF2D833E834F83588708C084
:107A700089859A85AB85BC858D839E83AF83B887C6
:107A8000209155033091560340915703509158036C
:107A90002D873E874F87588B29543B4641405040A5
:107AA0002CF028E43BE641E050E00DC08D859E853A
:107AB000AF85B889885B9449AE4FBF4F4CF428EB33
:107AC00034E94EEF5FEF29833A834B835C8308C030
:107AD0008D859E85AF85B88989839A83AB83BC8366
:107AE000A091F007B091F107BB8BAA8BFD01CF01EC
:107AF000AA2797FDA095BA2FA0904503B090460302
:107B0000C0904703D0904803A80EB91ECA1EDB1EC2
:107B1000A0924503B0924603C0924703D092480317
:107B2000E090F707F090F8070091F9071091FA0735
:107B3000E80EF91E0A1F1B1FE092F707F092F807E4
:107B40000093F9071093FA07F0910803F98BFF23CC
:107B500009F098C180910703882309F093C18091AF
:107B6000160686FF8FC18091A2079091A307AA27CE
:107B700097FDA095BA2FBC01CD0129813A814B8197
:107B80005C810E948E789B01AC0197FF04C021505C
:107B9000384F4F4F5F4F6BE0559547953795279579
:107BA0006A95D1F780919F01682E772488249924C3
:107BB000CA01B901A40193010E948E78DC01CB01B6
:107BC0008093960390939703A0939803B09399039F
:107BD000B7FF04C08150904FAF4FBF4F1C012D0124
:107BE0003CE055944794379427943A95D1F72092E6
:107BF0009603309297034092980350929903809194
:107C0000B1079091B207AA2797FDA095BA2FBC01A2
:107C1000CD012D813E814F8158850E948E7897FF3E
:107C200004C06150784F8F4F9F4F2BE095958795FB
:107C3000779567952A95D1F7A40193010E948E78D4
:107C4000DC01CB0180939A0390939B03A0939C0348
:107C5000B0939D03B7FF04C08150904FAF4FBF4F0B
:107C60009C01AD018CE055954795379527958A95F0
:107C7000D1F720939A0330939B0340939C03509336
:107C80009D03809196039091970390939A07809318
:107C9000990780919A0390919B0390939E078093FC
:107CA0009D07221933094409550920939A033093FB
:107CB0009B0340939C0350939D03E20EF31E041F0D
:107CC000151FE092F707F092F8070093F907109359
:107CD000FA0780919E018823B1F457FF04C02F5FFB
:107CE0003F4F4F4F5F4F5595479537952795A21AB0
:107CF000B30AC40AD50AA0924503B0924603C092C3
:107D00004703D09248032A893B8979010027F7FC71
:107D10000095102F80919A0390919B03A0919C0352
:107D2000B0919D03E80EF91E0A1F1B1FC801B70181
:107D300029813A814B815C810E948E789B01AC0144
:107D400097FF04C02150384F4F4F5F4FBBE0559510
:107D5000479537952795BA95D1F78091A001A82E20
:107D6000BB24CC24DD24CA01B901A60195010E94DF
:107D70008E78DC01CB0180938E0390938F03A093C8
:107D80009003B0939103B7FF04C08150904FAF4F61
:107D9000BF4F3C014D01ACE0959487947794679474
:107DA000AA95D1F760928E0370928F038092900310
:107DB00090929103C801B7012D813E814F81588572
:107DC0000E948E7897FF04C06150784F8F4F9F4F6D
:107DD000FBE09595879577956795FA95D1F7A6017C
:107DE00095010E948E78DC01CB01809392039093E1
:107DF0009303A0939403B0939503B7FF04C08150FD
:107E0000904FAF4FBF4FAC01BD01ECE0759567954A
:107E100057954795EA95D1F7409392035093930372
:107E200060939403709395032A893B8937FF03C0BD
:107E3000309521953F4F21343105E4F1D401C30140
:107E400097FE07C0B095A095909581959F4FAF4F35
:107E5000BF4F81389105A105B10584F4DB01CA014A
:107E600077FF07C0B095A095909581959F4FAF4F34
:107E7000BF4F81389105A105B105E4F081E0809301
:107E80002D0318C010929E0710929D0710929A071A
:107E900010929907109292031092930310929403F8
:107EA0001092950310928E0310928F0310929003FC
:107EB000109291038091920390919303A091940367
:107EC000B0919503BC01CD0124E630E040E050E0E4
:107ED0000E940279E0908E03F0908F03E21AF30A79
:107EE000F092B007E092AF0780918E0390918F03DC
:107EF000A0919003B0919103BC01CD0124E630E044
:107F000040E050E00E940279DA01C9012091920319
:107F1000309193038C01021B130B1093A507009360
:107F2000A4078091970190919801A0919901B09137
:107F30009A01BC01CD0128E631E040E050E00E940A
:107F40008E782091F7073091F8074091F90750910A
:107F5000FA07261737074807590764F0261B370B1F
:107F6000480B590B2093F7073093F8074093F90714
:107F70005093FA072091F7073091F8074091F907DD
:107F80005091FA0757FF0CC0260F371F481F591F83
:107F90002093F7073093F8074093F9075093FA07B7
:107FA0006091A2077091A3076E0D7F1D9B0144276E
:107FB00037FD4095542F8091490390914A03A09139
:107FC0004B03B0914C03820F931FA41FB51F8093E6
:107FD000490390934A03A0934B03B0934C038091C1
:107FE0000D0390910E03681B790BCB01AA2797FD17
:107FF000A095BA2F29853A854B855C85820F931F02
:10800000A41FB51F80934D0390934E03A0934F037D
:10801000B0935003C090B301D090B401E090B5018B
:10802000F090B601C816D906EA06FB06C4F488EA41
:1080300091E6A0E0B0E08C199D09AE09BF098093DC
:108040004D0390934E03A0934F03B093500380933E
:10805000490390934A03A0934B03B0934C03222708
:108060003327A9012C193D094E095F0980914D0361
:1080700090914E03A0914F03B09150038217930744
:10808000A407B507B4F4D701C601885A9146A040A9
:10809000B04080934D0390934E03A0934F03B09351
:1080A00050038093490390934A03A0934B03B093EA
:1080B0004C036091B1077091B207600F711F9B0173
:1080C000442737FD4095542F8091510390915203DE
:1080D000A0915303B0915403820F931FA41FB51FA7
:1080E0008093510390935203A0935303B09354038E
:1080F00080910B0390910C03681B790BCB01AA278D
:1081000097FDA095BA2F2D853E854F855889820F02
:10811000931FA41FB51F8093550390935603A093FC
:108120005703B0935803E090B701F090B801009165
:10813000B9011091BA01E816F9060A071B07C4F441
:1081400088EA91E6A0E0B0E08E199F09A00BB10B80
:108150008093550390935603A0935703B09358030D
:108160008093510390935203A0935303B09354030D
:1081700022273327A9012E193F09400B510B80916B
:10818000550390915603A0915703B091580382175D
:108190009307A407B507B4F4D801C701885A9146DC
:1081A000A040B0408093550390935603A09357038B
:1081B000B09358038093510390935203A0935303B9
:1081C000B09354038091450390914603A0914703D7
:1081D000B09148038093590390935A03A0935B0393
:1081E000B0935C038091550390915603A09157037F
:1081F000B09158038093750390937603A09377030F
:10820000B093780380914D0390914E03A0914F035A
:10821000B091500380936D0390936E03A0936F030E
:10822000B09370038091510390915203A091530336
:10823000B09154038093710390937203A0937303DE
:10824000B09374038091490390914A03A0914B032A
:10825000B0914C038093690390936A03A0936B03DE
:10826000B0936C0380911D0190911E0197FD0796BC
:1082700033E0959587953A95E1F79093B20780930F
:10828000B10780911B0190911C0197FD079623E097
:10829000959587952A95E1F79093A3078093A20778
:1082A00080914C0290914D020F9734F488E19CEF3D
:1082B0009093B2078093B10780914C0290914D0248
:1082C000079734F480E398EF9093B2078093B10757
:1082D000209102012A30A9F480914C0290914D0224
:1082E000835F934034F088EE93E09093B2078093DD
:1082F000B10780914C0290914D028A5F9340DCF06F
:1083000014C080914C0290914D02815D974034F0F1
:1083100088EE93E09093B2078093B10780914C026E
:1083200090914D02805E974034F080ED97E09093FD
:10833000B2078093B10780914A0290914B020F9748
:1083400034F488E19CEF9093A3078093A207809177
:108350004A0290914B02079734F480E398EF909390
:10836000A3078093A2072A30A9F480914A02909132
:108370004B02835F934034F088EE93E09093A30721
:108380008093A20780914A0290914B028A5F9340AA
:10839000DCF014C080914A0290914B02815D9740BD
:1083A00034F088EE93E09093A3078093A207809126
:1083B0004A0290914B02805E974034F080ED97E046
:1083C0009093A3078093A207E091AA01EE2309F4FA
:1083D000B7C040911D0150911E0180919E03909164
:1083E0009F03481B590B5093A5034093A40320916E
:1083F0001D0130911E01280F391F37FF02C02F5F6A
:108400003F4F3595279530939F0320939E03413826
:1084100051051CF080E890E005C040585F4F34F4EF
:1084200080E89FEF9093A5038093A4038E2F992754
:10843000A091A403B091A503A89FA001A99F500DEE
:10844000B89F500D112457FF02C0415F5F4F14E0E9
:10845000559547951A95E1F78091B1079091B2072C
:10846000840F951F9093B2078093B10760911B0111
:1084700070911C018091A0039091A103681B790B5E
:108480007093A3036093A20340911B0150911C01C0
:10849000480F591F57FF02C04F5F5F4F55954795D3
:1084A0005093A1034093A003613871051CF080E84C
:1084B00090E005C060587F4F34F480E89FEF9093C0
:1084C000A3038093A2032E2F33278091A2039091C0
:1084D000A303829FB001839F700D929F700D1124A2
:1084E000AB0177FF02C0415F5F4FE4E055954795D0
:1084F000EA95E1F78091A2079091A307840F951F59
:108500009093A3078093A207A29FC001A39F900D01
:10851000B29F900D11249C0180911D0190911E012C
:10852000820F931F90931E0180931D0180911B0168
:1085300090911C01860F971F90931C0180931B0143
:108540000091B4071091B5078091990790919A070F
:10855000101611065CF59C0197FF04C022273327F3
:10856000281B390BC901AA2797FDA095BA2F209186
:108570009E01332744275527BC01CD010E948E78E8
:108580009B01AC0197FF04C0215C3F4F4F4F5F4FF1
:1085900076E055954795379527957A95D1F780914F
:1085A000AF079091B007820F931F27C097FF03C0BA
:1085B000909581959F4FAA2797FDA095BA2F20915E
:1085C0009E01332744275527BC01CD010E948E7898
:1085D0009B01AC0197FF04C0215C3F4F4F4F5F4FA1
:1085E00066E055954795379527956A95D1F780911F
:1085F000AF079091B007821B930B9093B0078093C5
:10860000AF07E090BC07F090BD0780919D07909167
:108610009E071E141F045CF59C0197FF04C02227CF
:108620003327281B390BC901AA2797FDA095BA2F1C
:1086300020919E01332744275527BC01CD010E947C
:108640008E789B01AC0197FF04C0215C3F4F4F4FD8
:108650005F4F96E055954795379527959A95D1F7B1
:108660008091A4079091A507820F931F27C097FFC1
:1086700003C0909581959F4FAA2797FDA095BA2F8B
:1086800020919E01332744275527BC01CD010E942C
:108690008E789B01AC0197FF04C0215C3F4F4F4F88
:1086A0005F4F86E055954795379527958A95D1F781
:1086B0008091A4079091A507821B930B9093A50727
:1086C0008093A4078091160687FF44C09989992357
:1086D00009F040C0809107038823E1F5A1E0EA1684
:1086E000A1E0FA064CF08091B1079091B2078E0D8F
:1086F0009F1D805091400DC0B0E0EB16BFEFFB0610
:1087000064F48091B1079091B2078E0D9F1D805047
:108710009F4F9093B2078093B107E1E001301E07AD
:108720004CF08091A2079091A307800F911F805079
:1087300091400CC0FFEF00301F0764F48091A20746
:108740009091A307800F911F80509F4F9093A30794
:108750008093A207A2E2B3E06EE076E057E0FB016F
:108760008191BF01E82FFF27EE0FFF1FEF5CF84F4D
:108770000190F081E02DE259FF4FEF3FF10521F02C
:108780001CF0EFEFF0E004C0F7FF02C0E0E0F0E023
:108790004C91242F3327E217F307B1F0CF01821B4E
:1087A000930B97FD079613E0959587951A95E1F73A
:1087B000242F280F2C93822F9927E817F90714F4F8
:1087C000215001C02F5F2C935150119657FFC7CFF6
:1087D000E2E1CD5E0C94397980911803882301F58C
:1087E0008091ED028C7F8093ED02ABE4B4E0E0ED8C
:1087F000F6E09BE080910402882309F48C938D912C
:10880000818312829150389697FFF4CF80910402B1
:10881000882359F08091040281508093040205C09E
:108820008091ED0281608093ED02109274021092AB
:108830007602809171028E7F8093710285EA809327
:10884000BC00089580911806883F38F0EFEFF0E003
:10885000E81BF109EE5DFC4F80818093B0018091AF
:10886000B001882329F0843618F084E68093B001A3
:1088700080911A06883F38F0EFEFF0E0E81BF1092D
:10888000EE5DFC4F80818093AE018091AE01882324
:1088900029F0843618F084E68093AE018091270693
:1088A000883F38F0EFEFF0E0E81BF109EE5DFC4F98
:1088B00080818093A9018091A9018B3010F48AE016
:1088C00002C08F3F11F48093A90180915206883F26
:1088D00038F0EFEFF0E0E81BF109EE5DFC4F80812E
:1088E0008093C8078091C807823010F481E002C0ED
:1088F0008F3F11F48093C80780915406883F38F069
:10890000EFEFF0E0E81BF109EE5DFC4F8081809312
:10891000EE078091EE07823010F481E002C08F3FB5
:1089200011F48093EE0780913F06883F38F0EFEF17
:10893000F0E0E81BF109EE5DFC4F80818093C507F4
:1089400080914006883F38F0EFEFF0E0E81BF10936
:10895000EE5DFC4F808180939F0780914106883FA8
:1089600038F0EFEFF0E0E81BF109EE5DFC4F80819D
:108970008093CD0790911906983F18F49093AF011A
:1089800009C0EFEFF0E0E91BF109EE5DFC4F8081DB
:108990008093AF01983F18F49093AF0109C0EFEFB7
:1089A000F0E0E91BF109EE5DFC4F80818093AF019F
:1089B00080911C06883F38F0EFEFF0E0E81BF109EA
:1089C000EE5DFC4F80818093AD0180911E06883F53
:1089D00038F0EFEFF0E0E81BF109EE5DFC4F80812D
:1089E0008093AB0180912606883F38F0EFEFF0E0EE
:1089F000E81BF109EE5DFC4F80818093AC01809112
:108A00002806883F38F0EFEFF0E0E81BF109EE5D53
:108A1000FC4F80818093A80180912906883F38F01F
:108A2000EFEFF0E0E81BF109EE5DFC4F80818093F1
:108A3000AA0180912A06883F38F0EFEFF0E0E81BAA
:108A4000F109EE5DFC4F80818093A70180912B0698
:108A5000883F38F0EFEFF0E0E81BF109EE5DFC4FE6
:108A600080818093A60180913106883F38F0EFEF36
:108A7000F0E0E81BF109EE5DFC4F80818093A401DA
:108A800080913206883F38F0EFEFF0E0E81BF10903
:108A9000EE5DFC4F80818093020380913306883F16
:108AA00038F0EFEFF0E0E81BF109EE5DFC4F80815C
:108AB0008093010380913406883F38F0EFEFF0E0B7
:108AC000E81BF109EE5DFC4F8081809300038091EB
:108AD0003506883F38F0EFEFF0E0E81BF109EE5D76
:108AE000FC4F80818093FF0280914D06883F38F0D3
:108AF000EFEFF0E0E81BF109EE5DFC4F8081809321
:108B0000FE0280914E06883F38F0EFEFF0E0E81B60
:108B1000F109EE5DFC4F80818093FD0280914F064C
:108B2000883F38F0EFEFF0E0E81BF109EE5DFC4F15
:108B300080818093FC0280915006883F38F0EFEFEF
:108B4000F0E0E81BF109EE5DFC4F80818093FB02B1
:108B500080913606883F38F0EFEFF0E0E81BF1092E
:108B6000EE5DFC4F80818093A30180913A06883F9F
:108B700038F0EFEFF0E0E81BF109EE5DFC4F80818B
:108B80008093A20180914206883F38F0EFEFF0E039
:108B9000E81BF109EE5DFC4F80818093A10180917B
:108BA0004506883F38F0EFEFF0E0E81BF109EE5D95
:108BB000FC4F80818093A00180914606883F38F069
:108BC000EFEFF0E0E81BF109EE5DFC4F8081809350
:108BD0009F0180914706883F38F0EFEFF0E0E81BF7
:108BE000F109EE5DFC4F808180939E0180914C06DF
:108BF000883F38F0EFEFF0E0E81BF109EE5DFC4F45
:108C0000808180939D0180916706883F38F0EFEF67
:108C1000F0E0E81BF109EE5DFC4F80818093FE07D8
:108C20008091A401282F33272F5F3F4F8CE398E2D8
:108C3000B9010E94CD787093B2016093B101809127
:108C400024068093EF07809123068093B6079091C6
:108C50006906933320F181E08093FA02983F58F03F
:108C6000EFEFF0E0E91BF109EE5DFC4F808182330C
:108C700010F41092FA0280913C0890913D0897FF01
:108C800008C08091FA02882321F080914604806810
:108C900003C0809146048F778093460402C01092EF
:108CA000FA0280913C0890913D0897FF1DC0809189
:108CB00018038823C9F08091FA028823A9F08091D3
:108CC0000801909109018F5F9F4F71F488E99AE341
:108CD000909324028093230280E094EA9093090108
:108CE000809308011092FA028091FA02882339F0E9
:108CF0008091A001823D18F4825E8093A0010895C6
:108D0000A5E3B0E0E6E8F6E40C941D790E94F43B9C
:108D1000309102013C3010F4299A01C02998E0906A
:108D20001903F0901A03F9A2E8A28091B6079927D7
:108D30000A96E816F90614F499A388A380912103F2
:108D4000843608F05CC08091BA039091BB03009711
:108D500031F001979093BB038093BA0307C0109240
:108D600018038091ED028F7E8093ED023A3011F06E
:108D7000343110F0289A01C028988091EE02909129
:108D8000EF02895E9340C0F180912E06282F332791
:108D900039A328A38091ED0280618093ED02809138
:108DA0000A06A82FBB27AA0FBB1FFD01EB59F84FDE
:108DB0001182108280910B06282F3327220F331F38
:108DC000C9018B59984FFC0111821082AF5CB84FDA
:108DD00011961C921E922F5C384FD90111961C924D
:108DE0001E9280910D06E82FFF27EE0FFF1FEF5C0C
:108DF000F84F11821082AAC210921803A7C2809164
:108E000021038D3808F4A2C28091ED028F7E8093F9
:108E1000ED0290912F0682E3989FC0011124909358
:108E2000BB038093BA03E8A1F9A1B9978CF08091B4
:108E30001803882369F08091EE029091EF02FFEF12
:108E40008F3F9F0729F001969093EF028093EE02E7
:108E50008091EE029091EF028F3F910509F038F575
:108E600010923D0310923E0310923F031092400374
:108E70001092390310923A0310923B0310923C0374
:108E80001092A6031092A7031092A8031092A903B0
:108E90001092450310924603109247031092480324
:108EA0008A3F910549F481E08093C00305C0809119
:108EB000ED0282608093ED0280910C06E82FFF277F
:108EC000EE0FFF1FEF5CF84F808191818135910596
:108ED0000CF441C120911803222309F03CC1809178
:108EE0000D06E82FFF27EE0FFF1FEF5CF84F808184
:108EF00091818C3491050CF406C18091BC038F5F85
:108F00008093BC03893C08F426C13C3010F42998B6
:108F100001C0299A109218031092BC031092EF021C
:108F20001092EE0230910A06E32FFF27EE0FFF1F8B
:108F3000EF5CF84F8081918187349105B4F4809182
:108F40000B06E82FFF27EE0FFF1FEF5CF84F808125
:108F500091810190F081E02DF7FF03C0F095E1953C
:108F6000FF4FE734F1050CF478C041E020910B0687
:108F7000A22FBB27AA0FBB1FAF5CB84F8D919C914E
:108F800011978734910544F0E32FFF27EE0FFF1F61
:108F9000EF5CF84F808191818D919C918734910590
:108FA00074F080910A06E82FFF27EE0FFF1FEF5C99
:108FB000F84F80819181873491050CF042E0E22FD7
:108FC000FF27EE0FFF1FEF5CF84F80819181863401
:108FD000910574F480910A06E82FFF27EE0FFF1F1A
:108FE000EF5CF84F80819181873491050CF043E06C
:108FF000E22FFF27EE0FFF1FEF5CF84F808191817A
:109000008A5B9F4F74F480910A06E82FFF27EE0FCA
:10901000FF1FEF5CF84F80819181873491050CF040
:1090200044E0E22FFF27EE0FFF1FEF5CF84F808137
:1090300091818A5B9F4F74F480910A06E82FFF2785
:10904000EE0FFF1FEF5CF84F808191818634910510
:109050000CF445E0842F0E94AF2E80910B06E82F80
:10906000FF27EE0FFF1FEF5CF84F80819181019089
:10907000F081E02DF7FF03C0F095E195FF4F7E975B
:10908000BCF480910A06E82FFF27EE0FFF1FEF5C6C
:10909000F84F808191818A5B9F4F54F481E08093E7
:1090A000610488EE93E0909324028093230253C0DE
:1090B0000E94852F0E94782E80E00E945F07809199
:1090C00030060E941C768091160680FF10C08091A9
:1090D000150190911601875B934038F4809115013A
:1090E000909116018E5E924010F40E94401B1092E7
:1090F000210280E00E94463981E08093BF03809383
:109100002102579A1FC080819181855B9F4F0CF58A
:109110008091BC038F5F8093BC03893CE0F03C30BE
:1091200010F4299801C0299A109218031092BC03D8
:109130001092EF021092EE0281E00E94463981E027
:109140008093BF030E94852F68E770E00E948438F7
:1091500002C02093BC0380910C06E82FFF27EE0F7E
:10916000FF1FEF5CF84F808191818B5A9F4F0CF06D
:10917000EDC020911803E0910D06222309F0CAC02A
:10918000FF27EE0FFF1FEF5CF84F80819181855B19
:109190009F4F0CF0BCC08091BD038F5F8093BD03D7
:1091A000893C08F4D3C02093BD03809146048823F2
:1091B00009F0A6C08091BF03882309F4A1C081E013
:1091C00090E09093EF028093EE0281E08093180389
:1091D0001092A6031092A7031092A8031092A9035D
:1091E00010924503109246031092470310924803D1
:1091F00010924103109242031092430310924403D1
:1092000080912506E82EFF24002711278091EB0787
:109210009091EC079C01442737FD4095542FC801DD
:10922000B7010E948E78DC01CB01809355039093A7
:109230005603A0935703B09358038091FB07909176
:10924000FC079C01442737FD4095542FC801B70106
:109250000E948E78DC01CB0180934D0390934E03E6
:10926000A0934F03B09350038091750390917603C0
:10927000A0917703B09178038093510390935203A8
:10928000A0935303B093540380916D0390916E03A8
:10929000A0916F03B09170038093490390934A03A8
:1092A000A0934B03B0934C0310923D0310923E03E6
:1092B00010923F03109240031092390310923A0328
:1092C00010923B0310923C038091ED0288608093E2
:1092D000ED02909168068FE0989F90011124809193
:1092E000330390913403820F931F68E671E00E946C
:1092F000CD7897FD0196959587958093790326C043
:109300008CED95E090932402809323021FC020935C
:10931000BD031CC0FF27EE0FFF1FEF5CF84F8081DD
:1093200091818C34910584F08091BE038F5F80938E
:10933000BE03893C58F0109218031092BE0310929D
:10934000EF021092EE0202C01092BE0380919501CE
:10935000815080939501809195018F3F21F08091FC
:10936000ED0284FF82C30E9422448091C903909140
:10937000CA039C01220F331F280F391FA0900A0631
:10938000AA2DBB27AA0FBB1FFD01EF5CF84F9090E1
:109390002006492D552780819181849FF001859F6A
:1093A000F00D949FF00D11242E0F3F1F37FF02C0C8
:1093B0002D5F3F4FB9017595679575956795AB59C9
:1093C000B84F80912106082F11278D919C91809F85
:1093D0007001819FF00C909FF00C11246E0D7F1D89
:1093E0007093CA036093C9038091CB039091CC031F
:1093F0009C01220F331F280F391FB0900B06AB2D95
:10940000BB27AA0FBB1FFD01EF5CF84F8081918144
:10941000849FF001859FF00D949FF00D11242E0F75
:109420003F1F37FF02C02D5F3F4FA901559547955C
:1094300055954795AB59B84F8D919C91809F700180
:10944000819FF00C909FF00C11244E0D5F1D5093E6
:10945000CC034093CB039E012F5F3F4F8FE1E2ECA3
:10946000F1E0D90101900D928A95E1F78091FA021D
:10947000882309F448C0CB0177FD0396DC01B5953C
:10948000A795B595A795CA0157FD0396FC01F595DB
:10949000E795F595E7958091EB01682F772767FDB4
:1094A00070956A9F90016B9F300D7A9F300D11244B
:1094B00080910204482F552747FD50954E9FC001CB
:1094C0004F9F900D5E9F900D1124280F391F37FF7D
:1094D00002C0295F3F4F03E0359527950A95E1F7D4
:1094E0003093200320931F036E9F90016F9F300DD8
:1094F0007E9F300D11244A9FC0014B9F900D5A9FB3
:10950000900D112444C080916806082F1127DE01B8
:10951000A00FB11FFD0197819093EB01020F131F64
:10952000D8018C9180930204A92FBB27A7FDB09589
:10953000A69F9001A79F300DB69F300D1124E82FF4
:10954000FF27E7FDF095E49FC001E59F900DF49F94
:10955000900D1124280F391F37FF02C0295F3F4F9C
:1095600013E0359527951A95E1F730932003209362
:109570001F03A49F9001A59F300DB49F300D1124AF
:10958000E69FC001E79F900DF69F900D1124281BC8
:10959000390B37FF02C0295F3F4FF3E03595279520
:1095A000FA95E1F730931E0320931D0380910D0679
:1095B000E82FFF27EE0FFF1FEF5CF84F80819181AE
:1095C000909581959F4F90931C0380931B0383304C
:1095D000910514F0029705C0BFEF8E3F9B0734F44E
:1095E000029690931C0380931B0304C010921C03EB
:1095F00010921B038091FE039091FF032091FA03C8
:109600003091FB03820F931FC0901F03D090200363
:10961000C81AD90AD0922003C0921F038091FC037C
:109620009091FD032091F8033091F903820F931F6D
:1096300000911D0310911E03081B190B10931E03AC
:1096400000931D0380910C06E82FFF27EE0FFF1FEC
:10965000EF5CF84FE080F180E8E7F0E0EE0EFF1EEF
:10966000F0921A03E09219038091A9019927AA2781
:1096700097FDA095BA2FBC01CD010E943678DC0180
:10968000CB0120E030E040E251E4BC01CD010E947A
:10969000D777DC01CB01BC01CD010E941978DC0138
:1096A000CB018093F5078091A8018093CE0780912C
:1096B000A7019927AA2797FDA095BA2FBC01CD0134
:1096C0000E943678DC01CB0120E030E040E251E43A
:1096D000BC01CD010E94D777DC01CB01BC01CD01DB
:1096E0000E941978DC01CB018093A9078091A60123
:1096F0008093BE0780916D0480FF59C08091FE0762
:10970000813808F454C080916604992787FD9095AC
:10971000292D3327829FA001839F500D929F500DCA
:109720001124C40ED51ED0922003C0921F03809135
:109730006704992787FD9095829FB001839F700DE4
:10974000929F700D1124060F171F10931E03009394
:109750001D0380916804282F332727FD30958091C1
:109760001B0390911C03820F931F90931C03809303
:109770001B0380916A04282F332727FD30958091A1
:109780001B069927289FD001299FB00D389FB00D47
:109790001124B0939C01A0939B01809169049927A7
:1097A0008E159F0524F490931A03809319038091DA
:1097B000190390911A0397FF04C010921A03109294
:1097C00019038091160682FF02C01092CE074091C5
:1097D0001F0350912003CA0157FD03969C01359544
:1097E00027953595279537FF03C0309521953F4F35
:1097F0008091F2029091F30282179307B4F4CA01A8
:1098000057FF03C0909581959F4F97FD03969595BF
:109810008795959587959093F3028093F20285360C
:10982000910544F084E690E001C001979093F30223
:109830008093F20240911D0350911E03CA0157FD0F
:1098400003969C01359527953595279537FF03C0DD
:10985000309521953F4F8091F0029091F10282174F
:109860009307B4F4CA0157FF03C0909581959F4FA9
:1098700097FD039695958795959587959093F10219
:109880008093F0028536910544F084E690E001C0B3
:1098900001979093F1028093F0028091ED0284FF92
:1098A00008C01092F3021092F2021092F10210928C
:1098B000F002EB2DFF27EE0FFF1FEF5CF84F4091FA
:1098C0004306242F3327808191812817390744F4D8
:1098D00080916A0682FF04C081E08093060313C072
:1098E000EB2DFF27EE0FFF1FEF5CF84F842F99271A
:1098F00020914406821B9109208131812817390764
:1099000014F41092060340910B06E42FFF27EE0F8C
:10991000FF1FEF5CF84F50914306852F99272227B0
:109920003327281B390B808191818217930744F4D8
:1099300080916A0683FF04C081E08093050316C00E
:1099400080910503882391F0E42FFF27EE0FFF1F7E
:10995000EF5CF84F809144069927851B910920817F
:1099600031818217930714F410920503EA2DFF2723
:10997000EE0FFF1FEF5CF84F40914306242F332773
:10998000808191812817390744F480916A0680FF0D
:1099900004C081E08093030317C0809103038823F0
:1099A00099F0EA2DFF27EE0FFF1FEF5CF84F842F91
:1099B000992720914406821B910920813181281723
:1099C000390714F41092030340910A06E42FFF278D
:1099D000EE0FFF1FEF5CF84F50914306852F99273C
:1099E00022273327281B390B808191818217930707
:1099F00044F480916A0681FF04C081E080930403EF
:109A000016C080910403882391F0E42FFF27EE0F06
:109A1000FF1FEF5CF84F809144069927851B910941
:109A2000208131818217930714F4109204038091EE
:109A30000603882319F480910503811181E0809346
:109A4000070380910303882321F480910403882372
:109A500051F081E0809308031092070310920603EF
:109A60001092050302C080930803809107038823A6
:109A700021F480910803882369F080914206992798
:109A8000E8A1F9A18E179F0714F499A388A381E098
:109A900080932D038091ED0284FF1AC010921C0365
:109AA00010921B031092200310921F0310921E03AA
:109AB00010921D039AE59093F50788E78093CE07EF
:109AC0009093A9078093BE07109207031092080392
:109AD0008091C1079091C207A091C307B091C407BC
:109AE000209175033091760340917703509178036C
:109AF000820F931FA41FB51F8093C1079093C207C5
:109B0000A093C307B093C4078091C9079091CA0777
:109B1000A091CB07B091CC0720906D0330906E03DD
:109B200040906F0350907003820D931DA41DB51DCE
:109B30008093C9079093CA07A093CB07B093CC0733
:109B40008091B8079091B907A091BA07B091BB076F
:109B5000E0907103F090720300917303109174030D
:109B6000EAA2FBA20CA31DA38E0D9F1DA01FB11F77
:109B70008093B8079093B907A093BA07B093BB0737
:109B80008091AA079091AB07A091AC07B091AD0767
:109B9000E0906903F0906A0300916B0310916C03ED
:109BA000EEA2FFA208A719A78E0D9F1DA01FB11F2F
:109BB0008093AA079093AB07A093AC07B093AD072F
:109BC000F0900803FAA6FF2029F480910703882368
:109BD00009F460C010926503109266031092670347
:109BE0001092680310926103109262031092630353
:109BF000109264031092C1071092C2071092C3071B
:109C00001092C4071092C9071092CA071092CB078E
:109C10001092CC071092B8071092B9071092BA07A9
:109C20001092BB071092AA071092AB071092AC07D4
:109C30001092AD078091550390915603A091570360
:109C4000B09158038093510390935203A093530310
:109C5000B093540380914D0390914E03A0914F0314
:109C6000B09150038093490390934A03A0934B0310
:109C7000B0934C03109239021092380210920C03E8
:109C800010920B0310920E0310920D030AA50023ED
:109C900009F0F2C180910703882309F0EDC180919A
:109CA000FB059091FC05815092402CF480911803A3
:109CB000882309F4E1C190906908A090250660917D
:109CC000EB077091EC077BAB6AAB8091FB0790913F
:109CD000FC079DAB8CAB9FEF991609F4D9C0BB2450
:109CE000CC24DD24CA01B901A60195010E940279A4
:109CF00079018A01EAA9FBA9CF01AA2797FDA095BE
:109D0000BA2FE81AF90A0A0B1B0BC201B101A6010E
:109D100095010E94027959016A012CA93DA9C90146
:109D2000AA2797FDA095BA2FA81AB90ACA0ADB0A72
:109D3000292C332427FC3094432C532CC801B70121
:109D4000A20191010E948E7897FF04C061507E4F5E
:109D50008F4F9F4F3B014C0109E095948794779476
:109D600067940A95D1F7C601B501A20191010E943D
:109D70008E7897FF04C061507E4F8F4F9F4F5B01DD
:109D80006C0119E0D594C794B794A7941A95D1F7AC
:109D90008091F2029091F302813491053CF480911C
:109DA000F0029091F10281349105D4F0D401C30105
:109DB00097FE03C00196A11DB11D3C014D01959474
:109DC000879477946794D601C501D7FE03C00196A6
:109DD000A11DB11D5C016D01D594C794B794A794E2
:109DE00080910D06E82FFF27EE0FFF1FEF5CF84F65
:109DF000808191810190F081E02DF7FF03C0F09503
:109E0000E195FF4F7A97A4F0C401B30123E030E05D
:109E100040E050E00E94027939014A01C601B501D3
:109E200023E030E040E050E00E94027959016A01ED
:109E300080916B08282F332727FD3095432F532F10
:109E4000261537054805590514F439014A019927A3
:109E500087FD9095909581959F4FAA2797FDA09596
:109E6000BA2F681679068A069B0614F43C014D0148
:109E70002A153B054C055D0514F459016A01A81625
:109E8000B906CA06DB060CF0CFC05C016D01CCC080
:109E9000EA2CFF2400271127CA01B901A801970164
:109EA0000E94027939014A014AA95BA9CA01AA277D
:109EB00097FDA095BA2F681A790A8A0A9B0AC201EF
:109EC000B101A80197010E94027959016A016CA9A8
:109ED0007DA9CB01AA2797FDA095BA2FA81AB90A88
:109EE000CA0ADB0AD401C30197FE03C00F96A11D65
:109EF000B11D3C014D01F4E09594879477946794EB
:109F0000FA95D1F7D601C501D7FE03C00F96A11D62
:109F1000B11D5C016D01E4E0D594C794B794A7949A
:109F2000EA95D1F78091F2029091F3028134910584
:109F30003CF48091F0029091F10281349105A4F0FB
:109F4000C401B30123E030E040E050E00E94027918
:109F500039014A01C601B50123E030E040E050E09C
:109F60000E94027959016A0180910D06E82FFF27AE
:109F7000EE0FFF1FEF5CF84F808191810190F0811F
:109F8000E02DF7FF03C0F095E195FF4F7A97A4F01D
:109F9000C401B30123E030E040E050E00E940279C8
:109FA00039014A01C601B50123E030E040E050E04C
:109FB0000E94027959016A0171E2671671048104F5
:109FC00091042CF070E2672E712C812C912C80EE84
:109FD00068168FEF78068FEF88068FEF980644F4A7
:109FE00060EE662E6FEF762E6FEF862E6FEF962E59
:109FF00091E2A916B104C104D1042CF050E2A52EBF
:10A00000B12CC12CD12CA0EEAA16AFEFBA06AFEF3F
:10A01000CA06AFEFDA0644F440EEA42E4FEFB42E9A
:10A020004FEFC42E4FEFD42E8091550390915603DD
:10A03000A0915703B091580386199709A809B90947
:10A040008093550390935603A0935703B0935803FE
:10A0500080914D0390914E03A0914F03B091500316
:10A060008A199B09AC09BD0980934D0390934E0357
:10A07000A0934F03B093500380913802909139021E
:10A080008F3F910509F008F4C4C5BAA5BB2309F0B8
:10A090004EC580910703882309F049C580912D039F
:10A0A000882309F044C5E0914B06EBA7EE2309F4A1
:10A0B0003EC58091C1079091C207A091C307B0919E
:10A0C000C407B7FF04C081509F4FAF4FBF4FE92E69
:10A0D000FA2E0B2F112707FD1A95E092C107F09277
:10A0E000C2070093C3071093C4078091C9079091DA
:10A0F000CA07A091CB07B091CC07B7FF04C081502D
:10A100009F4FAF4FBF4F892F9A2FAB2FBB27A7FD74
:10A11000BA958CA79DA7AEA7BFA78093C9079093B8
:10A12000CA07A093CB07B093CC0780912506A82E31
:10A13000BB24CC24DD24209165033091660340913B
:10A14000670350916803C601B5010E948E7897FF9E
:10A1500004C061507F4F8F4F9F4F672E782E892EFE
:10A16000992487FC9A9460926503709266038092AA
:10A1700067039092680320916103309162034091DC
:10A18000630350916403C601B5010E948E7897FF66
:10A1900004C061507F4F8F4F9F4F272E382E492E7E
:10A1A000552447FC5A9420926103309262034092F6
:10A1B00063035092640380915D0390915E03A091CC
:10A1C0005F03B0916003B7FF04C081509F4FAF4F52
:10A1D000BF4F892F9A2FAB2FBB27A7FDBA9580932E
:10A1E0005D0390935E03A0935F03B0936003D80177
:10A1F000C70186199709A809B9098093B2039093FA
:10A20000B303A093B403B093B50320914A06E22EA2
:10A21000FF2400271127BC01CD01A80197010E944E
:10A22000027959016A012093C1033093C20340931C
:10A23000C3035093C4038CA59DA5AEA5BFA58219E9
:10A240009309A409B5098093B6039093B703A0932B
:10A25000B803B093B903BC01CD01A80197010E94D6
:10A2600002792093C5033093C6034093C7035093EC
:10A27000C803D601C501D7FE04C081509F4FAF4F20
:10A28000BF4F892F9A2FAB2FBB27A7FDBA9590936D
:10A290000C0380930B0357FF04C021503F4F4F4FD7
:10A2A0005F4FBB2757FDBA95A52F942F832F90930F
:10A2B0000E0380930D038091F2029091F30281349A
:10A2C0009105DCF48091F0029091F10281349105C6
:10A2D000A4F480910D06E82FFF27EE0FFF1FEF5C1F
:10A2E000F84F808191810190F081E02DF7FF03C04C
:10A2F000F095E195FF4F7A97E4F0809169088F3FE0
:10A30000C1F480910B0390910C0397FD01969595F4
:10A31000879590930C0380930B0380910D0390918C
:10A320000E0397FD01969595879590930E03809364
:10A330000D038091B8079091B907A091BA07B09129
:10A34000BB07B7FF04C081509F4FAF4FBF4F892F4E
:10A350009A2FAB2FBB27A7FDBA958093B807909390
:10A36000B907A093BA07B093BB078091AA07909151
:10A37000AB07A091AC07B091AD07B7FF04C0815007
:10A380009F4FAF4FBF4F892F9A2FAB2FBB27A7FDF2
:10A39000BA958093AA079093AB07A093AC07B093AC
:10A3A000AD078091750390917603A0917703B091EA
:10A3B00078032AA13BA14CA15DA1281B390B4A0BB4
:10A3C0005B0B2093AA033093AB034093AC035093F1
:10A3D000AD0380916D0390916E03A0916F03B091D6
:10A3E0007003EEA0FFA008A519A5E81AF90A0A0B48
:10A3F0001B0BE092AE03F092AF030093B0031093F7
:10A40000B1032093B2033093B3034093B40350934A
:10A41000B503E092B603F092B7030093B80310932C
:10A42000B9038091510390915203A0915303B091CD
:10A430005403821B930BA40BB50B80935103909391
:10A440005203A0935303B093540380914903909116
:10A450004A03A0914B03B0914C038E199F09A00BA6
:10A46000B10B8093490390934A03A0934B03B0939D
:10A470004C03FBA5FF23E1F020912B0330912C032B
:10A48000213831054CF08091860390918703019625
:10A49000909387038093860320583F4F4CF480911C
:10A4A0008603909187030197909387038093860397
:10A4B00010922C0310922B0381E090E09093CE0336
:10A4C0008093CD03A090B203B090B303C090B403C7
:10A4D000D090B503D601C501D7FE07C088279927BC
:10A4E000DC018A199B09AC09BD0981509240A0404A
:10A4F000B04034F084E090E09093CE038093CD039D
:10A500008091D3039091D403A091D503B091D60349
:10A510002091C1073091C2074091C3075091C407F1
:10A52000821B930BA40BB50B815E914BAF4FBF4FBA
:10A530008F539C49A040B04028F080916A0889312F
:10A540000CF4FFC031E0A31630E1B30630E0C306DF
:10A5500030E0D3060CF473C08091CF03882309F454
:10A560006AC0D601C501D7FE07C088279927DC013C
:10A570008A199B09AC09BD099C01AD01B7FF04C054
:10A5800021503E4F4F4F5F4FF9E055954795379516
:10A590002795FA95D1F78091CD039091CE03820F44
:10A5A000931F9093CE038093CD03D601C501D7FEB0
:10A5B00003C00796A11DB11DE3E0B595A79597953A
:10A5C0008795EA95D1F78093C1039093C203A09336
:10A5D000C303B093C40389589341A040B04064F0D2
:10A5E00088E893E1A0E0B0E08093C1039093C203B8
:10A5F000A093C303B093C4032091C1033091C2035D
:10A600004091C3035091C40357FF04C021503F4FF2
:10A610004F4F5F4F232F342F452F552747FD5A9516
:10A6200080910B0390910C03820F931F90930C0366
:10A6300080930B0306C081E08093CF0302C0109289
:10A64000CF0350E0A51650EFB5065FEFC5065FEFEC
:10A65000D5060CF073C08091D003882309F46AC03A
:10A66000D601C501D7FE07C088279927DC018A19C2
:10A670009B09AC09BD099C01AD01B7FF04C0215085
:10A680003E4F4F4F5F4F69E055954795379527955A
:10A690006A95D1F78091CD039091CE03820F931FDD
:10A6A0009093CE038093CD03D601C501D7FE03C09E
:10A6B0000796A11DB11D23E0B595A79597958795A0
:10A6C0002A95D1F78093C1039093C203A093C3034B
:10A6D000B093C40388579C4EAF4FBF4F64F488E7D4
:10A6E0009CEEAFEFBFEF8093C1039093C203A093A2
:10A6F000C303B093C4032091C1033091C2034091BE
:10A70000C3035091C40357FF04C021503F4F4F4F24
:10A710005F4F232F342F452F552747FD5A958091A2
:10A720000B0390910C03820F931F90930C03809363
:10A730000B0311C081E08093D0030DC01092D003B1
:10A740000AC01092CE031092CD0388EE93E090934E
:10A75000BC018093BB017BA5272F33278091CD03BC
:10A760009091CE032817390724F43093CE03209319
:10A77000CD03E0916A08EE2379F02E2F332727FDD1
:10A7800030958091CD039091CE032817390724F49A
:10A790003093CE032093CD034091B2035091B30385
:10A7A0006091B4037091B50341385105610571059D
:10A7B00074F080918A0390918B032091CD033091A6
:10A7C000CE03820F931F90938B0380938A0340588C
:10A7D0005F4F6F4F7F4F74F480918A0390918B038A
:10A7E0002091CD033091CE03821B930B90938B036A
:10A7F00080938A0381E090E09093CE038093CD0311
:10A80000A090B603B090B703C090B803D090B9033E
:10A81000D601C501D7FE07C088279927DC018A1910
:10A820009B09AC09BD0981509240A040B04034F072
:10A8300084E090E09093CE038093CD038091D70382
:10A840009091D803A091D903B091DA032091C90760
:10A850003091CA074091CB075091CC07821B930BD4
:10A86000A40BB50B815E914BAF4FBF4F8F539C49EB
:10A87000A040B04018F0E9310CF4FFC011E0A1167F
:10A8800010E1B10610E0C10610E0D1060CF473C06F
:10A890008091D103882309F46AC0D601C501D7FE8F
:10A8A00007C088279927DC018A199B09AC09BD09D3
:10A8B0009C01AD01B7FF04C021503E4F4F4F5F4F89
:10A8C00009E055954795379527950A95D1F78091D9
:10A8D000CD039091CE03820F931F9093CE0380936C
:10A8E000CD03D601C501D7FE03C00796A11DB11D3A
:10A8F00013E0B595A795979587951A95D1F780930D
:10A90000C5039093C603A093C703B093C8038958A7
:10A910009341A040B04064F088E893E1A0E0B0E04B
:10A920008093C5039093C603A093C703B093C80355
:10A930002091C5033091C6034091C7035091C803CD
:10A9400057FF04C021503F4F4F4F5F4F232F342FED
:10A95000452F552747FD5A9580910D0390910E0381
:10A96000820F931F90930E0380930D0306C081E026
:10A970008093D10302C01092D10330E0A31630EFD0
:10A98000B3063FEFC3063FEFD3060CF073C08091D0
:10A99000D203882309F46AC0D601C501D7FE07C0D7
:10A9A00088279927DC018A199B09AC09BD099C01FC
:10A9B000AD01B7FF04C021503E4F4F4F5F4FE9E05C
:10A9C0005595479537952795EA95D1F78091CD0311
:10A9D0009091CE03820F931F9093CE038093CD036B
:10A9E000D601C501D7FE03C00796A11DB11D73E0B6
:10A9F000B595A795979587957A95D1F78093C503D7
:10AA00009093C603A093C703B093C80388579C4E86
:10AA1000AF4FBF4F64F488E79CEEAFEFBFEF80937A
:10AA2000C5039093C603A093C703B093C8032091B6
:10AA3000C5033091C6034091C7035091C80357FF27
:10AA400004C021503F4F4F4F5F4F232F342F452FCE
:10AA5000552747FD5A9580910D0390910E03820F63
:10AA6000931F90930E0380930D0311C081E0809398
:10AA7000D2030DC01092D2030AC01092CE031092DE
:10AA8000CD0388EE93E09093BC018093BB015BA55E
:10AA9000252F33278091CD039091CE0328173907B6
:10AAA00024F43093CE032093CD0380916A08882349
:10AAB00079F0282F332727FD30958091CD03909191
:10AAC000CE032817390724F43093CE032093CD0307
:10AAD0004091B6035091B7036091B8037091B903E8
:10AAE000413851056105710574F08091880390919A
:10AAF00089032091CD033091CE03820F931F909351
:10AB000089038093880340585F4F6F4F7F4FCCF489
:10AB100080918803909189032091CD033091CE03D9
:10AB2000821B930B90938903809388030AC0109231
:10AB30000E0310920D0310920C0310920B0310924F
:10AB40002D038091CE07882341F410920E031092BA
:10AB50000D0310920C0310920B038091C10790918A
:10AB6000C207A091C307B091C4078093D303909309
:10AB7000D403A093D503B093D6038091C9079091D5
:10AB8000CA07A091CB07B091CC078093D7039093CD
:10AB9000D803A093D903B093DA03109265031092FF
:10ABA000660310926703109268031092610310927B
:10ABB0006203109263031092640310925D0310927B
:10ABC0005E0310925F03109260031092C10710920F
:10ABD000C2071092C3071092C4071092C9071092BF
:10ABE000CA071092CB071092CC071092B8071092A8
:10ABF000B9071092BA071092BB071092AA071092D9
:10AC0000AB071092AC071092AD0710923902109268
:10AC1000380200911B0310911C03C80117FF04C0E8
:10AC200088279927801B910B40976CF088EE93E062
:10AC30009093BC018093BB018091160684FD03C0F4
:10AC400081E08093C003F0902206AF2CBB24CC247B
:10AC5000DD24B801882777FD8095982F980117FF8C
:10AC600004C022273327201B310B442737FD409592
:10AC7000542F0E948E789B01AC01C601B5010E9441
:10AC80008E7897FF04C061507E4F8F4F9F4F59E0E1
:10AC900095958795779567955A95D1F79B018F2D57
:10ACA0009927809FD001819FB00D909FB00D1124F6
:10ACB000CD01B7FD03969595879595958795280FB6
:10ACC000391F442737FD4095542F2093A603309316
:10ACD000A7034093A8035093A90380914503909143
:10ACE0004603A0914703B0914803821B930BA40B2A
:10ACF000B50B8093450390934603A0934703B0930D
:10AD000048038155934CA040B04064F080E593EC3B
:10AD1000A0E0B0E08093450390934603A0934703DF
:10AD2000B09348038091450390914603A091470357
:10AD3000B0914803805B9C43AF4FBF4F64F480EBFE
:10AD40009CE3AFEFBFEF8093450390934603A0933E
:10AD50004703B0934803A0903303B0903403A11489
:10AD6000B10409F478C18091160683FF74C1809103
:10AD7000750390917603A0917703B0917803B7FFA4
:10AD800004C081509E4FAF4FBF4F29E0B595A795A6
:10AD9000979587952A95D1F76C0197FF04C0D094B9
:10ADA000C194D108D39480916D0390916E03A091CA
:10ADB0006F03B0917003B7FF04C081509E4FAF4F37
:10ADC000BF4F09E0B595A795979587950A95D1F757
:10ADD000BC0197FF03C0709561957F4FC616D706DB
:10ADE0000CF46B01B601D7FE02C0695F7F4F2B01E7
:10ADF00013E0559447941A95E1F7B2E0EB2EF12C4D
:10AE00004E0C5F1C0CE112E0A00EB11E7501002774
:10AE1000F7FC0095102F24EE3DEFA20EB31E80919B
:10AE2000F7079091F807A091F907B091FA076090A1
:10AE30009701709098018090990190909A01BC01BF
:10AE4000CD01A40193010E940279E21AF30A040BD6
:10AE5000150BC801B70128E631E040E050E00E9440
:10AE60000279DC01CB01ACE4EA2EAFEFFA2EE80E5A
:10AE7000F91E0091BB011091BC010115110589F566
:10AE800039E1C316D1046CF580912B0390912C030A
:10AE90008E0D9F1D90932C0380932B038091C003F4
:10AEA0008823F9F0C501AA2797FDA095BA2FBC0108
:10AEB000CD01A40193010E948E78DC01CB01809327
:10AEC000F7079093F807A093F907B093FA07BC012E
:10AED000CD010E9402793093320320933103109206
:10AEE000C003C701F4E0880F991FFA95E1F7B2019A
:10AEF0000E94CD78CB01AA2797FDA095BA2F20916B
:10AF0000F7073091F8074091F9075091FA07280F99
:10AF1000391F4A1F5B1F2093F7073093F8074093B0
:10AF2000F9075093FA07F090AC016F2D7727C69E72
:10AF3000C001C79E900DD69E900D112497FD4F968F
:10AF40006C01E5E0D594C794EA95E1F76C197D09A9
:10AF50006B0177FD7AC00115110509F06FC00091F2
:10AF6000F2021091F3028091F0029091F102080F29
:10AF7000191F17FF02C0095F1F4F73E01595079552
:10AF80007A95E1F7005C1F4FCA01B901A401930152
:10AF90000E940279DA01C901209131033091320314
:10AFA000442737FD4095542F821B930BA40BB50B00
:10AFB000845E9D4FAF4FBF4FBC01CD0128E631E00D
:10AFC00040E050E00E940279DC01CB01845B9040BC
:10AFD0008C9DA0018D9D500D9C9D500D1124CA018A
:10AFE000B8010E94CD7883E0F89E60011124C61656
:10AFF000D70614F4B60108C0882799278C199D0933
:10B00000681779070CF4BC019B01442737FD409574
:10B01000542F8091450390914603A0914703B0912E
:10B020004803820F931FA41FB51F8093450390937D
:10B030004603A0934703B09348030DC0015010404E
:10B040001093BC010093BB0106C084EF91E0909384
:10B05000BC018093BB0180912D03882381F0109265
:10B06000390310923A0310923B0310923C03109262
:10B070003D0310923E0310923F03109240037090E4
:10B0800008037720F1F48091CE07282F3327442737
:10B0900055278091750390917603A0917703B09125
:10B0A0007803BC01CD010E948E78DC01CB01BC018C
:10B0B000CD0128EF3AE240E050E00E9402792901F8
:10B0C00002C044245524909007039920F1F4809104
:10B0D000CE07282F33274427552780916D03909161
:10B0E0006E03A0916F03B0917003BC01CD010E946B
:10B0F0008E78DC01CB01BC01CD0128EF3AE240E0C3
:10B1000050E00E940279190102C022243324809168
:10B11000A4079091A507893C91051CF088EC90E06C
:10B1200005C088539F4F34F488E39FEF9093A507A1
:10B130008093A4078091AF079091B007893C910557
:10B140001CF088EC90E005C088539F4F34F488E3EE
:10B150009FEF9093B0078093AF078091B1079091D4
:10B16000B207AA2797FDA095BA2F2091F507A22E26
:10B17000BB24CC24DD24BC01CD01A60195010E9495
:10B180008E789B01AC018091A4079091A507AA2716
:10B1900097FDA095BA2F67E0880F991FAA1FBB1FC4
:10B1A0006A95D1F7280F391F4A1F5B1F57FF04C04C
:10B1B000215C3F4F4F4F5F4F06E0559547953795C0
:10B1C00027950A95D1F77201E20EF31EF092B207AD
:10B1D000E092B1078091A2079091A307AA2797FD5B
:10B1E000A095BA2FBC01CD01A60195010E948E78D1
:10B1F0009B01AC018091AF079091B007AA2797FD02
:10B20000A095BA2F17E0880F991FAA1FBB1F1A9588
:10B21000D1F7280F391F4A1F5B1F57FF04C0215C5D
:10B220003F4F4F4F5F4FB6E0559547953795279560
:10B23000BA95D1F78101020F131F1093A307009352
:10B24000A2078091F0079091F107880F991FAA2714
:10B2500097FDA095BA2F2091A9073327442755279A
:10B26000BC01CD010E948E785B016C0197FF08C084
:10B270008FE390E0A0E0B0E0A80EB91ECA1EDB1E6E
:10B28000A6E0D594C794B794A794AA95D1F78091D6
:10B29000BE07282F332744275527809159039091C3
:10B2A0005A03A0915B03B0915C03BC01CD010E94E5
:10B2B0008E78DC01CB01BC01CD0120EF35E540E00B
:10B2C00050E00E940279B501620F731F7093F1077D
:10B2D0006093F00791E0E91690E1F90634F080E020
:10B2E00090E19093B2078093B1078091B10790915C
:10B2F000B2078050904F34F480E090EF9093B20703
:10B300008093B1070150104134F080E090E19093B8
:10B31000A3078093A2078091A2079091A307805072
:10B32000904F34F480E090EF9093A3078093A207AE
:10B330006150704134F080E090E19093F107809388
:10B34000F0078091F0079091F1078050904F34F40E
:10B3500080E090EF9093F1078093F00780910001D7
:10B36000482F552780911F019091200148175907B8
:10B3700094F420911F013091200168A179A1649F6C
:10B38000C001659F900D749F900D1124B9010E941A
:10B39000B97879A368A388A199A1880F991F880F0C
:10B3A000991F99A388A34091160640FFA7C699202C
:10B3B00009F0A4C6772009F0A1C6CC24DD244601FB
:10B3C0008091090390910A039093DF058093DE0535
:10B3D00020918C0330918D032115310509F03FC078
:10B3E00080911501909116018959934058F087B5C5
:10B3F000853F20F480913C02815011C081E0809310
:10B40000E6034EC080911501909116018436910596
:10B4100008F587B58B30D0F080913C028F5F809328
:10B420003C029AE089029001112480910506821B5A
:10B4300087BD8CE291E090932402809323028EE5F5
:10B4400091E090938D0380938C032AC081E08093D8
:10B45000E50326C07092E5037092E60321C0809157
:10B46000130390911403A0911503B0911603E4E027
:10B47000880F991FAA1FBB1FEA95D1F780933D0241
:10B4800090933E02A0933F02B0934002D0923B02C1
:10B49000C0923A022150304030938D0320938C03A8
:10B4A0002091AF0141FF24C02233D8F48091C10123
:10B4B00081508093C1018F3FD9F510922E03809166
:10B4C000130390911403A0911503B0911603809378
:10B4D0000F0390931003A0931103B093120381E024
:10B4E00004C081E080932E0388EC8093C10120C0CA
:10B4F00080919B0190919C01820F911D20911B06D0
:10B500003327829FF001839FF00D929FF00D11244D
:10B51000CF01AA2797FDA095BA2F80930F03909390
:10B520001003A0931103B093120381E080932E03C4
:10B530008091750390917603A0917703B091780381
:10B54000E0909701F09098010091990110919A0173
:10B55000BC01CD01A80197010E94027959016A013D
:10B5600080916D0390916E03A0916F03B091700371
:10B57000BC01CD01A80197010E940279B901C50162
:10B580000E94D46F3C01CC971CF07CE3672E712C99
:10B59000C3010E94CF6B3C0180E2809396018091B1
:10B5A0002E03882309F436C48091ED0299279C016B
:10B5B0002071307084FD2EC460916C0660FD04C063
:10B5C0008091160681FD07C008A119A13093DC0304
:10B5D0002093DB0397C18091ED0281FF69C1409107
:10B5E000BD015091BE01CA010F96209119033091FF
:10B5F0001A0382179307ACF58091E503882389F538
:10B600008091E70381FF13C08D7F8093E7038091D2
:10B61000130390911403A0911503B0911603809326
:10B620000F0390931003A0931103B0931203809122
:10B63000E70381608093E703241B350B2F503040D4
:10B6400037FF03C0309521953F4F8091DB039091E8
:10B65000DC03820F931F9093DC038093DB038BE268
:10B660006EC0CA010F9728173907ACF58091E60321
:10B67000882389F58091E70380FF13C08E7F809334
:10B68000E7038091130390911403A0911503B091E7
:10B69000160380930F0390931003A0931103B093AC
:10B6A00012038091E70382608093E703241B350B2C
:10B6B000215F3F4F37FF03C0309521953F4F809169
:10B6C000DB039091DC03821B930B9093DC0380934C
:10B6D000DB038DE234C02091E703822F992783702A
:10B6E0009070892B59F12C7F2093E7031092DC0393
:10B6F0001092DB0320911303309114034091150342
:10B700005091160320930F033093100340931103BD
:10B710005093120361FF06C084EF91E090932402DE
:10B720008093230280911703882341F4233331054A
:10B73000410551051CF081E0809317038DE3809350
:10B7400096012091DB033091DC03C90137FF04C06F
:10B7500088279927821B930B815092400CF491C04B
:10B7600080911B069927289FA001299F500D389F83
:10B77000500D1124CA0160E075E00E94CD78CB0124
:10B78000AA2797FDA095BA2F20910F03309110039F
:10B790004091110350911203280F391F4A1F5B1F5C
:10B7A00020930F033093100340931103509312031F
:10B7B0001092DC031092DB03A0901303B0901403EB
:10B7C000C0901503D0901603D601C5018050944057
:10B7D000A040B04082179307A407B5075CF4D601D8
:10B7E000C50180509C4FAF4FBF4F281739074A07FC
:10B7F0005B0744F080930F0390931003A093110311
:10B80000B093120380916C0681FF06C084E690E03D
:10B81000909324028093230280911F06882389F548
:10B820004091090350910A0357FF02C04D5F5F4FDB
:10B83000559547955595479580911F019091200109
:10B84000209100013327489FB001499F700D589FF8
:10B85000700D1124CB01B9010E94CD787093BE0107
:10B860006093BD01663471051CF486E490E005C068
:10B870006739710534F086E990E09093BE018093BA
:10B88000BD0180918C0390918D03892BB9F180913A
:10B89000130390911403A0911503B09116038093A4
:10B8A0000F0390931003A0931103B093120326C0CB
:10B8B0008091130390911403A0911503B091160386
:10B8C00080599140A040B04080930F0390931003A3
:10B8D000A0931103B093120380911F06882311F0E7
:10B8E000992702C088E790E09093BE018093BD0144
:10B8F00088A199A190930A038093090300910903F9
:10B9000010910A03A0901303B0901403C090150384
:10B91000D090160320910F03309110034091110332
:10B92000509112032A153B054C055D0524F08091CA
:10B930006C0680FDB1C280918C0390918D03892BA0
:10B9400039F00091090310910A03CC24DD24D7C0FB
:10B95000D601C501821B930BA40BB50B8093AA03E0
:10B960009093AB03A093AC03B093AD038230E0E8B7
:10B970009E07EFEFAE07EFEFBE072CF481E090E8F3
:10B98000AFEFBFEF09C08F5F9F47A040B04064F0AA
:10B990008FEF9FE7A0E0B0E08093AA039093AB0302
:10B9A000A093AC03B093AD03C090AA03D090AB03B7
:10B9B0008091AE01282F3327442755278091AA0371
:10B9C0009091AB03A091AC03B091AD03BC01CD014C
:10B9D0000E948E7897FF04C0615E7F4F8F4F9F4F0C
:10B9E00055E095958795779567955A95D1F760932A
:10B9F000AA037093AB038093AC039093AD036530BF
:10BA00002EEF72072FEF82072FEF92072CF484E0BE
:10BA10009EEFAFEFBFEF09C0605074408040904090
:10BA200064F080E094E0A0E0B0E08093AA039093FB
:10BA3000AB03A093AC03B093AD038090AA039090A6
:10BA4000AB0320913A0230913B0237FF02C0295FDD
:10BA50003F4F43E0359527954A95E1F74FEF223860
:10BA600034071CF421E83FEF05C02038310514F0FD
:10BA700020E830E0C901AA2797FDA095BA2F2091B0
:10BA8000B001332744275527BC01CD010E948E7891
:10BA900097FF04C06D5F7F4F8F4F9F4F22E09595BA
:10BAA0008795779567952A95D1F79B015FEF613070
:10BAB00075071CF420E03FEF06C06F3F710519F0D9
:10BAC00014F020E031E08091E703882349F0C901B8
:10BAD00037FD03969C0135952795359527950DC023
:10BAE00080916C0680FF09C0C90137FD07969C0153
:10BAF000A3E035952795AA95E1F7820E931E209134
:10BB0000AD01222309F454C06091350370913603CE
:10BB1000809137039091380397FF04C061587F4F9D
:10BB20008F4F9F4FF7E09595879577956795FA9595
:10BB3000D1F73327442755270E948E7897FF04C0FA
:10BB4000615E7F4F8F4F9F4FE5E095958795779585
:10BB50006795EA95D1F76093AA037093AB0380933E
:10BB6000AC039093AD036138AFEF7A07AFEF8A076C
:10BB7000AFEF9A072CF480E89FEFAFEFBFEF0AC05A
:10BB80006F3F71058105910569F064F080E091E0F7
:10BB9000A0E0B0E08093AA039093AB03A093AC0322
:10BBA000B093AD038091AA039091AB03880E991EC8
:10BBB0008091AB01282F332780916D08992787FD4D
:10BBC0009095289FF001299FF00D389FF00D1124CA
:10BBD0009F01F7FF02C021583F4F220F232F221F42
:10BBE000330BFFEF21383F071CF420E83FEF06C07E
:10BBF0002F3F310519F014F020E031E0820E931E42
:10BC0000C401AA2797FDA095BA2FE0900903F090F0
:10BC10000A039701442737FD4095542FBC01CD01FD
:10BC20000E948E7897FF04C061507E4F8F4F9F4FC8
:10BC300059E095958795779567955A95D1F7061BA5
:10BC4000170B8091DB039091DC03892B09F060C016
:10BC50001E141F040CF05CC09601D7FE03C0309583
:10BC600021953F4F2D33310540F48091DF039091B2
:10BC7000E0038017910774F526C02C53304045E04F
:10BC8000369527954A95E1F72031310510F02FE0E0
:10BC900030E04091DF035091E0031C141D04E4F4F4
:10BCA00080E190E0821B930B489F9001499F300DEB
:10BCB000589F300D112494E0369527959A95E1F719
:10BCC0002017310720F58091BF019091C00108171E
:10BCD0001907F4F08C011CC0205F3F4F8091BF0119
:10BCE0009091C001829FB001839F700D929F700D53
:10BCF00011249B0184E0369527958A95E1F740173A
:10BD0000510714F08A0104C00217130708F08901D3
:10BD1000C801AA2797FDA095BA2F1DE0880F991F8B
:10BD2000AA1FBB1F1A95D1F79301442737FD4095F1
:10BD3000542FBC01CD010E9402792093AE033093B1
:10BD4000AF034093B0035093B1030091AE03109141
:10BD5000AF038091DD039091DE039C01220F331F1E
:10BD6000280F391F200F311F37FF02C02D5F3F4FB3
:10BD7000A90155954795559547955093DE034093F6
:10BD8000DD0380911706282F3327220F331F220F40
:10BD9000331F241735076CF48091EF07282F3327C2
:10BDA000220F331F220F331F2055304042175307F5
:10BDB00024F03093DE032093DD0380916C0680FF36
:10BDC00014C08091DD039091DE03A8A1B9A18A1768
:10BDD0009B0724F0B093DE03A093DD03E091DD0325
:10BDE000F091DE03F9A3E8A357C028A139A12E19C9
:10BDF0003F0937FF02C02D5F3F4F35952795359599
:10BE00002795E090DD03F090DE03E20EF31EF9A229
:10BE1000E8A242C080911F06882301F560910903C2
:10BE200070910A0377FF02C06D5F7F4F759567952C
:10BE30007595679540911F015091200180910001F7
:10BE4000282F3327649FC001659F900D749F900D2C
:10BE50001124B9010E94CD78CB0101C0992790939C
:10BE6000BE018093BD018091BD019091BE018734D8
:10BE700091051CF486E490E005C08639910534F004
:10BE800086E990E09093BE018093BD0108A119A1BD
:10BE90001093DE030093DD038091ED0299279C014E
:10BEA0002270307081FF1CC18091E1039091E20308
:10BEB000A091E303B091E4030097A105B10521F03F
:10BEC000809117038130B1F428A139A1C901AA27B3
:10BED00097FDA095BA2F2EE0880F991FAA1FBB1FB0
:10BEE0002A95D1F78093E1039093E203A093E303B3
:10BEF000B093E40380911703813019F482E08093BA
:10BF0000170348A159A1CA01AA2797FDA095BA2FE6
:10BF10009301442737FD4095542FBC01CD010E9469
:10BF20008E78DC01CB018093AE039093AF03A09396
:10BF3000B003B093B103B7FF04C08150904EAF4F30
:10BF4000BF4F5C016D018DE0D594C794B794A79461
:10BF50008A95D1F7A092AE03B092AF03C092B0031E
:10BF6000D092B1036091EE027091EF025FE0603A0F
:10BF7000750750F58091E1039091E203A091E303EE
:10BF8000B091E4039C01AD010AE0569547953795C1
:10BF900027950A95D1F7821B930BA40BB50BA6012D
:10BFA000950114E0220F331F441F551F1A95D1F736
:10BFB000820F931FA41FB51F8093E1039093E203A8
:10BFC000A093E303B093E40360547F4118F580919C
:10BFD000E1039091E203A091E303B091E4039C019B
:10BFE000AD01FCE05695479537952795FA95D1F721
:10BFF000821B930BA40BB50BA6019501E2E0220F67
:10C00000331F441F551FEA95D1F7820F931FA41FBA
:10C01000B51F29C080913A0290913B0280913A026B
:10C0200090913B0297FF03C0909581959F4F843676
:10C0300091050CF58091E1039091E203A091E30357
:10C04000B091E4039C01AD017EE05695479537958C
:10C0500027957A95D1F7821B930BA40BB50B8A0D0C
:10C060009B1DAC1DBD1D8093E1039093E203A09343
:10C07000E303B093E4038091E1039091E203A09184
:10C08000E303B091E4036EE0B695A7959795879585
:10C090006A95D1F790930A038093090340911D0696
:10C0A000442399F055279C01BA010E94CD78C9011B
:10C0B000861B970B9093E0038093DF03260F371FB7
:10C0C0003093C0012093BF0119C01092E003109279
:10C0D000DF038FEF93E09093C0018093BF010EC008
:10C0E000109217031092E1031092E2031092E303FF
:10C0F0001092E40330930A03209309039091B6074A
:10C1000098AB292F3327220F331F220F331F285DAF
:10C110003F4FA8A1B9A12A173B0714F039A328A3C0
:10C12000B091EF07B9AB8B2F9927880F991F880F14
:10C13000991F80559040E8A1F9A18E179F0714F42C
:10C1400099A388A380917202882321F480917408B6
:10C150008F3FA1F08091EE029091EF020297C0977D
:10C1600068F4E8A0F9A01E141F0444F481E090E0F4
:10C170009093EF028093EE0239A328A308A119A19E
:10C180001093C3050093C2058091A6039091A70365
:10C19000A091A803B091A90322E0880F991FAA1FBC
:10C1A000BB1F2A95D1F7C090F007D090F107C81AAD
:10C1B000D90A013A11058CF0C80117FD0196959531
:10C1C00087958C159D050CF46C01909581959F4F7A
:10C1D000C816D90694F46C0110C011E5C116D1043B
:10C1E0001CF0E0E5CE2ED12C20EBC2162FEFD206AC
:10C1F00024F470EBC72E7FEFD72E49A9242F3327C5
:10C20000220F331F220F331FC90168A179A1861B9A
:10C21000970B8C159D050CF46C0188A199A1821BCC
:10C22000930BC816D9060CF46C018091B10790915C
:10C23000B20760911F0370912003861B970B9093A8
:10C24000C0078093BF07A090CE0720913D03309197
:10C250003E0340913F0350914003AA2041F0461A0B
:10C26000570AC201AA2797FDA095BA2F04C0AA2792
:10C2700097FDA095BA2F280F391F4A1F5B1F2093E7
:10C280003D0330933E0340933F035093400380911E
:10C290003D0390913E03A0913F03B0914003815034
:10C2A0009A4FA040B04064F080E09AEFA0E0B0E088
:10C2B00080933D0390933E03A0933F03B0934003CC
:10C2C00080913D0390913E03A0913F03B0914003C4
:10C2D00080509640AF4FBF4F64F480E096E0AFEFE0
:10C2E000BFEF80933D0390933E03A0933F03B09331
:10C2F0004003B0902C062B2D33278091BF079091DF
:10C30000C007289F7001299FF00C389FF00C112462
:10C310009701F7FE02C0295F3F4F790153E0F59482
:10C32000E7945A95E1F70091B1011091B20198019B
:10C33000442737FD4095542F80913D0390913E0353
:10C34000A0913F03B0914003BC01CD010E9402794E
:10C35000E20EF31E90909D01692D7727882799277B
:10C360009601D7FE04C0222733272C193D0937FF39
:10C3700002C02F5F3F4F3595279548A159A1240F43
:10C38000351F442737FD4095542F0E948E7897FF24
:10C3900004C0615C7F4F8F4F9F4F26E09595879536
:10C3A000779567952A95D1F79B016E157F050CF45B
:10C3B0007B01309521953F4FE216F3060CF479018D
:10C3C0008091A2079091A30760911D0370911E03B5
:10C3D000861B970B9093A1078093A00720913903A8
:10C3E00030913A0340913B0350913C03AA2041F025
:10C3F000261A370AC101AA2797FDA095BA2F04C0B3
:10C40000AA2797FDA095BA2F280F391F4A1F5B1F37
:10C410002093390330933A0340933B0350933C03FA
:10C420008091390390913A03A0913B03B0913C0372
:10C4300081509A4FA040B04064F080E09AEFA0E0B5
:10C44000B0E08093390390933A03A0933B03B093F9
:10C450003C038091390390913A03A0913B03B09142
:10C460003C0380509640AF4FBF4F64F480E096E0AD
:10C47000AFEFBFEF8093390390933A03A0933B0350
:10C48000B0933C032B2D33278091A0079091A107F7
:10C49000289FD001299FB00D389FB00D11249D0118
:10C4A000B7FF02C0295F3F4F5901B3E0B594A7948D
:10C4B000BA95E1F79801442737FD4095542F8091B4
:10C4C000390390913A03A0913B03B0913C03BC0126
:10C4D000CD010E940279A20EB31E692D772788270D
:10C4E00099279601D7FE04C0222733272C193D092E
:10C4F00037FF02C02F5F3F4F35952795E8A1F9A17F
:10C500002E0F3F1F442737FD4095542F0E948E78F1
:10C5100097FF04C0615C7F4F8F4F9F4FF6E095956A
:10C52000879577956795FA95D1F79B016A157B05F5
:10C530000CF45B01309521953F4FA216B3060CF425
:10C5400059012090FC02E0ED6E2EE6E07E2E77E8A9
:10C55000872E76E0972E6BE0362E5FEC452E57E067
:10C56000552ED4012C9112160CF0ECC0203419F485
:10C5700008A119A11EC0E8A1F9A1CF01AA2797FD22
:10C58000A095BA2F332727FD3095432F532FBC0199
:10C59000CD010E948E7897FF04C0615C7F4F8F4F62
:10C5A0009F4F46E095958795779567954A95D1F782
:10C5B0008B01F4012181203419F40E0D1F1D22C0BE
:10C5C000203C19F40E191F091DC0C701AA2797FDA9
:10C5D000A095BA2F332727FD3095432F532FBC0149
:10C5E000CD010E948E7897FF04C0615C7F4F8F4F12
:10C5F0009F4F36E095958795779567953A95D1F752
:10C60000060F171FF4012281203419F40A0D1B1D97
:10C6100022C0203C19F40A191B091DC0C501AA2714
:10C6200097FDA095BA2F332727FD3095432F532F21
:10C63000BC01CD010E948E7897FF04C0615C7F4FE2
:10C640008F4F9F4F26E095958795779567952A950B
:10C65000D1F7060F171FF4012381203419F40C0DB4
:10C660001D1D22C0203C19F40C191D091DC0C60156
:10C67000AA2797FDA095BA2F332727FD3095432F82
:10C68000532FBC01CD010E948E7897FF04C0615CDE
:10C690007F4F8F4F9F4FB6E095958795779567951C
:10C6A000BA95D1F7060F171FD2018D919C91801773
:10C6B00091075CF4BC01600F711F77FF02C06F5FD0
:10C6C0007F4F8B011595079511C0B1E0B21528F089
:10C6D000000F111F081B190B09C0222D3327801BC7
:10C6E000910BB9010E94CD78060F171FE8A98E2F74
:10C6F0009927880F991F880F991F8017910754F465
:10C70000F9A98F2F9927880F991F880F991F08174C
:10C7100019070CF08C01C80117FD039695958795B4
:10C7200095958795F3018183880F991F880F991F2D
:10C730009801281B390BC901880F8283D2010D9300
:10C740001C9303C0F301118212823A9402E010E0BC
:10C75000400E511E24E030E0820E931E48E050E06F
:10C76000640E751E37FEFDCEE2E1CB5C0C94397988
:10C770008091F4039091F503A091F603B091F70333
:10C780008093EC039093ED03A093EE03B093EF033B
:10C790008091F0039091F103A091F203B091F30323
:10C7A0008093E8039093E903A093EA03B093EB032B
:10C7B00008951092FF031092FE031092FD03109251
:10C7C000FC03089584B1806A84B93D9A82E58CBDEA
:10C7D0001DBC459A81E0809301088AEA8093120883
:10C7E00083E8809313088AE0809314081092160857
:10C7F00010921508109218081092170810926C08E1
:10C8000010923408089530910108332309F085C04F
:10C810000DB407FE82C084E080932202459A2EB5B3
:10C820008091030499278130910589F08230910528
:10C830001CF4892B21F03EC00297B9F03BC0309325
:10C840003308209304042138A9F581E008C0253578
:10C8500049F480910404820F8093040482E0809361
:10C86000030428C03093030425C080913308E82FC7
:10C87000FF27E15BF74F20838F5F80933308909110
:10C8800004048A31A0F0291769F48AE1AFE4B8E022
:10C89000E5E3F8E00D9001928A95E1F781E080935D
:10C8A000340802C0309334081092030403C0920F7E
:10C8B0009093040420911108203208F028C0459874
:10C8C0000000000000000000000000000000000068
:10C8D0000000000000000000000000000000000058
:10C8E0000000000000000000000000000000000048
:10C8F000E0910A08F0910B08E20FF11D80818EBDD6
:10C90000809131089081890F8093310803C081E0C4
:10C91000809301082F5F209311080895EF92FF92F2
:10C920000F931F93809125069927880F991F880FD1
:10C93000991F7C010027F7FC0095102F809175034B
:10C9400090917603A0917703B0917803BC01CD015B
:10C95000A80197010E9402793093160820931508C8
:10C9600080916D0390916E03A0916F03B09170035D
:10C97000BC01CD01A80197010E94027930931808EB
:10C98000209317082091F7073091F8074091F90795
:10C990005091FA07DA01C901E3E0880F991FAA1F35
:10C9A000BB1FEA95D1F7820F931FA41FB51F820FFB
:10C9B000931FA41FB51F20919701309198014091BA
:10C9C000990150919A01BC01CD010E9402793093E6
:10C9D0001E0820931D088091860390918703209163
:10C9E000480230914902821B930B90932408809354
:10C9F0002308E0917C03F0917D038091C60790911C
:10CA0000C707BF010E94CD78CB019B01220F331FC6
:10CA1000220F331F280F391F280F391F37FF02C07D
:10CA20002D5F3F4F359527953595279530931A08FB
:10CA3000209319088091F3079091F407BF010E9499
:10CA4000CD789B01220F331F220F331F260F371F74
:10CA5000260F371F37FF02C02D5F3F4F35952795B3
:10CA60003595279530931C0820931B0810927D0361
:10CA700010927C031092C7071092C6071092F40719
:10CA80001092F3078091140899278D30910509F4CD
:10CA900066C08E3091055CF48B30910509F48EC030
:10CAA0008C3091050CF00FC10A9761F0A8C18F304E
:10CAB000910509F47CC18F3091050CF45CC140975D
:10CAC00099F19DC180910203809325088091010313
:10CAD0008093260880910003809327088091FF02AD
:10CAE000809328088091FE02809329088091FD029E
:10CAF00080932A088091FC0280932B088091FB028E
:10CB000080932C088091ED0280932D088091ED0296
:10CB1000837F8093ED020E94852F80932E08809161
:10CB2000790380932F086BC180916E0890916F08F4
:10CB3000909326088093250880917208909173083D
:10CB4000909328088093270880911F0190912001DD
:10CB5000809329088091000180932A0850C1809118
:10CB60005706809325088091580680932608809167
:10CB700059068093270880915A068093280880914F
:10CB80005B068093290880915F0680932A08809134
:10CB9000600680932B088091610680932C08809119
:10CBA000640680932D088091620680932E08809100
:10CBB000630680932F0880916506DAC0F89480910F
:10CBC0000C06E82FFF27EE0FFF1FEF5CF84F0190D8
:10CBD000F081E02DE038F1051CF0EFE7F0E006C051
:10CBE0002FEFE138F20714F4E1E8FFEFE0932508B6
:10CBF00080910D06E82FFF27EE0FFF1FEF5CF84F27
:10CC00000190F081E02DE038F1051CF0EFE7F0E055
:10CC100006C06FEFE138F60714F4E1E8FFEFE093A8
:10CC2000260880910B06E82FFF27EE0FFF1FEF5C11
:10CC3000F84F0190F081E02DE038F1051CF0EFE7AE
:10CC4000F0E006C08FEFE138F80714F4E1E8FFEFF9
:10CC5000E093270880910A06E82FFF27EE0FFF1FB9
:10CC6000EF5CF84F0190F081E02DE038F1051CF009
:10CC7000EFE7F0E006C02FEFE138F20714F4E1E847
:10CC8000FFEF7894E093280880912203809329088D
:10CC90008091230380932A088091240380932B089A
:10CCA0008091250380932C088091260380932D0882
:10CCB0008091270380932E088091280380932F086A
:10CCC0008091290355C080916104863018F010923C
:10CCD000610485E08093250880916606809326088C
:10CCE0008091130390911403A0911503B091160342
:10CCF000BC01CD0125E030E040E050E00E94027927
:10CD0000309328082093270880910F0390911003F7
:10CD1000A0911103B0911203BC01CD0125E030E0D8
:10CD200040E050E00E94027930932A0820932908BD
:10CD300080915C0680932B0880915D0680932C087F
:10CD400080915E0680932D088091210380932E08A8
:10CD5000809131079091320780932F088091C2050E
:10CD60009091C30597FD0396959587959595879521
:10CD70008093300844C01092250880E580932608EF
:10CD800086E0809327088EE0809328088091020136
:10CD9000809329088091460480932A088091470453
:10CDA00080932B088091480480932C0828C08091A0
:10CDB0003E068093250880916B068093260880911B
:10CDC000A3018093270880913706809328088091DB
:10CDD0003806809329088091390680932A0880912B
:10CDE000A20180932B0880913B0680932C088091B0
:10CDF0003C0680932D0880913D0680932E088091FB
:10CE00003408882309F4CFC08AEF8093EA01409167
:10CE1000360850913708CA0181509E4F8F5F93406A
:10CE2000B0F42091380830913908C90181509E4FE3
:10CE30008F5F934060F48091160685FF08C0509381
:10CE4000FF034093FE033093FD032093FC03809186
:10CE50003C0890913D0821E08936920724F4909394
:10CE600034038093330380913303909134032091F2
:10CE7000310330913203821B930B845E9D4F68E631
:10CE800071E00E94CD78845B904090933003809352
:10CE90002F03209140083091410880912302909106
:10CEA00024028217930740F480916104882321F4BF
:10CEB00030932402209323028091350899278836E5
:10CEC000910549F18936910524F48736910531F0B1
:10CED00072C08936910509F445C06DC08091420841
:10CEE000809369088091430880936B08809144087F
:10CEF00080936A088091450880936C088091460869
:10CF000080936D08809147088093EB0180914808D9
:10CF10008093020450C08091420880930C08809155
:10CF2000430880930D088091440880930E088091F7
:10CF3000450880930F0880914608809310088091DF
:10CF4000B20590914708892B8093B20590914808CB
:10CF5000909300048091B30583709C70892B80931B
:10CF6000B30529C08091420880930208809143084C
:10CF700080930308809144088093040880914508B9
:10CF80008093050880914608909147089093070880
:10CF90008093060880914808909149089093090869
:10CFA0008093080808C01092FF031092FE031092AD
:10CFB000FD031092FC031F910F91FF90EF900895D5
:10CFC00080910108882309F43BC0459882E198E0EC
:10CFD00090930B0880930A0890910104E92FFF2792
:10CFE000EF51FE4F9F5F909301048081809314085E
:10CFF000993010F010920104109201080E948E6482
:10D0000081E0809311080000000000000000000093
:10D010000000000000000000000000000000000010
:10D020000000000000000000000000000000000000
:10D0300000000000000080911208809331088EBD2E
:10D04000089587B18C6087B942984398109206047E
:10D0500080E88093ED01109205048093EC0108951F
:10D0600080910B04815080930B048F3F09F0F4C032
:10D0700094E090930B048091ED02807BE1F080912D
:10D080005506882349F080910E04882311F490936B
:10D09000060481E080930E04809156068823B9F03F
:10D0A00080910F04882319F484E08093050481E0C3
:10D0B00080930F040CC080930E0480930F04809122
:10D0C000510680930C048091530680930D04809147
:10D0D0000E04882309F040C080916A06282F332768
:10D0E00024FF07C080911803882319F425FD4DC043
:10D0F0004EC090915206983F50F08091C8078D3DE8
:10D1000030F080910C0488230CF43FC040C0983F5D
:10D1100048F08091C8078A3028F480910C04882355
:10D12000B4F133C0809106048150809306048F3F90
:10D1300079F58091C8078150809306048091ED01B4
:10D14000813011F480E801C086958093ED018091D3
:10D15000ED0190910C0417C08091060481508093DA
:10D1600006048F3FA9F489E0809306048091ED01C5
:10D17000813011F480E801C086958093ED018091A3
:10D18000ED0190915506892311F0429A01C0429811
:10D1900080910F04882309F043C080916A06282FEC
:10D1A000332724FF07C080911803882319F426FD34
:10D1B00050C034C090915406983F50F08091EE07D3
:10D1C0008D3D30F080910D0488230CF442C026C0C0
:10D1D000983F48F08091EE078A3028F480910D0442
:10D1E0008823E4F036C080910504815080930504C3
:10D1F0008F3F91F58091EE078150809305048091D7
:10D20000EC01813011F480E801C086958093EC0137
:10D210008091EC0190910D048923D9F443980895ED
:10D22000809105048150809305048F3FA9F489E023
:10D23000809305048091EC01813011F480E801C0F5
:10D2400086958093EC018091EC019091560689239C
:10D2500011F0439A0895439808954FB724E130E0C0
:10D26000F8948091C9008F778093C9008091C9009C
:10D270008F7B8093C9008091C9008F7D8093C90006
:10D280005A9A52985B9A539A832F99278093CD008C
:10D290002093CC008091C80082608093C80080E118
:10D2A0008093C9008091CA008F778093CA008091D3
:10D2B000CA008F7B8093CA008091CA008F7D8093C3
:10D2C000CA008091CA008F7E8093CA008091CA00F4
:10D2D000877F8093CA008091C9008B7F8093C900AB
:10D2E0008091CA0084608093CA008091CA008260E5
:10D2F0008093CA008091C80087FF03C08091CE0050
:10D30000F9CF8091C90080688093C9004FBF08950C
:10D31000FF920F931F93CF93DF9380E197E20E94D8
:10D320009316EC01FF248091C9008F778093C90088
:10D330008091C9008F7E8093C9005A9889E39AE052
:10D340009F938F930CE612E11F930F93E0912D04AE
:10D35000F0912E0409950F900F900F900F9002C03E
:10D360004A996CC0CE010E949C168823C9F3E091B3
:10D370002D04F0912E04FF2009F468C08FE69AE096
:10D380009F938F931F930F930995529A0F900F902D
:10D390000F900F90CE010E949C168823D9F383E64C
:10D3A00090E05A9A019797FFFCCF8FE891E05A9846
:10D3B000019797FFFCCF89E090E05A9A019797FF79
:10D3C000FCCF89E090E05A98019797FFFCCF8FE857
:10D3D00091E05A9A019797FFFCCF8FE891E05A9815
:10D3E000019797FFFCCF89E090E05A9A019797FF49
:10D3F000FCCF89E090E05A98019797FFFCCF8FE827
:10D4000091E05A9A019797FFFCCF8FE891E05A98E4
:10D41000019797FFFCCF89E090E05A9A019797FF18
:10D42000FCCF89E090E05A98019797FFFCCF8FE8F6
:10D4300091E05A9A019797FFFCCF13C08AE590E0DC
:10D440000E949316EC0191E0F92E91CF85E79AE0C6
:10D450009F938F931F930F9309950F900F900F90A9
:10D460000F9052985A980E942D69E5E0CDB7DEB72B
:10D470000C944679EF92FF920F931F93CF93DF9313
:10D48000482F00E010E08091EE01813061F41092AD
:10D49000EE0184E48093100410921204109211049F
:10D4A000109213042BC180911004882319F421E0F9
:10D4B00030E001C0980190911104992371F4232B5D
:10D4C00011F081E010C084E4809310049093120462
:10D4D0009093110490931304FAC0913069F4232BB4
:10D4E00009F0EBC082E080931104809112048F5FF9
:10D4F0008093120483E0E9C09230D1F4232B09F029
:10D50000DCC083E0809310044093130490911204D4
:10D51000923039F41092140447FF03C081E08093E5
:10D52000140483E0809311049F5F90931204CFC092
:10D53000933009F0C2C0232B09F0BFC090931004B0
:10D5400082E080931104809112048F5F8093120413
:10D5500020911304822F9927782F6627842F9927EB
:10D56000682B792B80913006813049F47370CB01A0
:10D570008050924063E070E00E94CD7817C0823006
:10D5800061F47770CB018050944066E070E00E94B7
:10D59000CD782695269526950BC0737068567140F8
:10D5A000CB0177FD0196BC0175956795269526956B
:10D5B000022F11270F7010700F5F1F4F0D301105D4
:10D5C00008F074C07801E00EF11EF701EF5CF84F2F
:10D5D000808191819B01281B390BC90137FF03C052
:10D5E000909581959F4F069794F480912103883CF4
:10D5F00030F480912103865F8093210308C088EC7A
:10D600008093210380916F008F7D80936F00F701DD
:10D61000EF5CF84F808191819C01220F331F280F0E
:10D62000391F260F371F37FF02C02D5F3F4FE9011B
:10D63000D595C795D595C795CB0101968C179D07B4
:10D6400014F4219706C061507040C617D7070CF438
:10D65000219680912103843BD0F0F701EF5CF84FD5
:10D6600080819181FE01E81BF90BCF0163E070E03E
:10D670000E94CD78CB01880F991F860F971F25E652
:10D6800037E0E20EF31EF7019183808307C025E6A1
:10D6900037E0E20EF31EF70111821082000F111F16
:10D6A0000F5C184FF801D183C08311C002311105FE
:10D6B00070F081E08093EE010AC081E08093EE017A
:10D6C000109212041092140484E480931004809148
:10D6D0001204803198F080911404882331F48091F1
:10D6E000EE01882311F48093950110921204109298
:10D6F00014041092110484E480931004E6E0CDB782
:10D70000DEB70C944579CF93FC0197FF05C0CFEFAE
:10D71000F095E195FF4F01C0C1E028E631E0CF016F
:10D72000B9010E94CD78FC018B35910554F08B55E1
:10D7300090408A35910538F484EB90E08E1B9F0B66
:10D74000FC0141E00DC0CF01855B90408A35910519
:10D7500018F4E45BF04003C02E1B3F0BF9014FEFC0
:10D76000EE0FFF1FE058F54F259134918C2F99272C
:10D7700087FD9095289FB001299F700D389F700DEF
:10D780001124842F992787FD9095689FA001699F98
:10D79000500D789F500D1124CA01CF9108952AE5AC
:10D7A00030E0281B390BC9010E94836B0895CF9389
:10D7B000DF9380E00E94B87180911F019091200159
:10D7C0006AE070E00E94CD789F938F9380911F0153
:10D7D000909120016AE070E00E94CD787F936F9372
:10D7E0008EE49BE09F938F93CBEAD1E7DF93CF93B7
:10D7F000E0912D04F0912E0409952DB73EB7285FD6
:10D800003F4F2DBF8091EA018823B9F186E00E9445
:10D81000B87180910608909107086AE070E00E9454
:10D82000B9787F936F938FED90E09F938F93809162
:10D83000F7079091F807A091F907B091FA072091A6
:10D840009701309198014091990150919A01BC0142
:10D85000CD010E9402793F932F9387E59BE09F9330
:10D860008F93DF93CF93E0912D04F0912E040995CF
:10D870008DB79EB70A968DBF12C086E00E94B87120
:10D8800083E69BE09F938F93DF93CF93E0912D04EA
:10D89000F0912E0409950F900F900F900F908091AA
:10D8A00000048823C1F086E00E94B87180910004D2
:10D8B00099279F938F938AE69BE09F938F93DF93A3
:10D8C000CF93E0912D04F0912E0409952DB73EB72A
:10D8D0002A5F3F4F2DBF80E10E94B8718091F50112
:10D8E0009091F6016CE370E00E94B9789F938F935A
:10D8F0008091F5019091F6016CE370E00E94B97897
:10D900007F936F9380917208909173089F938F9388
:10D9100085E79BE09F938F93CBEAD1E7DF93CF938B
:10D92000E0912D04F0912E040995809116062DB7F3
:10D930003EB7265F3F4F2DBF80FF29C08AE10E947E
:10D94000B8718091960199279F938F9380911303CB
:10D9500090911403A0911503B0911603BC01CD0161
:10D9600024E630E040E050E00E9402793F932F939C
:10D9700082E89BE09F938F93DF93CF93E0912D04F8
:10D98000F0912E0409958DB79EB708968DBFDF9153
:10D99000CF910895CF93DF9380E00E94B87180917A
:10D9A000EF06992787FD90959F938F938091E706C7
:10D9B000992787FD90959F938F938091DF069927F4
:10D9C00087FD90959F938F938091D706992787FD28
:10D9D00090959F938F9389E89BE09F938F93CBEAD9
:10D9E000D1E7DF93CF93E0912D04F0912E040995B8
:10D9F00080E10E94B8712DB73EB7245F3F4F2DBF25
:10DA000080910F07992787FD90959F938F93809121
:10DA10000707992787FD90959F938F938091FF0625
:10DA2000992787FD90959F938F938091F70699276B
:10DA300087FD90959F938F9389E99BE09F938F93A8
:10DA4000DF93CF93E0912D04F0912E0409958091FE
:10DA500008062DB73EB7245F3F4F2DBF853098F4A1
:10DA600080E10E94B87189EA9BE09F938F93DF93D6
:10DA7000CF93E0912D04F0912E0409950F900F9013
:10DA80000F900F9018C08730B0F488E10E94B871F1
:10DA90008FED90E09F938F938AEB9BE09F938F9302
:10DAA000DF93CF93E0912D04F0912E0409958DB76B
:10DAB0009EB706968DBFDF91CF9108950F931F9368
:10DAC00080E00E94B8712AE030E080916E08909169
:10DAD0006F08B9010E94B9789F938F9380916E0867
:10DAE00090916F08B9010E94B9787F936F938091EC
:10DAF0001F0190912001B9010E94CD789F938F93CF
:10DB000080911F0190912001B9010E94CD787F93EF
:10DB10006F9383EC9BE09F938F930BEA11E71F9326
:10DB20000F93E0912D04F0912E04099580E10E945D
:10DB3000B8718DB79EB70C968DBF80917208909189
:10DB400073089F938F9380917008909171089F93B1
:10DB50008F9386ED9BE09F938F931F930F93E0919C
:10DB60002D04F0912E0409958DB79EB708968DBFB0
:10DB70001F910F9108950F931F93CF93DF9380917F
:10DB8000EA01CBEAD1E7882309F478C080E00E945B
:10DB9000B8718091030899279F938F93809105080E
:10DBA00099279F938F9382EE9BE09F938F938E0193
:10DBB000DF93CF93E0912D04F0912E0409958DB75A
:10DBC0009EB708968DBF80910408833031F48CE0B5
:10DBD0000E94B87181EF9BE005C08CE00E94B87193
:10DBE00086EF9BE09F938F93DF93CF93E0912D047B
:10DBF000F0912E0409950F900F900F900F90809147
:10DC0000020881FF12C08CE00E94B8718BEF9BE08C
:10DC10009F938F931F930F93E0912D04F0912E0407
:10DC200009950F900F900F900F9080E10E94B871AE
:10DC30008FED90E09F938F93809108089091090851
:10DC40009F938F9380910608909107086AE070E097
:10DC50000E94B9787F936F9380E09CE09F938F93AD
:10DC60008BEA91E79F938F93E0912D04F0912E041E
:10DC700009958DB79EB70A968DBF12C082E00E94AB
:10DC8000B87180E19CE09F938F93DF93CF93E091F5
:10DC90002D04F0912E0409950F900F900F900F9086
:10DCA000DF91CF911F910F910895CF93C82F2091AD
:10DCB00015042093160499278F32910509F18033BA
:10DCC00091051CF44F97A1F02CC08F34910501F100
:10DCD0008F38910531F5222319F481E090E038C0A6
:10DCE00086E0289FF0011124EA5CF44F849117C06C
:10DCF00086E0289FF0011124E95CF44F84910FC065
:10DD000086E0289FF0011124E85CF44F849107C05D
:10DD100086E0289FF0011124E75CF44F8491809302
:10DD2000150490911504809116049813C0E00E9488
:10DD3000BE719091150486E0989FF0011124E65C75
:10DD4000F44F259134918C2FF901099580E090E0F2
:10DD5000CF91089510926F0810926E081092730878
:10DD60001092720810927108109270081092740844
:10DD70008AE090E00E949316909318048093170411
:10DD80000895CF93DF9380911704909118040E9417
:10DD90009C16882309F4AFC0809117049091180451
:10DDA0000A969093180480931704E0E0F0E09F0136
:10DDB00090E05FEFA0EDB6E04BE0ED018B8187FFD7
:10DDC0000BC09F5F8D81E80FF11D8981280F311DE8
:10DDD0008E81851708F4582F4150189647FFEDCFD4
:10DDE00050937408232B41F520911D0430911E049B
:10DDF00040911F0450912004BB27A52F942F832FFF
:10DE000090931C0480931B04AA27BB27281B390B63
:10DE10004A0B5B0BCF01AA27BB27280F391F4A1FCC
:10DE20005B1F20931D0430931E0440931F045093E6
:10DE30002004E5E0F0E013C020911B0430911C04A5
:10DE40002E173F0718F4E21BF30B02C0E0E0F0E0EE
:10DE5000892F9927880F991FE80FF91F3596F0939E
:10DE60006F08E0936E08EF3FF10578F480911F0191
:10DE7000909120018E9F90018F9F300D9E9F300DBD
:10DE80001124C90164E670E013C0CF01969587950F
:10DE90009695879520911F0130912001289FA00120
:10DEA000299F500D389F500D1124CA0169E170E07F
:10DEB0000E94B978709371086093700820911904DA
:10DEC00030911A042E0F3F1F30931A042093190427
:10DED0005EE02131350778F08091720890917308E7
:10DEE0000196909373088093720820513E403093BE
:10DEF0001A0420931904DF91CF910895002422275A
:10DF00003327442751E0BB27EE27FF27A0E1660F08
:10DF1000771F881F991F001C221F331F441F660F85
:10DF2000771F881F991F001C221F331F441F2AF4CC
:10DF3000050E2B1F3E1F4F1F04C0051A2B0B3E0B57
:10DF40004F0B550FBB1FEE1F587F556047FD5250BA
:10DF5000AA95E9F6E695B7955795E695B79557953D
:10DF6000852F9B2F08952227332741E0552768E00E
:10DF7000880F991F221F331F880F991F221F331FDD
:10DF80001AF4240F351F02C0241B350B440F551FF4
:10DF9000487F456037FD42506A9551F75695479541
:10DFA00056954795842F0895AA2797FF04C080951A
:10DFB00090958A1F9A1F77FF04C0609570956A1F1D
:10DFC0007A1F669F9001779FA001679F300D411DCA
:10DFD0005A1F300D411D5A1F889FF001999F2E0F27
:10DFE0003F1F401D511D899F300D411D5A1F300D8F
:10DFF000411D5A1FCA01B901112480CF4FB720E437
:10E0000030E0F8948091C9008F778093C9008091A7
:10E01000C9008F7B8093C9008091C9008F7D809358
:10E02000C9005A9A52985B9A539A832F99278093E2
:10E03000CD002093CC008091C80082608093C800FE
:10E0400088E18093C9008091CA008F778093CA00CD
:10E050008091CA008F7B8093CA008091CA008F7D17
:10E060008093CA008091CA008F7E8093CA008091FD
:10E07000CA00877F8093CA008091C9008B7F8093FC
:10E08000C9008091CA0084608093CA008091CA0050
:10E0900082608093CA008091C80087FF03C080918E
:10E0A000CE00F9CF8091C90080688093C9004FBF2E
:10E0B00008950F931F93CF93DF93482F4F5F8931BC
:10E0C00008F089C080913007841710F4409330071E
:10E0D000CB0183539B4268E170E00E94CD78A42F6E
:10E0E000BB27FD01EA0FFB1FEF5CF84F8081918198
:10E0F0009B01281B390BC90137FF03C090958195FF
:10E100009F4F069794F480912103883C30F48091CE
:10E110002103865F8093210308C088EC809321034C
:10E1200080916F008F7D80936F00FD01EA0FFB1FD0
:10E13000EF5CF84F808191819C01220F331F280FE3
:10E14000391F260F371F37FF02C02D5F3F4FE901F0
:10E15000D595C795D595C795CB0101968C179D0789
:10E1600014F4219706C061507040C617D7070CF40D
:10E17000219680912103843BD8F08D010A0F1B1F4B
:10E18000F801EF5CF84F80819181FE01E81BF90BEB
:10E19000CF0163E070E00E94CD78CB01880F991F1A
:10E1A000860F971F0B59184FF8019183808307C082
:10E1B000AA0FBB1FAB59B84F11961C921E92E42FA9
:10E1C000FF27EE0FFF1FEF5CF84FD183C083443071
:10E1D00011F410929501DF91CF911F910F91089545
:10E1E000CF93DF9320917508822F9927807F9070BD
:10E1F000409709F06CC02F3109F046C08091760835
:10E200008093250420917808209327048091790831
:10E2100080932604822F99279093320780933107A9
:10E22000222309F054C080910A06282F3327220F99
:10E23000331FF901EB59F84F1182108280910B06C0
:10E24000A82FBB27AA0FBB1FFD01EB59F84F118266
:10E25000108280910D06E82FFF27EE0FFF1FCF01E0
:10E260008B59984FEC01198218822F5C384FE901C5
:10E2700019821882AF5CB84F11961C921E92EF5C07
:10E28000F84F1182108223C0C22FCF70CA30F8F429
:10E290008091760880939F088091770880939E08EC
:10E2A000809178088093A108809179088093A008D4
:10E2B00060919E0870919F088C2F0E945970609108
:10E2C000A0087091A1088C2F8F5F0E945970DF9178
:10E2D000CF910895CF93C82F8F3F49F480912804A0
:10E2E0008F3F29F410922A041092290432C0209101
:10E2F0002A04222339F4CF3111F485E001C084E0EF
:10E3000080932B0480912B04909129048217A0F410
:10E31000892F8095809329048F3F19F48EEF809385
:10E32000290480912904C81711F40E94F0701092FA
:10E330002A04109229040BC0E22FFF27EB58F74F55
:10E34000C0832F5F20932A049C0F90932904C093CD
:10E350002804CF91089590912404933240F4E92F3A
:10E36000FF27E558F74F80839F5F9093240408951B
:10E37000833218F48D5F80932404089590E2EEE7D1
:10E38000F8E08FE19193815087FFFCCF0895CF9300
:10E39000CFB723E031E0F8948091C9008F77809364
:10E3A000C9008091C9008F7B8093C9008091C9000A
:10E3B0008F7D8093C9005A9A52985B9A539A832F03
:10E3C00099278093CD002093CC008091C800826073
:10E3D0008093C80088E18093C9008091CA008F773C
:10E3E0008093CA008091CA008F7B8093CA0080917D
:10E3F000CA0080628093CA008091CA0080618093C5
:10E40000CA008091CA0088608093CA008091C900C8
:10E4100084608093C9008091CA0084608093CA00A0
:10E420008091CA0082608093CA008091C80087FFF3
:10E4300003C08091CE00F9CF8091C900806880939D
:10E44000C9008091C90080648093C9000E94BE7198
:10E45000CFBFCF910895282F99278F709070892B67
:10E4600031F4209580912304822B80932304089516
:10E470008091F101882309F441C08091ED0285FF6C
:10E480000AC082E980937B0883E280937C0885E55B
:10E4900080937D0802C010927B088091F2018F303A
:10E4A00071F4809123040E94556E882341F081E924
:10E4B00080937B0880937C0881E380937D08109291
:10E4C000F1018091C80085FFFCCF8091C9008F7E4B
:10E4D0008093C9008091C9008E7F8093C90080918C
:10E4E0007B08882311F48EEF01C08EE78093CE0065
:10E4F000809123048093F2011092230408951F92C7
:10E500000F920FB60F9211248F939F93EF93FF9367
:10E510009091F101992309F040C080912C04882347
:10E5200061F480917B08882311F483E003C0813972
:10E5300099F481E080932C040FC0833099F480918A
:10E540007B08882349F090937B088091C9008E7FD7
:10E550008093C9008EEF1EC08091C90081608093B6
:10E56000C9000EC0833261F48091C9008E7F809310
:10E57000C9008FEF8093CE0081E08093F10114C039
:10E5800080912C04E82FFF27E558F74F8F5F809389
:10E590002C0480818093CE0007C010922C048091BF
:10E5A000C90080618093C900FF91EF919F918F9185
:10E5B0000F900FBE0F901F901895EF92FF920F9340
:10E5C0001F93CF93DF937C018B01EA01452B39F038
:10E5D000F80181918F01F70109952197C9F7E6E0CC
:10E5E000CDB7DEB70C944579EF92FF920F931F934E
:10E5F000CF93DF937C018B01EA01452B41F0F801B9
:10E600000F5F1F4F8491F70109952197C1F7E6E04D
:10E61000CDB7DEB70C9445790F931F93CF938C0140
:10E62000C62F161634F480E2F8010995C1501C1665
:10E63000D4F3CF911F910F9108950F931F93CF9310
:10E640008C01C62F161634F480E3F8010995C150E9
:10E650001C16D4F3CF911F910F910895A5E3B0E05C
:10E66000E4E3F3E70C941D792E96EEADFFAD2E9703
:10E6700088249924540180912204882321F42C9623
:10E680001FAE1EAE2C975EE4452E512C4C0E5D1E27
:10E690006F01B60105C0153239F00894C11CD11CB8
:10E6A000F60114911123B9F7A601461B570B31F05F
:10E6B0002C968EAD9FAD2C970E94F472112309F415
:10E6C0006AC20894C11CD11CFF24FDA6FCA64FEF12
:10E6D000E42EF9A6F6010894C11CD11C149115373B
:10E6E00021F0812F80628837B1F4F0FE0AC0F20178
:10E6F00024E030E0420E531E80809180A280B380DF
:10E700000AC0F20142E050E0440E551E8081918122
:10E710004C01AA24BB24103221F489A58823D1F608
:10E720001DC0133219F458E0F52AD4CF1A3211F073
:10E730001D3291F41A3259F4F20182E090E0480E51
:10E74000591EE081ECA7EE232CF6E195ECA790E1B1
:10E75000F92AAFEDFA22BECF1B3211F419A7BACFB6
:10E760001E32C1F5F6010894C11CD11C14911A3255
:10E7700079F4F20122E030E0420E531E40815181D3
:10E780003FEF4F3F530714F44FEF5FEFE42EA2CF5C
:10E7900040E050E0812F80538A30A0F4CA0133E07A
:10E7A000880F991F3A95E1F7840F951F480F591F5D
:10E7B000410F511D40535040F6010894C11CD11C1B
:10E7C0001491E8CF8FEF4F3F580714F44FEF5FEFEE
:10E7D000E42E85CF103329F4F4FC7CCF90E2F92AA3
:10E7E00079CF812F81538930D8F440E050E0CA01BD
:10E7F00023E0880F991F2A95E1F7840F951F480F92
:10E80000591F410F511D40535040F6010894C11C3F
:10E81000D11C1491812F80538A3048F34CA75FCFCD
:10E82000183619F4A4E0FA2A55CF1C3619F4B1E0D1
:10E83000FB2A50CF133661F43E010894611C711C11
:10E84000F20122E030E0420E531E808189833CC1F8
:10E85000143421F0143611F0193651F5143411F432
:10E8600031E0F32AF0FE0AC0F20144E050E0440E29
:10E87000551E80809180A280B3800CC0F20182E09E
:10E8800090E0480E591E808191814C01AA2497FC8A
:10E89000A094BA2CB7FE0AC0B094A094909480942F
:10E8A000811C911CA11CB11C8DE289A70AE06FC0DC
:10E8B0001F3411F01F3631F41F3411F491E0F92A9E
:10E8C00008E064C0103779F4F201A2E0B0E04A0E2B
:10E8D0005B1E808191814C01AA24BB2400E1B0E43D
:10E8E000FB2A18E753C01337C1F5F20122E030E0EC
:10E8F000420E531E608071806114710489F43E01E0
:10E900000894611C711C88E289838EE6F30181837F
:10E9100085E78B838CE68C838D8389E28E831F82CF
:10E92000E7FC13C08E2D992787FD9095AC0160E020
:10E9300070E0C3010E94C977009729F0382E36187D
:10E94000E3140CF0C3C03E2CC1C0F30101900020C1
:10E95000E9F731973E2E3618B9C0153511F0153745
:10E9600031F4153511F4F1E0FF2A0AE00FC0183533
:10E9700019F0183709F0A0C000E1F3FE07C08114B8
:10E980009104A104B10411F020E4F22A19A6EDA625
:10E99000E7FC02C03FEDF32289E2682E712C6C0E79
:10E9A0007D1E81149104A104B10421F44DA54423DA
:10E9B00009F47BC0802F9927AA27BB278EA79FA782
:10E9C000A8ABB9AB202E332490E0891690E09906CD
:10E9D00091E0A90690E0B90648F0C501B4012EA562
:10E9E0003FA548A959A90E94E07817C0AFEF8A1641
:10E9F0009104A104B10449F040F0C401B1010E94A6
:10EA0000B9789B014427552708C0882D602F0E94A4
:10EA1000AD78282F3327442755272AAB3BAB4CAB87
:10EA20005DAB0A3059F48AA9880F880F880F9AA91C
:10EA3000990F890F382D381B832F10C0003139F4FE
:10EA40008AA98295807F482D481B842F07C08AA9F8
:10EA5000880F880F880F582D581B852F90E02EA502
:10EA60003FA548A959A982169306A406B50608F041
:10EA700091E08AA89BA8ACA8BDA88A3010F4805D5C
:10EA800004C0895A183509F48F7DD3018E933D0156
:10EA9000992309F099CF083041F4F3FE06C0803382
:10EAA00021F080E3FD0182933F01CE010196382ED3
:10EAB0003618F8E23F0E0BC0112309F46CC03E017A
:10EAC0000894611C711C1983B1E03B2E19A6032D1B
:10EAD0002DA4231827FC222489A5882311F00F5F79
:10EAE00002C0F6FC0E5F020DEF2CFF24C7018073FD
:10EAF0009070892B49F48CA5801B682F2C968EADC5
:10EB00009FAD2C970E940C7389A5882331F041E0BA
:10EB100050E0BE01675D7F4F0AC0E6FE0EC080E395
:10EB20008AA71BA742E050E0BE01665D7F4F2C968E
:10EB30008EAD9FAD2C970E94DD72C70180739070DF
:10EB4000809749F48CA5801B682F2C968EAD9FADC5
:10EB50002C970E941D73622D2C968EAD9FAD2C9725
:10EB60000E941D73832D992787FD9095AC01B301F9
:10EB70002C968EAD9FAD2C970E94DD72E4FE89CD60
:10EB80002CA5201B2CA7622F2C968EAD9FAD2C9709
:10EB90000E940C737ECDE2E1CB5C0C9439792FB7E7
:10EBA00040E0F894E0E0F0E081E280935700949137
:10EBB000E2E0F0E0809357003491E4E0F0E08093ED
:10EBC000570084912FBF9E3199F4363941F4893032
:10EBD00011F441E00DC08A3059F442E009C03739E0
:10EBE00039F4863011F443E003C0853009F444E081
:10EBF000842F992708959FB7F8948091C900877F43
:10EC00008093C9008091C9008F7E8093C900809154
:10EC1000C9008F778093C9008091C9008F7B809352
:10EC2000C9008091C9008F7D8093C90052985A9A7B
:10EC300053985B9A9FBF08951F93CF93DF93182F2C
:10EC400080912204882309F48DC08091F001181767
:10EC500009F488C080912104882321F40E94CF7593
:10EC60008093210489E09DE09F938F93CCE6D2E1CD
:10EC7000DF93CF93E0912D04F0912E0409950F902E
:10EC80000F900F900F90812F99278230910501F1FD
:10EC9000833091052CF4009761F0019769F024C04E
:10ECA00084309105D9F084309105ACF00597C9F016
:10ECB0001BC089EF9CE002C087EE9CE09F938F937E
:10ECC000DF93CF93E0912D04F0912E04099518C0A5
:10ECD0008EEC9CE0F3CF8BEA9CE0F0CF8DE99CE0DA
:10ECE000EDCF85E99CE0EACF86E19DE09F938F938D
:10ECF000DF93CF93E0912D04F0912E04099510E05D
:10ED00000F900F900F900F9080912104843011F09C
:10ED1000823099F40E94FB75812F8150833018F462
:10ED20000E942D691DC0143019F40E94C77118C0CB
:10ED30001530B1F40E94FE6F13C0112389F08CE2EC
:10ED40009DE09F938F938CE692E19F938F93E09148
:10ED50002D04F0912E0409950F900F900F900F90B5
:10ED60001093F001DF91CF911F9108950F931F939E
:10ED700081E0809322044091EF01E5E4FCE020E093
:10ED800030E05FE4849199272F5F3F4F829FB0016D
:10ED9000839F700D929F700D11244627515031961C
:10EDA00057FFF0CF4093EF01EDE1FCE020E030E0D1
:10EDB00057E2849199272F5F3F4F829FB001839F35
:10EDC000700D929F700D112446275150319657FFB8
:10EDD000F0CF4093EF0180912104882321F40E9419
:10EDE000CF75809321048091EF01833459F088E13D
:10EDF00090E029E20FB6F894A895809360000FBECA
:10EE0000209360008EE293E790932E0480932D046C
:10EE100087E49DE09F938F930CE612E11F930F937D
:10EE2000E0912D04F0912E0409950F900F900F9012
:10EE30000F9087E690E09F938F9380E590E09F93FB
:10EE40008F931F921F92809102016AE00E94AD7819
:10EE5000892F99279F938F93809102010E94AD780B
:10EE600099279F938F938DE69DE09F938F931F9398
:10EE70000F93E0912D04F0912E04099585E49CE018
:10EE80009F938F931F930F93E0912D04F0912E0485
:10EE900009958DE19CE09F938F931F930F93E091D1
:10EEA0002D04F0912E0409958DB79EB746968DBF1F
:10EEB00081EA9DE09F938F931F930F93E0912D0420
:10EEC000F0912E04099583EC8093810080916F006E
:10EED000806280936F000F900F900F900F901F91A2
:10EEE0000F91089580912204882361F08091F001B0
:10EEF000843011F40E9438728091EF01833411F054
:10EF00001092220408951F920F920FB60F921124AF
:10EF10002F933F934F935F936F937F938F939F9321
:10EF2000AF93BF93EF93FF932091CE009091F001A8
:10EF3000892F8150833020F4822F0E943A6A0BC0BF
:10EF4000943021F4822F0E942B7205C0953019F461
:10EF5000822F0E946A71FF91EF91BF91AF919F91B3
:10EF60008F917F916F915F914F913F912F910F9072
:10EF70000FBE0F901F901895FB01DC0140FF05C0EC
:10EF800002C005900D9205900D9242505040C8F776
:10EF90000895FC014150504030F001900616D1F721
:10EFA0003197CF0108958827992708955058192E31
:10EFB00084D001D06AC0BA17620773078407950727
:10EFC000B1F188F40EF410940B2EBA2FA02D062E5A
:10EFD000622F202D072E732F302D082E842F402DC9
:10EFE000092E952F502DFF275523B9F0591B49F0B5
:10EFF000573E98F0469537952795A795F04053953D
:10F00000C9F776F0BA0F621F731F841F30F487951B
:10F0100077956795B795F040939517FA0F2E089559
:10F02000BF1BBB27BA0B620B730B840BF6CFDEF64C
:10F0300070C097FB4ED09F3738F0FEE9F91B982F30
:10F04000872F762F6B2F05C061C096958795779592
:10F050006795F150D0F73EF4909580957095619545
:10F060007F4F8F4F9F4F0895E89403C097FB0EF496
:10F07000F3DFB62F672F782F892F9EE9002405C074
:10F080009A95BB0F661F771F881F11249923A1F043
:10F090008823B2F79F3F59F0BB0F48F421F40020BA
:10F0A00011F460FF04C06F5F7F4F8F4F9F4F881F29
:10F0B0009795879597F9089529C0052E092607FA8F
:10F0C000440F551F5F3F79F0AA27A51708F051E0BC
:10F0D0004795880F991F9F3F31F0BB27B91708F05C
:10F0E00091E0879508959F919F91112414C097FBFB
:10F0F000880F991F9F3F31F0BB27B91708F091E0A7
:10F10000879508959F919F91112405C066277727C1
:10F110008827992708959FEF80EC0895629FD0017A
:10F12000739FF001829FE00DF11D649FE00DF11DC2
:10F13000929FF00D839FF00D749FF00D659FF00D71
:10F140009927729FB00DE11DF91F639FB00DE11D5E
:10F15000F91FBD01CF0111240895991B79E004C066
:10F16000991F961708F0961B881F7A95C9F7809506
:10F170000895AA1BBB1B51E107C0AA1FBB1FA617FE
:10F18000B70710F0A61BB70B881F991F5A95A9F750
:10F1900080959095BC01CD01089597FB092E072617
:10F1A0000AD077FD04D0E5DF06D000201AF4709570
:10F1B00061957F4F0895F6F7909581959F4F08953B
:10F1C000A1E21A2EAA1BBB1BFD010DC0AA1FBB1F6B
:10F1D000EE1FFF1FA217B307E407F50720F0A21BDD
:10F1E000B30BE40BF50B661F771F881F991F1A944A
:10F1F00069F760957095809590959B01AC01BD0174
:10F20000CF01089597FB092E05260ED057FD04D097
:10F21000D7DF0AD0001C38F45095409530952195E1
:10F220003F4F4F4F5F4F0895F6F79095809570953B
:10F2300061957F4F8F4F9F4F08952F923F924F922E
:10F240005F926F927F928F929F92AF92BF92CF9276
:10F25000DF92EF92FF920F931F93CF93DF93CDB77F
:10F26000DEB7CA1BDB0B0FB6F894DEBF0FBECDBFF7
:10F2700009942A88398848885F846E847D848C84C8
:10F280009B84AA84B984C884DF80EE80FD800C81D1
:10F290001B81AA81B981CE0FD11D0FB6F894DEBFB4
:10F2A0000FBECDBFED010895EE0FFF1F0590F49145
:10F2B000E02D0994F999FECFB2BDA1BDF89A11963F
:10F2C00000B40895F7DF01921A94E1F70895F2DF90
:10F2D000E02DF0DFF02D0895F999FECFB2BDA1BD6C
:10F2E00000BC11960FB6F894FA9AF99A0FBE0895D9
:10F2F000F3DF012CF1DF112408950190EDDF1A9462
:04F30000E1F7089594
:10F304005E010A010164FF01FFFF140001FC01FC1E
:10F314000101737373FF03007D0000C409C4096411
:10F32400001148656C6C6F20576F726C64000000AC
:10F3340000000000000000000000000000000000C9
:10F3440000000000000000000000000000000000B9
:10F3540000000000000000000000000000000000A9
:10F364000000000000000000000000000000000099
:10F37400000053706F727400004E6F726D616C0008
:10F3840000426567696E6E65720000517561647252
:10F394006F0000640001200B050000ECFF64404195
:10F3A4005A4664640A02969696960840403A10FBC0
:10F3B40030380190D0030090D00300F4017800FFAE
:10F3C400036400020406070808080706040200FE96
:10F3D400FCFAF9F8F8F8F9FAFCFE0002040607084A
:10F3E400080B0A0D0B0C0E0B0F10FA200101017013
:04F3F400FF010F0006
:00000001FF
